 CryLiveCreate

 Timestamp is 5036e4af (Fri Aug 24 04:19:27 2012)

 Preferred load address is 0000000037500000

 Start         Length     Name                   Class
 0001:00000000 0001d5a5H .text                   CODE
 0001:0001d5b0 00000092H .text$x                 CODE
 0001:0001d650 00000110H .text$yc                CODE
 0001:0001d760 000002b5H .text$yd                CODE
 0002:00000000 00000380H .idata$5                DATA
 0002:00000380 00000008H .CRT$XCA                DATA
 0002:00000388 00000058H .CRT$XCU                DATA
 0002:000003e0 00000008H .CRT$XCZ                DATA
 0002:000003e8 00000008H .CRT$XIA                DATA
 0002:000003f0 00000008H .CRT$XIAA               DATA
 0002:000003f8 00000008H .CRT$XIZ                DATA
 0002:00000400 00003ef8H .rdata                  DATA
 0002:000042f8 00000058H .rdata$debug            DATA
 0002:00004350 00000000H .rdata$r                DATA
 0002:00004350 00000008H .rtc$IAA                DATA
 0002:00004358 00000008H .rtc$IZZ                DATA
 0002:00004360 00000008H .rtc$TAA                DATA
 0002:00004368 00000008H .rtc$TZZ                DATA
 0002:00004370 00001aecH .xdata                  DATA
 0002:00005e5c 00000020H .didat$2                DATA
 0002:00005e7c 00000020H .didat$3                DATA
 0002:00005ea0 00000078H .didat$4                DATA
 0002:00005f18 000000e8H .didat$6                DATA
 0002:00006000 00000078H .didat$7                DATA
 0002:00006078 00000050H .idata$2                DATA
 0002:000060c8 00000014H .idata$3                DATA
 0002:000060e0 00000380H .idata$4                DATA
 0002:00006460 0000060cH .idata$6                DATA
 0002:00006a70 000000adH .edata                  DATA
 0003:00000000 000001e8H .data                   DATA
 0003:000001e8 00000078H .didat$5                DATA
 0003:00000260 000019b8H .bss                    DATA
 0004:00000000 00001b24H .pdata                  DATA
 0005:00000000 00000008H .tls$                   DATA

  Address         Publics by Value              Rva+Base               Lib:Object

 0000:00000000       ___safe_se_handler_table   0000000000000000     <absolute>
 0000:00000000       ___safe_se_handler_count   0000000000000000     <absolute>
 0000:00000000       __ImageBase                0000000037500000     <linker-defined>
 0001:00000000       ??0PS3TargetInfo@@QEAA@XZ  0000000037501000 f   PS3TmHelperLib:PS3TmHelper.obj
 0001:000000e0       ?SNPS3FTPEvenCallback@@YAXHIIJIPEAEPEAX@Z 00000000375010e0 f   PS3TmHelperLib:PS3TmHelper.obj
 0001:000001c0       ?SNPS3EnumerateTargetsCallback@@YAHHPEAX@Z 00000000375011c0 f   PS3TmHelperLib:PS3TmHelper.obj
 0001:00000400       ??0PS3TmHelper@@QEAA@XZ    0000000037501400 f   PS3TmHelperLib:PS3TmHelper.obj
 0001:00000460       ?Initialize@PS3TmHelper@@QEAA_NXZ 0000000037501460 f   PS3TmHelperLib:PS3TmHelper.obj
 0001:000004b0       ?ConnectTo@PS3TmHelper@@QEAA_NAEAUPS3TargetInfo@@@Z 00000000375014b0 f   PS3TmHelperLib:PS3TmHelper.obj
 0001:000004f0       ?IsPoweredOn@PS3TmHelper@@QEAA_NAEAUPS3TargetInfo@@@Z 00000000375014f0 f   PS3TmHelperLib:PS3TmHelper.obj
 0001:00000540       ?FillTargetAddress@PS3TmHelper@@QEAA_NAEAUPS3TargetInfo@@@Z 0000000037501540 f   PS3TmHelperLib:PS3TmHelper.obj
 0001:00000680       ?Launch@PS3TmHelper@@QEAA_NAEBUPS3TargetInfo@@PEBD11@Z 0000000037501680 f   PS3TmHelperLib:PS3TmHelper.obj
 0001:000008a0       ?Reset@PS3TmHelper@@QEAA_NAEBUPS3TargetInfo@@_N@Z 00000000375018a0 f   PS3TmHelperLib:PS3TmHelper.obj
 0001:00000910       ?MakeDir@PS3TmHelper@@QEAAJAEAUPS3TargetInfo@@PEBD@Z 0000000037501910 f   PS3TmHelperLib:PS3TmHelper.obj
 0001:00000990       ?CopyFileTo@PS3TmHelper@@QEAA_NAEAUPS3TargetInfo@@PEBD1@Z 0000000037501990 f   PS3TmHelperLib:PS3TmHelper.obj
 0001:00000b00       ?CopyFileFrom@PS3TmHelper@@QEAA_NAEAUPS3TargetInfo@@PEBD1@Z 0000000037501b00 f   PS3TmHelperLib:PS3TmHelper.obj
 0001:00000c30       ?DeleteFileA@PS3TmHelper@@QEAA_NAEAUPS3TargetInfo@@PEBD@Z 0000000037501c30 f   PS3TmHelperLib:PS3TmHelper.obj
 0001:00000c30       ?DeleteFolder@PS3TmHelper@@QEAA_NAEAUPS3TargetInfo@@PEBD@Z 0000000037501c30 f   PS3TmHelperLib:PS3TmHelper.obj
 0001:00000cc0       ?GetDirectoryList@PS3TmHelper@@QEAA_NAEAUPS3TargetInfo@@PEBDAEAHPEAUPS3DirEntryEx@@@Z 0000000037501cc0 f   PS3TmHelperLib:PS3TmHelper.obj
 0001:00000e40       ?Instance@PS3TmDynApi@@SAPEAV1@XZ 0000000037501e40 f   PS3TmHelperLib:PS3TmDynApi.obj
 0001:00000ec0       ?Initialize@PS3TmDynApi@@AEAA_NXZ 0000000037501ec0 f   PS3TmHelperLib:PS3TmDynApi.obj
 0001:00001340       ??0CryLock_WinMutex@@QEAA@XZ 0000000037502340 f   CryLiveCreate.obj
 0001:00001370       ??1CryLock_WinMutex@@QEAA@XZ 0000000037502370 f   CryLiveCreate.obj
 0001:00001380       ?Lock@CryLock_WinMutex@@QEAAXXZ 0000000037502380 f   CryLiveCreate.obj
 0001:00001390       ?Unlock@CryLock_WinMutex@@QEAAXXZ 0000000037502390 f   CryLiveCreate.obj
 0001:000013a0       ??0CryConditionVariable@@QEAA@XZ 00000000375023a0 f   CryLiveCreate.obj
 0001:000013f0       ??1CryConditionVariable@@QEAA@XZ 00000000375023f0 f   CryLiveCreate.obj
 0001:00001420       ??0CrySimpleThreadSelf@@QEAA@XZ 0000000037502420 f   CryLiveCreate.obj
 0001:00001440       ?WaitForThread@CrySimpleThreadSelf@@QEAAXXZ 0000000037502440 f   CryLiveCreate.obj
 0001:00001470       ??1CrySimpleThreadSelf@@UEAA@XZ 0000000037502470 f   CryLiveCreate.obj
 0001:000014a0       ?StartThread@CrySimpleThreadSelf@@IEAAXP6AIPEAX@Z0@Z 00000000375024a0 f   CryLiveCreate.obj
 0001:000014f0       ?CryThreadSetName@@YAXIPEBD@Z 00000000375024f0 f   CryLiveCreate.obj
 0001:00001560       ?Init@_CryMemoryManagerPoolHelper@@SAXXZ 0000000037502560 f i CryLiveCreate.obj
 0001:00001760       ?CryGetIMemoryManager@@YAPEAUIMemoryManager@@XZ 0000000037502760 f   CryLiveCreate.obj
 0001:000017b0       ?CryInterlockedDecrement@@YAJPECH@Z 00000000375027b0 f   CryLiveCreate.obj
 0001:000017c0       ?CryCreateCriticalSectionInplace@@YAXPEAX@Z 00000000375027c0 f   CryLiveCreate.obj
 0001:000017d0       DllMain                    00000000375027d0 f   CryLiveCreate.obj
 0001:000017e0       ?destroy@sp_counted_base@detail@boost@@UEAAXXZ 00000000375027e0 f   CryLiveCreate.obj
 0001:000017e0       DeleteLiveCreate           00000000375027e0 f   CryLiveCreate.obj
 0001:00001800       ?CryFatalError@@YAXPEBDZZ  0000000037502800 f i CryLiveCreate.obj
 0001:000018a0       ?AddLabelFmt@CDummyMemReplay@@UEAAXPEBDZZ 00000000375028a0 f i CryLiveCreate.obj
 0001:000018b0       ?ClearFileSyncQueue@CNullManager@LiveCreate@@UEAAXXZ 00000000375028b0 f i LiveCreate.obj
 0001:000018b0       ?Flush@CDummyMemReplay@@UEAAXXZ 00000000375028b0 f i CryLiveCreate.obj
 0001:000018b0       ?OnPeerConnected@CameraController@LiveCreate@@UEAAXPEAUSPeerLink@2@@Z 00000000375028b0 f i LiveCreateCtrl_Camera.obj
 0001:000018b0       ?MarkBucket@CDummyMemReplay@@UEAAXH_KPEAX0@Z 00000000375028b0 f i CryLiveCreate.obj
 0001:000018b0       ?UnMapPage@CDummyMemReplay@@UEAAXPEAX_K@Z 00000000375028b0 f i CryLiveCreate.obj
 0001:000018b0       ?SetCustomPlatformName@CNullManager@LiveCreate@@UEAAXPEBD@Z 00000000375028b0 f i LiveCreate.obj
 0001:000018b0       ?OnFileUploadEnd@IObserver@FileSyncManager@LiveCreate@@UEAAXPEBD_N@Z 00000000375028b0 f i LiveCreate.obj
 0001:000018b0       ?UnregisterContainer@CDummyMemReplay@@UEAAXPEBX@Z 00000000375028b0 f i CryLiveCreate.obj
 0001:000018b0       ?UnbindFromContainer@CDummyMemReplay@@UEAAXPEBX0@Z 00000000375028b0 f i CryLiveCreate.obj
 0001:000018b0       ?SetLogEnabled@CNullManager@LiveCreate@@UEAAX_N@Z 00000000375028b0 f i LiveCreate.obj
 0001:000018b0       ?OnBeginSendToPeers@CameraController@LiveCreate@@UEAAXXZ 00000000375028b0 f i LiveCreateCtrl_Camera.obj
 0001:000018b0       ?AddSizerTree@CDummyMemReplay@@UEAAXPEBD@Z 00000000375028b0 f i CryLiveCreate.obj
 0001:000018b0       ?OnBeginSendToPeers@FileChangeNotifyController@LiveCreate@@UEAAXXZ 00000000375028b0 f i LiveCreateCtrl_FileChangeNotify.obj
 0001:000018b0       ?UnMarkBucket@CDummyMemReplay@@UEAAXHPEAX@Z 00000000375028b0 f i CryLiveCreate.obj
 0001:000018b0       ?OnBeginSendToPeers@EntitiesController@LiveCreate@@UEAAXXZ 00000000375028b0 f i LiveCreateCtrl_Entities.obj
 0001:000018b0       ?OnRegistered@CommonController@LiveCreate@@UEAAXPEAUIManager@2@@Z 00000000375028b0 f i LiveCreateCtrl_Common.obj
 0001:000018b0       ?OnUnregistered@CommonController@LiveCreate@@UEAAXPEAUIManager@2@@Z 00000000375028b0 f i LiveCreateCtrl_Common.obj
 0001:000018b0       ?StartOnCommandLine@CDummyMemReplay@@UEAAXPEBD@Z 00000000375028b0 f i CryLiveCreate.obj
 0001:000018b0       ?ExitScope_Free@CDummyMemReplay@@UEAAX_K@Z 00000000375028b0 f i CryLiveCreate.obj
 0001:000018b0       ?Start@CDummyMemReplay@@UEAAX_NPEBD@Z 00000000375028b0 f i CryLiveCreate.obj
 0001:000018b0       ?SyncModifiedFile@CNullManager@LiveCreate@@UEAAXPEBD0H0@Z 00000000375028b0 f i LiveCreate.obj
 0001:000018b0       ?OnSystemEvent@CSystemEventListner_LiveCreate@@UEAAXW4ESystemEvent@@_K1@Z 00000000375028b0 f i CryLiveCreate.obj
 0001:000018b0       ?OnFileUploadStart@IObserver@FileSyncManager@LiveCreate@@UEAAXPEBD@Z 00000000375028b0 f i LiveCreate.obj
 0001:000018b0       ?EndScanFolder@PlatformHandlerBase@LiveCreate@@UEAAXPEAX@Z 00000000375028b0 f i PlatformHandlerBase.obj
 0001:000018b0       ?Terminate@?$CrySimpleThread@VNetPeerServerAcceptThread@LiveCreate@@@@MEAAXXZ 00000000375028b0 f i LiveCreateNetwork.obj
 0001:000018b0       ?AddFrameStart@CDummyMemReplay@@UEAAXXZ 00000000375028b0 f i CryLiveCreate.obj
 0001:000018b0       ?UnMarkPool@CDummyMemReplay@@UEAAXHPEAX@Z 00000000375028b0 f i CryLiveCreate.obj
 0001:000018b0       ?OnBeginSendToPeers@CVarController@LiveCreate@@UEAAXXZ 00000000375028b0 f i LiveCreateCtrl_CVar.obj
 0001:000018b0       ?AddContextV@CDummyMemReplay@@UEAAXHIPEBDPEAD@Z 00000000375028b0 f i CryLiveCreate.obj
 0001:000018b0       ?GetInfo@CDummyMemReplay@@UEAAXAEAUCryReplayInfo@@@Z 00000000375028b0 f i CryLiveCreate.obj
 0001:000018b0       ?Stop@CDummyMemReplay@@UEAAXXZ 00000000375028b0 f i CryLiveCreate.obj
 0001:000018b0       ?OnPeerConnected@CommonController@LiveCreate@@UEAAXPEAUSPeerLink@2@@Z 00000000375028b0 f i LiveCreateCtrl_Common.obj
 0001:000018b0       ?RegisterContainer@CDummyMemReplay@@UEAAXPEBXH@Z 00000000375028b0 f i CryLiveCreate.obj
 0001:000018b0       ?Cancel@CryRunnable@@UEAAXXZ 00000000375028b0 f i LiveCreateFileSync.obj
 0001:000018b0       ?AddTexturePoolContext@CDummyMemReplay@@UEAAXPEAXHHHPEBDI@Z 00000000375028b0 f i CryLiveCreate.obj
 0001:000018b0       ?OnFileUploadProgress@CManager@LiveCreate@@MEAAXPEBD0HHW4EResultCode@IObserver@FileSyncManager@2@0@Z 00000000375028b0 f i LiveCreate.obj
 0001:000018b0       ?OnBeginSendToPeers@CommonController@LiveCreate@@UEAAXXZ 00000000375028b0 f i LiveCreateCtrl_Common.obj
 0001:000018b0       ?AllocUsage@CDummyMemReplay@@UEAAXW4Class@EMemReplayAllocClass@@_K1@Z 00000000375028b0 f i CryLiveCreate.obj
 0001:000018b0       ?RemoveAllocReference@CDummyMemReplay@@UEAAXPEAX@Z 00000000375028b0 f i CryLiveCreate.obj
 0001:000018b0       ?OnPeerDisconnected@CameraController@LiveCreate@@UEAAXPEAUSPeerLink@2@@Z 00000000375028b0 f i LiveCreateCtrl_Camera.obj
 0001:000018b0       ?EnablePeer@CNullManager@LiveCreate@@UEAAXPEAUSPeerLink@2@_N@Z 00000000375028b0 f i LiveCreate.obj
 0001:000018b0       ?MapPage@CDummyMemReplay@@UEAAXPEAX_K@Z 00000000375028b0 f i CryLiveCreate.obj
 0001:000018b0       ?ExitScope@CDummyMemReplay@@UEAAXXZ 00000000375028b0 f i CryLiveCreate.obj
 0001:000018b0       ?SwapContainers@CDummyMemReplay@@UEAAXPEBX0@Z 00000000375028b0 f i CryLiveCreate.obj
 0001:000018b0       ?OnUpdate@CommonController@LiveCreate@@UEAAXXZ 00000000375028b0 f i LiveCreateCtrl_Common.obj
 0001:000018b0       ?AddAllocReference@CDummyMemReplay@@UEAAXPEAX0@Z 00000000375028b0 f i CryLiveCreate.obj
 0001:000018b0       ?Terminate@?$CrySimpleThread@VNetPeerCommThread@LiveCreate@@@@MEAAXXZ 00000000375028b0 f i LiveCreateNetwork.obj
 0001:000018b0       ?DumpStats@CDummyMemReplay@@UEAAXXZ 00000000375028b0 f i CryLiveCreate.obj
 0001:000018b0       ?RemoveContext@CDummyMemReplay@@UEAAXXZ 00000000375028b0 f i CryLiveCreate.obj
 0001:000018b0       ?BindToContainer@CDummyMemReplay@@UEAAXPEBX0@Z 00000000375028b0 f i CryLiveCreate.obj
 0001:000018b0       ?OnFileUploadProgress@IObserver@FileSyncManager@LiveCreate@@UEAAXPEBD0HHW4EResultCode@123@0@Z 00000000375028b0 f i LiveCreate.obj
 0001:000018b0       ?OnBeginSendToPeers@ScreenshotController@LiveCreate@@UEAAXXZ 00000000375028b0 f i LiveCreateCtrl_Screenshot.obj
 0001:000018b0       ?SetEnabled@CNullManager@LiveCreate@@UEAAX_N@Z 00000000375028b0 f i LiveCreate.obj
 0001:000018b0       ?Terminate@?$CrySimpleThread@VFileSyncManager@LiveCreate@@@@MEAAXXZ 00000000375028b0 f i LiveCreateFileSync.obj
 0001:000018b0       ?AddLabel@CDummyMemReplay@@UEAAXPEBD@Z 00000000375028b0 f i CryLiveCreate.obj
 0001:000018b0       ?ExitScope_Alloc@CDummyMemReplay@@UEAAX_K00@Z 00000000375028b0 f i CryLiveCreate.obj
 0001:000018b0       ?MarkPool@CDummyMemReplay@@UEAAXH_KPEAX0PEBD@Z 00000000375028b0 f i CryLiveCreate.obj
 0001:000018b0       ??1PS3TmHelper@@QEAA@XZ    00000000375028b0 f i PS3TmHelperLib:PS3TmHelper.obj
 0001:000018b0       ?DumpSymbols@CDummyMemReplay@@UEAAXXZ 00000000375028b0 f i CryLiveCreate.obj
 0001:000018b0       ?RegisterFixedAddressRange@CDummyMemReplay@@UEAAXPEAX_KPEBD@Z 00000000375028b0 f i CryLiveCreate.obj
 0001:000018b0       ?OnFileUploadStart@CManager@LiveCreate@@MEAAXPEBD@Z 00000000375028b0 f i LiveCreate.obj
 0001:000018b0       ?OnBeginSendToPeers@ExecuteConsoleStringController@LiveCreate@@UEAAXXZ 00000000375028b0 f i LiveCreateCtrl_ExecuteConsoleString.obj
 0001:000018b0       ?Sync@CNullManager@LiveCreate@@UEAAXPEAUIController@2@@Z 00000000375028b0 f i LiveCreate.obj
 0001:000018b0       ?SetFileSyncEnabled@CNullManager@LiveCreate@@UEAAX_N@Z 00000000375028b0 f i LiveCreate.obj
 0001:000018b0       ?AddContext@CDummyMemReplay@@UEAAXHIPEBD@Z 00000000375028b0 f i CryLiveCreate.obj
 0001:000018b0       ?ExitScope_Realloc@CDummyMemReplay@@UEAAX_K000@Z 00000000375028b0 f i CryLiveCreate.obj
 0001:000018b0       ?AddScreenshot@CDummyMemReplay@@UEAAXXZ 00000000375028b0 f i CryLiveCreate.obj
 0001:000018b0       ?BucketEnableCleanups@CDummyMemReplay@@UEAAXPEAX_N@Z 00000000375028b0 f i CryLiveCreate.obj
 0001:000018b0       ?OnPeerDisconnected@CommonController@LiveCreate@@UEAAXPEAUSPeerLink@2@@Z 00000000375028b0 f i LiveCreateCtrl_Common.obj
 0001:000018b0       ?Update@CNullManager@LiveCreate@@UEAAXXZ 00000000375028b0 f i LiveCreate.obj
 0001:000018b0       ?Sync@CNullManager@LiveCreate@@UEAAXPEBD@Z 00000000375028b0 f i LiveCreate.obj
 0001:000018c0       ?CryPureCallHandler@@YAXXZ 00000000375028c0 f   CryLiveCreate.obj
 0001:000018d0       ?CryInvalidParameterHandler@@YAXPEB_W00I_K@Z 00000000375028d0 f   CryLiveCreate.obj
 0001:000018e0       ModuleInitISystem          00000000375028e0 f   CryLiveCreate.obj
 0001:000019b0       CryModuleGetMemoryInfo     00000000375029b0 f   CryLiveCreate.obj
 0001:000019f0       ?CryDeleteCriticalSectionInplace@@YAXPEAX@Z 00000000375029f0 f   CryLiveCreate.obj
 0001:00001a20       ?CryGetIMemReplay@@YAPEAUIMemReplay@@XZ 0000000037502a20 f i CryLiveCreate.obj
 0001:00001ad0       CryModuleMalloc            0000000037502ad0 f   CryLiveCreate.obj
 0001:00001b70       CryModuleFree              0000000037502b70 f   CryLiveCreate.obj
 0001:00001be0       ??2@YAPEAX_K@Z             0000000037502be0 f   CryLiveCreate.obj
 0001:00001c50       ??_U@YAPEAX_K@Z            0000000037502c50 f   CryLiveCreate.obj
 0001:00001cc0       ??3@YAXPEAX@Z              0000000037502cc0 f   CryLiveCreate.obj
 0001:00001d60       ??_V@YAXPEAX@Z             0000000037502d60 f   CryLiveCreate.obj
 0001:00001e00       ??_EICryFactory@@MEAAPEAXI@Z 0000000037502e00 f i CryLiveCreate.obj
 0001:00001e00       ??_GICryFactory@@MEAAPEAXI@Z 0000000037502e00 f i CryLiveCreate.obj
 0001:00001e30       ??_GCSystemEventListner_LiveCreate@@UEAAPEAXI@Z 0000000037502e30 f i CryLiveCreate.obj
 0001:00001e30       ??_ECSystemEventListner_LiveCreate@@UEAAPEAXI@Z 0000000037502e30 f i CryLiveCreate.obj
 0001:00001e30       ??_EISystemEventListener@@UEAAPEAXI@Z 0000000037502e30 f i CryLiveCreate.obj
 0001:00001e30       ??_GISystemEventListener@@UEAAPEAXI@Z 0000000037502e30 f i CryLiveCreate.obj
 0001:00001e60       CreateLiveCreate           0000000037502e60 f   CryLiveCreate.obj
 0001:00001ef0       ?GetFactory@CEngineModule_CryLiveCreate@@UEBAPEAUICryFactory@@XZ 0000000037502ef0 f i CryLiveCreate.obj
 0001:00001f00       ?GetName@CEngineModule_CryLiveCreate@@MEAAPEBDXZ 0000000037502f00 f i CryLiveCreate.obj
 0001:00001f10       ?GetCategory@CEngineModule_CryLiveCreate@@MEAAPEBDXZ 0000000037502f10 f i CryLiveCreate.obj
 0001:00001f20       ?Initialize@CEngineModule_CryLiveCreate@@MEAA_NAEAUSSystemGlobalEnvironment@@AEBUSSystemInitParams@@@Z 0000000037502f20 f i CryLiveCreate.obj
 0001:00001fe0       ??_ECEngineModule_CryLiveCreate@@MEAAPEAXI@Z 0000000037502fe0 f i CryLiveCreate.obj
 0001:00001fe0       ??_EICryUnknown@@MEAAPEAXI@Z 0000000037502fe0 f i CryLiveCreate.obj
 0001:00001fe0       ??_GCEngineModule_CryLiveCreate@@MEAAPEAXI@Z 0000000037502fe0 f i CryLiveCreate.obj
 0001:00001fe0       ??_GICryUnknown@@MEAAPEAXI@Z 0000000037502fe0 f i CryLiveCreate.obj
 0001:00002010       ?_AllocData@?$CryStringT@D@@IEAAX_K@Z 0000000037503010 f i CryLiveCreate.obj
 0001:00002080       ?_Free@?$CryStringT@D@@IEAAXXZ 0000000037503080 f i CryLiveCreate.obj
 0001:000020d0       ?_Assign@?$CryStringT@D@@IEAAXPEBD_K@Z 00000000375030d0 f i CryLiveCreate.obj
 0001:000021b0       ?_MakeUnique@?$CryStringT@D@@IEAAXXZ 00000000375031b0 f i CryLiveCreate.obj
 0001:00002270       ?_Concatenate@?$CryStringT@D@@IEAAXPEBD_K01@Z 0000000037503270 f i CryLiveCreate.obj
 0001:00002320       ??_ECDummyMemReplay@@UEAAPEAXI@Z 0000000037503320 f i CryLiveCreate.obj
 0001:00002320       ??_GIMemReplay@@UEAAPEAXI@Z 0000000037503320 f i CryLiveCreate.obj
 0001:00002320       ??_EIMemReplay@@UEAAPEAXI@Z 0000000037503320 f i CryLiveCreate.obj
 0001:00002320       ??_GCDummyMemReplay@@UEAAPEAXI@Z 0000000037503320 f i CryLiveCreate.obj
 0001:00002350       ??_GCrySimpleThreadSelf@@UEAAPEAXI@Z 0000000037503350 f i CryLiveCreate.obj
 0001:00002350       ??_ECrySimpleThreadSelf@@UEAAPEAXI@Z 0000000037503350 f i CryLiveCreate.obj
 0001:000023a0       ??0CFactory@CEngineModule_CryLiveCreate@@AEAA@XZ 00000000375033a0 f i CryLiveCreate.obj
 0001:00002440       ?GetClassNameA@CFactory@CEngineModule_CryLiveCreate@@UEBAPEBDXZ 0000000037503440 f i CryLiveCreate.obj
 0001:00002450       ?GetClassID@CFactory@CEngineModule_CryLiveCreate@@UEBAAEBUCryGUID@@XZ 0000000037503450 f i CryLiveCreate.obj
 0001:00002460       ?ClassSupports@CFactory@CEngineModule_CryLiveCreate@@UEBAXAEAPEBUCryGUID@@AEA_K@Z 0000000037503460 f i CryLiveCreate.obj
 0001:00002470       ?sp_enable_shared_from_this@detail@boost@@YAXZZ 0000000037503470 f i CryLiveCreate.obj
 0001:00002490       ?ClassSupports@CFactory@CEngineModule_CryLiveCreate@@UEBA_NAEBUCryGUID@@@Z 0000000037503490 f i CryLiveCreate.obj
 0001:000024d0       ?dispose@?$sp_counted_impl_p@VCEngineModule_CryLiveCreate@@@detail@boost@@UEAAXXZ 00000000375034d0 f i CryLiveCreate.obj
 0001:000024f0       ??_GCFactory@CEngineModule_CryLiveCreate@@UEAAPEAXI@Z 00000000375034f0 f i CryLiveCreate.obj
 0001:000024f0       ??_ECFactory@CEngineModule_CryLiveCreate@@UEAAPEAXI@Z 00000000375034f0 f i CryLiveCreate.obj
 0001:00002530       ??_G?$sp_counted_impl_p@VCEngineModule_CryLiveCreate@@@detail@boost@@UEAAPEAXI@Z 0000000037503530 f i CryLiveCreate.obj
 0001:00002530       ??_E?$sp_counted_impl_p@VCEngineModule_CryLiveCreate@@@detail@boost@@UEAAPEAXI@Z 0000000037503530 f i CryLiveCreate.obj
 0001:00002530       ??_Esp_counted_base@detail@boost@@UEAAPEAXI@Z 0000000037503530 f i CryLiveCreate.obj
 0001:00002530       ??_Gsp_counted_base@detail@boost@@UEAAPEAXI@Z 0000000037503530 f i CryLiveCreate.obj
 0001:00002560       ??$?0VCEngineModule_CryLiveCreate@@@shared_count@detail@boost@@QEAA@PEAVCEngineModule_CryLiveCreate@@@Z 0000000037503560 f i CryLiveCreate.obj
 0001:00002670       ??_Gbad_alloc@std@@UEAAPEAXI@Z 0000000037503670 f i CryLiveCreate.obj
 0001:00002670       ??_Ebad_alloc@std@@UEAAPEAXI@Z 0000000037503670 f i CryLiveCreate.obj
 0001:000026b0       ?QueryInterface@CEngineModule_CryLiveCreate@@MEBAPEAXAEBUCryGUID@@@Z 00000000375036b0 f i CryLiveCreate.obj
 0001:00002700       ??0?$CryStringT@D@@QEAA@PEBD@Z 0000000037503700 f i CryLiveCreate.obj
 0001:00002780       ??4?$CryStringT@D@@QEAAAEAV0@AEBV0@@Z 0000000037503780 f i CryLiveCreate.obj
 0001:00002830       ??0?$CryStringT@D@@QEAA@PEBD_K@Z 0000000037503830 f i CryLiveCreate.obj
 0001:000028c0       ?append@?$CryStringT@D@@QEAAAEAV1@_KD@Z 00000000375038c0 f i CryLiveCreate.obj
 0001:000029b0       ?_ConcatenateInPlace@?$CryStringT@D@@IEAAXPEBD_K@Z 00000000375039b0 f i CryLiveCreate.obj
 0001:00002a70       ?CreateClassInstance@CFactory@CEngineModule_CryLiveCreate@@UEBA?AV?$shared_ptr@UICryUnknown@@@boost@@XZ 0000000037503a70 f i CryLiveCreate.obj
 0001:00002b40       ?resize@?$CryStringT@D@@QEAAX_KD@Z 0000000037503b40 f i CryLiveCreate.obj
 0001:00002bb0       __delayLoadHelper2         0000000037503bb0 f   delayhlp.obj
 0001:00002f40       __HrLoadAllImportsForDll   0000000037503f40 f   delayhlp.obj
 0001:00003050       ??_GIObserver@FileSyncManager@LiveCreate@@UEAAPEAXI@Z 0000000037504050 f i LiveCreate.obj
 0001:00003050       ??_EIObserver@FileSyncManager@LiveCreate@@UEAAPEAXI@Z 0000000037504050 f i LiveCreate.obj
 0001:00003080       ?Initialize@CManager@LiveCreate@@UEAA_NII@Z 0000000037504080 f   LiveCreate.obj
 0001:00003130       ?Shutdown@CManager@LiveCreate@@UEAA_NXZ 0000000037504130 f   LiveCreate.obj
 0001:000031b0       ?IsEnabled@CManager@LiveCreate@@UEAA_NXZ 00000000375041b0 f   LiveCreate.obj
 0001:000031c0       ?SetEnabled@CManager@LiveCreate@@UEAAX_N@Z 00000000375041c0 f   LiveCreate.obj
 0001:000031d0       ?IsFileSyncEnabled@CManager@LiveCreate@@UEAA_NXZ 00000000375041d0 f   LiveCreate.obj
 0001:000031e0       ?SetFileSyncEnabled@CManager@LiveCreate@@UEAAX_N@Z 00000000375041e0 f   LiveCreate.obj
 0001:000031f0       ?IsLogEnabled@CManager@LiveCreate@@UEAA_NXZ 00000000375041f0 f   LiveCreate.obj
 0001:00003230       ?SetLogEnabled@CManager@LiveCreate@@UEAAX_N@Z 0000000037504230 f   LiveCreate.obj
 0001:00003280       ?SyncModifiedFile@CManager@LiveCreate@@UEAAXPEBD0H0@Z 0000000037504280 f   LiveCreate.obj
 0001:000032b0       ?ClearFileSyncQueue@CManager@LiveCreate@@UEAAXXZ 00000000375042b0 f   LiveCreate.obj
 0001:000032c0       ?IsFileSyncGroupDone@CManager@LiveCreate@@UEAA_NH@Z 00000000375042c0 f   LiveCreate.obj
 0001:000032d0       ?IsFileAllowedToSync@CManager@LiveCreate@@UEAA_NPEBD@Z 00000000375042d0 f   LiveCreate.obj
 0001:000032f0       ?CommitData@CManager@LiveCreate@@UEAA_NPEBD0PEAXH@Z 00000000375042f0 f   LiveCreate.obj
 0001:00003360       ?SendControllerData@CManager@LiveCreate@@IEAA_NPEAUIController@2@PEAUSPeerLink@2@IPEBEI@Z 0000000037504360 f   LiveCreate.obj
 0001:000034b0       ?Sync@CManager@LiveCreate@@UEAAXPEBD@Z 00000000375044b0 f   LiveCreate.obj
 0001:000034e0       ?IsConnectedTo@CManager@LiveCreate@@UEAA_NPEBD@Z 00000000375044e0 f   LiveCreate.obj
 0001:000034f0       ?EnablePeer@CManager@LiveCreate@@UEAAXPEAUSPeerLink@2@_N@Z 00000000375044f0 f   LiveCreate.obj
 0001:00003510       ?DisconnectPeer@CManager@LiveCreate@@UEAA_NPEAUSPeerLink@2@@Z 0000000037504510 f   LiveCreate.obj
 0001:00003540       ?DisconnectAllPeers@CManager@LiveCreate@@UEAA_NXZ 0000000037504540 f   LiveCreate.obj
 0001:00003560       ?IsAnyPeerConnected@CManager@LiveCreate@@UEAA_NXZ 0000000037504560 f   LiveCreate.obj
 0001:00003570       ?OnFileUploadEnd@CManager@LiveCreate@@MEAAXPEBD_N@Z 0000000037504570 f   LiveCreate.obj
 0001:000035d0       ?_Rotate_left@?$_Rb_global@_N@priv@stlpmtx_std@@SAXPEAU_Rb_tree_node_base@23@AEAPEAU423@@Z 00000000375045d0 f i LiveCreate.obj
 0001:00003630       ?_Rotate_right@?$_Rb_global@_N@priv@stlpmtx_std@@SAXPEAU_Rb_tree_node_base@23@AEAPEAU423@@Z 0000000037504630 f i LiveCreate.obj
 0001:00003690       ?_Rebalance@?$_Rb_global@_N@priv@stlpmtx_std@@SAXPEAU_Rb_tree_node_base@23@AEAPEAU423@@Z 0000000037504690 f i LiveCreate.obj
 0001:00003880       ?CryLog@@YAXPEBDZZ         0000000037504880 f i LiveCreate.obj
 0001:000038e0       ??_ECNullManager@LiveCreate@@UEAAPEAXI@Z 00000000375048e0 f i LiveCreate.obj
 0001:000038e0       ??_GCNullManager@LiveCreate@@UEAAPEAXI@Z 00000000375048e0 f i LiveCreate.obj
 0001:000038e0       ??_EIManager@LiveCreate@@UEAAPEAXI@Z 00000000375048e0 f i LiveCreate.obj
 0001:000038e0       ??_GIManager@LiveCreate@@UEAAPEAXI@Z 00000000375048e0 f i LiveCreate.obj
 0001:00003910       ?LogMessage@CNullManager@LiveCreate@@UEAAXW4ELogMessageType@2@PEBDZZ 0000000037504910 f i LiveCreate.obj
 0001:00003920       ?IsNullImplementation@CNullManager@LiveCreate@@UEAA_NXZ 0000000037504920 f i LiveCreate.obj
 0001:00003920       ?IsFileSyncQueueEmpty@CNullManager@LiveCreate@@UEAA_NXZ 0000000037504920 f i LiveCreate.obj
 0001:00003920       ?IsFileSyncGroupDone@CNullManager@LiveCreate@@UEAA_NH@Z 0000000037504920 f i LiveCreate.obj
 0001:00003920       ?OnSend@CommonController@LiveCreate@@UEAA_NPEAUSPeerLink@2@AEAUSDataSync@IController@2@@Z 0000000037504920 f i LiveCreateCtrl_Common.obj
 0001:00003920       ?OnBeforeVarChange@CVarController@LiveCreate@@UEAA_NPEAUICVar@@PEBD@Z 0000000037504920 f i LiveCreateCtrl_CVar.obj
 0001:00003930       ?GetLinkTo@CNullManager@LiveCreate@@UEAAPEAUSPeerLink@2@PEBD@Z 0000000037504930 f i LiveCreate.obj
 0001:00003930       ?ConnectToPeer@CNullManager@LiveCreate@@UEAAPEAUSPeerLink@2@AEBUSPeerInfo@2@@Z 0000000037504930 f i LiveCreate.obj
 0001:00003930       ?GetPeerCount@CNullManager@LiveCreate@@UEAAIXZ 0000000037504930 f i LiveCreate.obj
 0001:00003930       ?GetControllerByName@CNullManager@LiveCreate@@UEAAPEAUIController@2@PEBD@Z 0000000037504930 f i LiveCreate.obj
 0001:00003930       ?QueryComposite@CEngineModule_CryLiveCreate@@MEBAPEAXPEBD@Z 0000000037504930 f i CryLiveCreate.obj
 0001:00003930       ?GetPlatformHandlerFactoryAt@CNullManager@LiveCreate@@UEAAPEAUIPlatformHandlerFactory@2@I@Z 0000000037504930 f i LiveCreate.obj
 0001:00003930       ?GetFileModificationTime@PlatformHandlerBase@LiveCreate@@UEAA_KPEBD@Z 0000000037504930 f i PlatformHandlerBase.obj
 0001:00003930       ?GetFileModificationTime@PlatformHandler_PS3@LiveCreate@@UEAA_KPEBD@Z 0000000037504930 f i PlatformHandler_PS3.obj
 0001:00003930       ?GetNextController@CNullManager@LiveCreate@@UEAAPEAUIController@2@PEAU32@@Z 0000000037504930 f i LiveCreate.obj
 0001:00003930       ?GatherPlatforms@IPlatformHandlerFactory@LiveCreate@@UEAAIPEAUSPeerInfo@2@I@Z 0000000037504930 f i LiveCreate.obj
 0001:00003930       ?GetPeerAt@CNullManager@LiveCreate@@UEAAPEAUSPeerLink@2@I@Z 0000000037504930 f i LiveCreate.obj
 0001:00003930       ?BeginScanFolder@PlatformHandlerBase@LiveCreate@@UEAAPEAXPEBD@Z 0000000037504930 f i PlatformHandlerBase.obj
 0001:00003930       ?GetPlatformHandlerFactoryCount@CNullManager@LiveCreate@@UEAAIXZ 0000000037504930 f i LiveCreate.obj
 0001:00003930       ?AddPeer@CNullManager@LiveCreate@@UEAAPEAUSPeerLink@2@AEBUSPeerInfo@2@@Z 0000000037504930 f i LiveCreate.obj
 0001:00003930       ?GatherPlatforms@CNullManager@LiveCreate@@UEAAHPEAUSPeerInfo@2@H@Z 0000000037504930 f i LiveCreate.obj
 0001:00003930       ?GetFirstController@CNullManager@LiveCreate@@UEAAPEAUIController@2@XZ 0000000037504930 f i LiveCreate.obj
 0001:00003930       ?GetControllerCount@CNullManager@LiveCreate@@UEAAIXZ 0000000037504930 f i LiveCreate.obj
 0001:00003930       ?get_deleter@?$sp_counted_impl_p@VCEngineModule_CryLiveCreate@@@detail@boost@@UEAAPEAXAEBVsp_typeinfo@23@@Z 0000000037504930 f i CryLiveCreate.obj
 0001:00003940       ?Shutdown@CNullManager@LiveCreate@@UEAA_NXZ 0000000037504940 f i LiveCreate.obj
 0001:00003940       ?FindMachineAddressByName@CNullManager@LiveCreate@@UEAA_NPEBDPEADI@Z 0000000037504940 f i LiveCreate.obj
 0001:00003940       ?FindMachineAddressByName@PlatformHandlerFactory_EditorPC@LiveCreate@@UEAA_NPEBDPEADI@Z 0000000037504940 f i PlatformHandler_EditorPC.obj
 0001:00003940       ?Launch@PlatformHandlerBase@LiveCreate@@UEAA_NPEBD00@Z 0000000037504940 f i PlatformHandlerBase.obj
 0001:00003940       ?CopyFileTo@PlatformHandlerBase@LiveCreate@@UEAA_NPEBD0@Z 0000000037504940 f i PlatformHandlerBase.obj
 0001:00003940       ?SearchForGameBuilds@PlatformHandlerBase@LiveCreate@@UEAA_NXZ 0000000037504940 f i PlatformHandlerBase.obj
 0001:00003940       ?RegisterPlatformHandlerFactory@CNullManager@LiveCreate@@UEAA_NPEAUIPlatformHandlerFactory@2@@Z 0000000037504940 f i LiveCreate.obj
 0001:00003940       ?IsFileAllowedToSync@CNullManager@LiveCreate@@UEAA_NPEBD@Z 0000000037504940 f i LiveCreate.obj
 0001:00003940       ?FindMachineAddressByName@PlatformHandlerFactory_GamePC@LiveCreate@@UEAA_NPEBDPEADI@Z 0000000037504940 f i PlatformHandler_GamePC.obj
 0001:00003940       ?IsLinkedTo@CNullManager@LiveCreate@@UEAA_NPEBD@Z 0000000037504940 f i LiveCreate.obj
 0001:00003940       ?EraseFile@PlatformHandlerBase@LiveCreate@@UEAA_NPEBD@Z 0000000037504940 f i PlatformHandlerBase.obj
 0001:00003940       ?CopyFileFrom@PlatformHandler_GamePC@LiveCreate@@UEAA_NPEBD0@Z 0000000037504940 f i PlatformHandler_GamePC.obj
 0001:00003940       ?IsNullImplementation@CManager@LiveCreate@@UEAA_NXZ 0000000037504940 f i LiveCreate.obj
 0001:00003940       ?Initialize@CNullManager@LiveCreate@@UEAA_NII@Z 0000000037504940 f i LiveCreate.obj
 0001:00003940       ?IsOn@PlatformHandlerBase@LiveCreate@@UEAA_NXZ 0000000037504940 f i PlatformHandlerBase.obj
 0001:00003940       ?CommitData@CNullManager@LiveCreate@@UEAA_NPEBD0PEAXH@Z 0000000037504940 f i LiveCreate.obj
 0001:00003940       ?RegisterListener@CNullManager@LiveCreate@@UEAA_NPEAUIManagerListener@2@@Z 0000000037504940 f i LiveCreate.obj
 0001:00003940       ?CopyFileTo@PlatformHandler_GamePC@LiveCreate@@UEAA_NPEBD0@Z 0000000037504940 f i PlatformHandler_GamePC.obj
 0001:00003940       ?UnregisterController@CNullManager@LiveCreate@@UEAA_NPEAUIController@2@@Z 0000000037504940 f i LiveCreate.obj
 0001:00003940       ?CopyFileFrom@PlatformHandlerBase@LiveCreate@@UEAA_NPEBD0@Z 0000000037504940 f i PlatformHandlerBase.obj
 0001:00003940       ?UnregisterPlatformHandlerFactory@CNullManager@LiveCreate@@UEAA_NPEAUIPlatformHandlerFactory@2@@Z 0000000037504940 f i LiveCreate.obj
 0001:00003940       ?DisconnectPeer@CNullManager@LiveCreate@@UEAA_NPEAUSPeerLink@2@@Z 0000000037504940 f i LiveCreate.obj
 0001:00003940       ?GetPeerInfo@CNullManager@LiveCreate@@UEAA_NPEAUSPeerLink@2@AEAUSPeerInfo@2@@Z 0000000037504940 f i LiveCreate.obj
 0001:00003940       ?NextScanFolderEntry@PlatformHandlerBase@LiveCreate@@UEAA_NPEAXPEAUSScanFolderEntry@2@@Z 0000000037504940 f i PlatformHandlerBase.obj
 0001:00003940       ?EnterScope@CDummyMemReplay@@UEAA_NW4Class@EMemReplayAllocClass@@GH@Z 0000000037504940 f i CryLiveCreate.obj
 0001:00003940       ?IsOn@PlatformHandler_GamePC@LiveCreate@@UEAA_NXZ 0000000037504940 f i PlatformHandler_GamePC.obj
 0001:00003940       ?DisconnectAllPeers@CNullManager@LiveCreate@@UEAA_NXZ 0000000037504940 f i LiveCreate.obj
 0001:00003940       ?IsConnectedTo@CNullManager@LiveCreate@@UEAA_NPEBD@Z 0000000037504940 f i LiveCreate.obj
 0001:00003940       ?IsEnabled@CNullManager@LiveCreate@@UEAA_NXZ 0000000037504940 f i LiveCreate.obj
 0001:00003940       ?IsLogEnabled@CNullManager@LiveCreate@@UEAA_NXZ 0000000037504940 f i LiveCreate.obj
 0001:00003940       ?Reset@PlatformHandlerBase@LiveCreate@@UEAA_NW4EResetMode@SProfile@2@@Z 0000000037504940 f i PlatformHandlerBase.obj
 0001:00003940       ?CopyFileTo@PlatformHandler_EditorPC@LiveCreate@@UEAA_NPEBD0@Z 0000000037504940 f i PlatformHandler_EditorPC.obj
 0001:00003940       ?Reset@PlatformHandler_EditorPC@LiveCreate@@UEAA_NW4EResetMode@SProfile@2@@Z 0000000037504940 f i PlatformHandler_EditorPC.obj
 0001:00003940       ?IsAnyPeerConnected@CNullManager@LiveCreate@@UEAA_NXZ 0000000037504940 f i LiveCreate.obj
 0001:00003940       ?RegisterController@CNullManager@LiveCreate@@UEAA_NPEAUIController@2@@Z 0000000037504940 f i LiveCreate.obj
 0001:00003940       ?IsFileSyncEnabled@CNullManager@LiveCreate@@UEAA_NXZ 0000000037504940 f i LiveCreate.obj
 0001:00003940       ?EraseFolder@PlatformHandlerBase@LiveCreate@@UEAA_NPEBD@Z 0000000037504940 f i PlatformHandlerBase.obj
 0001:00003940       ?Launch@PlatformHandler_GamePC@LiveCreate@@UEAA_NPEBD00@Z 0000000037504940 f i PlatformHandler_GamePC.obj
 0001:00003940       ?UnregisterListener@CNullManager@LiveCreate@@UEAA_NPEAUIManagerListener@2@@Z 0000000037504940 f i LiveCreate.obj
 0001:00003940       ?Reset@PlatformHandler_GamePC@LiveCreate@@UEAA_NW4EResetMode@SProfile@2@@Z 0000000037504940 f i PlatformHandler_GamePC.obj
 0001:00003940       ?Launch@PlatformHandler_EditorPC@LiveCreate@@UEAA_NPEBD00@Z 0000000037504940 f i PlatformHandler_EditorPC.obj
 0001:00003940       ?IsOn@PlatformHandler_EditorPC@LiveCreate@@UEAA_NXZ 0000000037504940 f i PlatformHandler_EditorPC.obj
 0001:00003940       ?CopyFileFrom@PlatformHandler_EditorPC@LiveCreate@@UEAA_NPEBD0@Z 0000000037504940 f i PlatformHandler_EditorPC.obj
 0001:00003950       ?GetCustomPlatformName@CNullManager@LiveCreate@@UEAAPEBDXZ 0000000037504950 f i LiveCreate.obj
 0001:00003950       ?GetDescription@CommonController@LiveCreate@@UEAAPEBDXZ 0000000037504950 f i LiveCreateCtrl_Common.obj
 0001:00003950       ?GetUniqueName@CommonController@LiveCreate@@UEAAPEBDXZ 0000000037504950 f i LiveCreateCtrl_Common.obj
 0001:00003950       ?GetDisplayName@CommonController@LiveCreate@@UEAAPEBDXZ 0000000037504950 f i LiveCreateCtrl_Common.obj
 0001:00003960       ?GetCustomPlatformName@CManager@LiveCreate@@UEAAPEBDXZ 0000000037504960 f   LiveCreate.obj
 0001:00003970       ??$find@PEAPEAUSPeerLink@LiveCreate@@PEAU12@@stlpmtx_std@@YAPEAPEAUSPeerLink@LiveCreate@@PEAPEAU12@0AEBQEAU12@@Z 0000000037504970 f i LiveCreate.obj
 0001:00003970       ??$find@PEAPEAUIPlatformHandlerFactory@LiveCreate@@PEAU12@@stlpmtx_std@@YAPEAPEAUIPlatformHandlerFactory@LiveCreate@@PEAPEAU12@0AEBQEAU12@@Z 0000000037504970 f i LiveCreate.obj
 0001:00003970       ??$find@PEAPEAUNetPeerConnection@LiveCreate@@PEAX@stlpmtx_std@@YAPEAPEAUNetPeerConnection@LiveCreate@@PEAPEAU12@0AEBQEAX@Z 0000000037504970 f i LiveCreateNetwork.obj
 0001:00003970       ??$find@PEAPEAUSX360WalkDir@PlatformHandler_X360@LiveCreate@@PEAX@stlpmtx_std@@YAPEAPEAUSX360WalkDir@PlatformHandler_X360@LiveCreate@@PEAPEAU123@0AEBQEAX@Z 0000000037504970 f i PlatformHandler_X360.obj
 0001:00003a00       ?_Rebalance_for_erase@?$_Rb_global@_N@priv@stlpmtx_std@@SAPEAU_Rb_tree_node_base@23@PEAU423@AEAPEAU423@11@Z 0000000037504a00 f i LiveCreate.obj
 0001:00003d50       ??_GPlatformHandlerFactory_EditorPC@LiveCreate@@UEAAPEAXI@Z 0000000037504d50 f i LiveCreate.obj
 0001:00003d50       ??_GPlatformHandlerFactory_GamePC@LiveCreate@@UEAAPEAXI@Z 0000000037504d50 f i LiveCreate.obj
 0001:00003d50       ??_EPlatformHandlerFactory_GamePC@LiveCreate@@UEAAPEAXI@Z 0000000037504d50 f i LiveCreate.obj
 0001:00003d50       ??_EPlatformHandlerFactory_X360@LiveCreate@@UEAAPEAXI@Z 0000000037504d50 f i PlatformHandler_X360.obj
 0001:00003d50       ??_GPlatformHandlerFactory_X360@LiveCreate@@UEAAPEAXI@Z 0000000037504d50 f i PlatformHandler_X360.obj
 0001:00003d50       ??_GIPlatformHandlerFactory@LiveCreate@@UEAAPEAXI@Z 0000000037504d50 f i LiveCreate.obj
 0001:00003d50       ??_EIPlatformHandlerFactory@LiveCreate@@UEAAPEAXI@Z 0000000037504d50 f i LiveCreate.obj
 0001:00003d50       ??_EPlatformHandlerFactory_EditorPC@LiveCreate@@UEAAPEAXI@Z 0000000037504d50 f i LiveCreate.obj
 0001:00003d80       ?IsFileSyncQueueEmpty@CManager@LiveCreate@@UEAA_NXZ 0000000037504d80 f   LiveCreate.obj
 0001:00003de0       ?GetPlatformHandlerFactoryCount@CManager@LiveCreate@@UEAAIXZ 0000000037504de0 f   LiveCreate.obj
 0001:00003e00       ?GetControllerCount@CManager@LiveCreate@@UEAAIXZ 0000000037504e00 f   LiveCreate.obj
 0001:00003e10       ?GetPeerCount@CManager@LiveCreate@@UEAAIXZ 0000000037504e10 f   LiveCreate.obj
 0001:00003e30       ?_M_erase@?$_Rb_tree@PEAXU?$_BinaryPredWrapper@PEAXPEAUIManagerListener@LiveCreate@@U?$less@PEAUIManagerListener@LiveCreate@@@stlpmtx_std@@@priv@stlpmtx_std@@PEAXU?$_Identity@PEAX@23@U?$_SetTraitsT@PEAX@23@V?$allocator@PEAX@3@@priv@stlpmtx_std@@AEAAXPEAU_Rb_tree_node_base@23@@Z 0000000037504e30 f i LiveCreate.obj
 0001:00003e30       ?_M_erase@?$_Rb_tree@PEAXU?$_BinaryPredWrapper@PEAXPEAUIPlatformHandler@LiveCreate@@U?$less@PEAUIPlatformHandler@LiveCreate@@@stlpmtx_std@@@priv@stlpmtx_std@@PEAXU?$_Identity@PEAX@23@U?$_SetTraitsT@PEAX@23@V?$allocator@PEAX@3@@priv@stlpmtx_std@@AEAAXPEAU_Rb_tree_node_base@23@@Z 0000000037504e30 f i LiveCreateCtrl_Screenshot.obj
 0001:00003e90       ?LogMessage@CManager@LiveCreate@@UEAAXW4ELogMessageType@2@PEBDZZ 0000000037504e90 f   LiveCreate.obj
 0001:00004010       ?GetPlatformHandlerFactoryAt@CManager@LiveCreate@@UEAAPEAUIPlatformHandlerFactory@2@I@Z 0000000037505010 f   LiveCreate.obj
 0001:00004020       ?GetFirstController@CManager@LiveCreate@@UEAAPEAUIController@2@XZ 0000000037505020 f   LiveCreate.obj
 0001:00004040       ?GetNextController@CManager@LiveCreate@@UEAAPEAUIController@2@PEAU32@@Z 0000000037505040 f   LiveCreate.obj
 0001:00004110       ?Sync@CManager@LiveCreate@@UEAAXPEAUIController@2@@Z 0000000037505110 f   LiveCreate.obj
 0001:000042d0       ?GatherPlatforms@CManager@LiveCreate@@UEAAHPEAUSPeerInfo@2@H@Z 00000000375052d0 f   LiveCreate.obj
 0001:00004380       ?FindMachineAddressByName@CManager@LiveCreate@@UEAA_NPEBDPEADI@Z 0000000037505380 f   LiveCreate.obj
 0001:00004420       ?CreatePlatformHandlerInstance@CManager@LiveCreate@@QEAAPEAUIPlatformHandler@2@AEBUSPeerInfo@2@@Z 0000000037505420 f   LiveCreate.obj
 0001:00004510       ?GetPeerInfo@CManager@LiveCreate@@UEAA_NPEAUSPeerLink@2@AEAUSPeerInfo@2@@Z 0000000037505510 f   LiveCreate.obj
 0001:00004590       ?GetPeerAt@CManager@LiveCreate@@UEAAPEAUSPeerLink@2@I@Z 0000000037505590 f   LiveCreate.obj
 0001:000045c0       ?FindLink@CManager@LiveCreate@@IEAAPEAUSPeerLink@2@PEAX@Z 00000000375055c0 f   LiveCreate.obj
 0001:00004610       ?FindLinkByAddress@CManager@LiveCreate@@IEAAPEAUSPeerLink@2@PEBD@Z 0000000037505610 f   LiveCreate.obj
 0001:000047f0       ?clear@?$_Rb_tree@PEAXU?$_BinaryPredWrapper@PEAXPEAUIManagerListener@LiveCreate@@U?$less@PEAUIManagerListener@LiveCreate@@@stlpmtx_std@@@priv@stlpmtx_std@@PEAXU?$_Identity@PEAX@23@U?$_SetTraitsT@PEAX@23@V?$allocator@PEAX@3@@priv@stlpmtx_std@@QEAAXXZ 00000000375057f0 f i LiveCreate.obj
 0001:000047f0       ?clear@?$_Rb_tree@PEAXU?$_BinaryPredWrapper@PEAXPEAUIPlatformHandler@LiveCreate@@U?$less@PEAUIPlatformHandler@LiveCreate@@@stlpmtx_std@@@priv@stlpmtx_std@@PEAXU?$_Identity@PEAX@23@U?$_SetTraitsT@PEAX@23@V?$allocator@PEAX@3@@priv@stlpmtx_std@@QEAAXXZ 00000000375057f0 f i LiveCreateCtrl_Screenshot.obj
 0001:00004860       ?_M_create_node@?$_Rb_tree@PEAXU?$_BinaryPredWrapper@PEAXPEAUIPlatformHandler@LiveCreate@@U?$less@PEAUIPlatformHandler@LiveCreate@@@stlpmtx_std@@@priv@stlpmtx_std@@PEAXU?$_Identity@PEAX@23@U?$_SetTraitsT@PEAX@23@V?$allocator@PEAX@3@@priv@stlpmtx_std@@IEAAPEAU_Rb_tree_node_base@23@AEBQEAX@Z 0000000037505860 f i LiveCreateCtrl_Screenshot.obj
 0001:00004860       ?_M_create_node@?$_Rb_tree@PEAXU?$_BinaryPredWrapper@PEAXPEAUIManagerListener@LiveCreate@@U?$less@PEAUIManagerListener@LiveCreate@@@stlpmtx_std@@@priv@stlpmtx_std@@PEAXU?$_Identity@PEAX@23@U?$_SetTraitsT@PEAX@23@V?$allocator@PEAX@3@@priv@stlpmtx_std@@IEAAPEAU_Rb_tree_node_base@23@AEBQEAX@Z 0000000037505860 f i LiveCreate.obj
 0001:000048c0       ?IsLinkedTo@CManager@LiveCreate@@UEAA_NPEBD@Z 00000000375058c0 f   LiveCreate.obj
 0001:000048e0       ?GetLinkTo@CManager@LiveCreate@@UEAAPEAUSPeerLink@2@PEBD@Z 00000000375058e0 f   LiveCreate.obj
 0001:000048f0       ?SetCustomPlatformName@CManager@LiveCreate@@UEAAXPEBD@Z 00000000375058f0 f   LiveCreate.obj
 0001:00004940       ?OnConnected@CManager@LiveCreate@@IEAAXPEAX@Z 0000000037505940 f   LiveCreate.obj
 0001:00004b60       ?OnDisconnected@CManager@LiveCreate@@IEAAXPEAX@Z 0000000037505b60 f   LiveCreate.obj
 0001:00004ce0       ?_M_insert_overflow@?$_Impl_vector@PEAXV?$allocator@PEAX@stlpmtx_std@@@priv@stlpmtx_std@@AEAAXPEAPEAXAEBQEAXAEBU__true_type@3@_K_N@Z 0000000037505ce0 f i LiveCreate.obj
 0001:00004e50       ??$_M_find@PEBD@?$_Rb_tree@V?$CryStringT@D@@U?$less@V?$CryStringT@D@@@stlpmtx_std@@U?$pair@$$CBV?$CryStringT@D@@PEAUIController@LiveCreate@@@3@U?$_Select1st@U?$pair@$$CBV?$CryStringT@D@@PEAUIController@LiveCreate@@@stlpmtx_std@@@priv@3@U?$_MapTraitsT@U?$pair@$$CBV?$CryStringT@D@@PEAUIController@LiveCreate@@@stlpmtx_std@@@63@V?$allocator@U?$pair@$$CBV?$CryStringT@D@@PEAUIController@LiveCreate@@@stlpmtx_std@@@3@@priv@stlpmtx_std@@AEBAPEAU_Rb_tree_node_base@12@AEBQEBD@Z 0000000037505e50 f i LiveCreate.obj
 0001:00005060       ??$_M_lower_bound@PEBD@?$_Rb_tree@V?$CryStringT@D@@U?$less@V?$CryStringT@D@@@stlpmtx_std@@U?$pair@$$CBV?$CryStringT@D@@PEAUIController@LiveCreate@@@3@U?$_Select1st@U?$pair@$$CBV?$CryStringT@D@@PEAUIController@LiveCreate@@@stlpmtx_std@@@priv@3@U?$_MapTraitsT@U?$pair@$$CBV?$CryStringT@D@@PEAUIController@LiveCreate@@@stlpmtx_std@@@63@V?$allocator@U?$pair@$$CBV?$CryStringT@D@@PEAUIController@LiveCreate@@@stlpmtx_std@@@3@@priv@stlpmtx_std@@AEBAPEAU_Rb_tree_node_base@12@AEBQEBD@Z 0000000037506060 f i LiveCreate.obj
 0001:000051a0       ?UnregisterPlatformHandlerFactory@CManager@LiveCreate@@UEAA_NPEAUIPlatformHandlerFactory@2@@Z 00000000375061a0 f   LiveCreate.obj
 0001:00005230       ?UnregisterListener@CManager@LiveCreate@@UEAA_NPEAUIManagerListener@2@@Z 0000000037506230 f   LiveCreate.obj
 0001:000052b0       ?insert_unique@?$_Rb_tree@PEAXU?$_BinaryPredWrapper@PEAXPEAUIPlatformHandler@LiveCreate@@U?$less@PEAUIPlatformHandler@LiveCreate@@@stlpmtx_std@@@priv@stlpmtx_std@@PEAXU?$_Identity@PEAX@23@U?$_SetTraitsT@PEAX@23@V?$allocator@PEAX@3@@priv@stlpmtx_std@@QEAA?AU?$pair@U?$_Rb_tree_iterator@PEAXU?$_SetTraitsT@PEAX@priv@stlpmtx_std@@@priv@stlpmtx_std@@_N@3@AEBQEAX@Z 00000000375062b0 f i LiveCreateCtrl_Screenshot.obj
 0001:000052b0       ?insert_unique@?$_Rb_tree@PEAXU?$_BinaryPredWrapper@PEAXPEAUIManagerListener@LiveCreate@@U?$less@PEAUIManagerListener@LiveCreate@@@stlpmtx_std@@@priv@stlpmtx_std@@PEAXU?$_Identity@PEAX@23@U?$_SetTraitsT@PEAX@23@V?$allocator@PEAX@3@@priv@stlpmtx_std@@QEAA?AU?$pair@U?$_Rb_tree_iterator@PEAXU?$_SetTraitsT@PEAX@priv@stlpmtx_std@@@priv@stlpmtx_std@@_N@3@AEBQEAX@Z 00000000375062b0 f i LiveCreate.obj
 0001:00005520       ?erase@?$_Rb_tree@V?$CryStringT@D@@U?$less@V?$CryStringT@D@@@stlpmtx_std@@U?$pair@$$CBV?$CryStringT@D@@PEAUIController@LiveCreate@@@3@U?$_Select1st@U?$pair@$$CBV?$CryStringT@D@@PEAUIController@LiveCreate@@@stlpmtx_std@@@priv@3@U?$_MapTraitsT@U?$pair@$$CBV?$CryStringT@D@@PEAUIController@LiveCreate@@@stlpmtx_std@@@63@V?$allocator@U?$pair@$$CBV?$CryStringT@D@@PEAUIController@LiveCreate@@@stlpmtx_std@@@3@@priv@stlpmtx_std@@QEAAXU?$_Rb_tree_iterator@U?$pair@$$CBV?$CryStringT@D@@PEAUIController@LiveCreate@@@stlpmtx_std@@U?$_MapTraitsT@U?$pair@$$CBV?$CryStringT@D@@PEAUIController@LiveCreate@@@stlpmtx_std@@@priv@2@@23@@Z 0000000037506520 f i LiveCreate.obj
 0001:00005590       ?_M_erase@?$_Rb_tree@V?$CryStringT@D@@U?$less@V?$CryStringT@D@@@stlpmtx_std@@V1@U?$_Identity@V?$CryStringT@D@@@priv@3@U?$_SetTraitsT@V?$CryStringT@D@@@53@V?$allocator@V?$CryStringT@D@@@3@@priv@stlpmtx_std@@AEAAXPEAU_Rb_tree_node_base@23@@Z 0000000037506590 f i LiveCreateCtrl_CVar.obj
 0001:00005590       ?_M_erase@?$_Rb_tree@V?$CryStringT@D@@U?$less@V?$CryStringT@D@@@stlpmtx_std@@U?$pair@$$CBV?$CryStringT@D@@PEAUIController@LiveCreate@@@3@U?$_Select1st@U?$pair@$$CBV?$CryStringT@D@@PEAUIController@LiveCreate@@@stlpmtx_std@@@priv@3@U?$_MapTraitsT@U?$pair@$$CBV?$CryStringT@D@@PEAUIController@LiveCreate@@@stlpmtx_std@@@63@V?$allocator@U?$pair@$$CBV?$CryStringT@D@@PEAUIController@LiveCreate@@@stlpmtx_std@@@3@@priv@stlpmtx_std@@AEAAXPEAU_Rb_tree_node_base@23@@Z 0000000037506590 f i LiveCreate.obj
 0001:00005610       ?_M_create_node@?$_Rb_tree@V?$CryStringT@D@@U?$less@V?$CryStringT@D@@@stlpmtx_std@@U?$pair@$$CBV?$CryStringT@D@@PEAUIController@LiveCreate@@@3@U?$_Select1st@U?$pair@$$CBV?$CryStringT@D@@PEAUIController@LiveCreate@@@stlpmtx_std@@@priv@3@U?$_MapTraitsT@U?$pair@$$CBV?$CryStringT@D@@PEAUIController@LiveCreate@@@stlpmtx_std@@@63@V?$allocator@U?$pair@$$CBV?$CryStringT@D@@PEAUIController@LiveCreate@@@stlpmtx_std@@@3@@priv@stlpmtx_std@@IEAAPEAU_Rb_tree_node_base@23@AEBU?$pair@$$CBV?$CryStringT@D@@PEAUIController@LiveCreate@@@3@@Z 0000000037506610 f i LiveCreate.obj
 0001:000056a0       ?RegisterPlatformHandlerFactory@CManager@LiveCreate@@UEAA_NPEAUIPlatformHandlerFactory@2@@Z 00000000375066a0 f   LiveCreate.obj
 0001:00005760       ?RegisterListener@CManager@LiveCreate@@UEAA_NPEAUIManagerListener@2@@Z 0000000037506760 f   LiveCreate.obj
 0001:00005790       ?GetControllerByName@CManager@LiveCreate@@UEAAPEAUIController@2@PEBD@Z 0000000037506790 f   LiveCreate.obj
 0001:000057d0       ?AddPeerLink@CManager@LiveCreate@@QEAAPEAUSPeerLink@2@PEAUIPlatformHandler@2@PEAX@Z 00000000375067d0 f   LiveCreate.obj
 0001:00005990       ?OnReceivedPeerInfo@CManager@LiveCreate@@IEAAXPEAXAEBUSPeerInfo@2@@Z 0000000037506990 f   LiveCreate.obj
 0001:00005b80       ?_M_insert@?$_Rb_tree@V?$CryStringT@D@@U?$less@V?$CryStringT@D@@@stlpmtx_std@@U?$pair@$$CBV?$CryStringT@D@@PEAUIController@LiveCreate@@@3@U?$_Select1st@U?$pair@$$CBV?$CryStringT@D@@PEAUIController@LiveCreate@@@stlpmtx_std@@@priv@3@U?$_MapTraitsT@U?$pair@$$CBV?$CryStringT@D@@PEAUIController@LiveCreate@@@stlpmtx_std@@@63@V?$allocator@U?$pair@$$CBV?$CryStringT@D@@PEAUIController@LiveCreate@@@stlpmtx_std@@@3@@priv@stlpmtx_std@@AEAA?AU?$_Rb_tree_iterator@U?$pair@$$CBV?$CryStringT@D@@PEAUIController@LiveCreate@@@stlpmtx_std@@U?$_MapTraitsT@U?$pair@$$CBV?$CryStringT@D@@PEAUIController@LiveCreate@@@stlpmtx_std@@@priv@2@@23@PEAU_Rb_tree_node_base@23@AEBU?$pair@$$CBV?$CryStringT@D@@PEAUIController@LiveCreate@@@3@00@Z 0000000037506b80 f i LiveCreate.obj
 0001:00005c70       ?insert_unique@?$_Rb_tree@V?$CryStringT@D@@U?$less@V?$CryStringT@D@@@stlpmtx_std@@U?$pair@$$CBV?$CryStringT@D@@PEAUIController@LiveCreate@@@3@U?$_Select1st@U?$pair@$$CBV?$CryStringT@D@@PEAUIController@LiveCreate@@@stlpmtx_std@@@priv@3@U?$_MapTraitsT@U?$pair@$$CBV?$CryStringT@D@@PEAUIController@LiveCreate@@@stlpmtx_std@@@63@V?$allocator@U?$pair@$$CBV?$CryStringT@D@@PEAUIController@LiveCreate@@@stlpmtx_std@@@3@@priv@stlpmtx_std@@QEAA?AU?$pair@U?$_Rb_tree_iterator@U?$pair@$$CBV?$CryStringT@D@@PEAUIController@LiveCreate@@@stlpmtx_std@@U?$_MapTraitsT@U?$pair@$$CBV?$CryStringT@D@@PEAUIController@LiveCreate@@@stlpmtx_std@@@priv@2@@priv@stlpmtx_std@@_N@3@AEBU?$pair@$$CBV?$CryStringT@D@@PEAUIController@LiveCreate@@@3@@Z 0000000037506c70 f i LiveCreate.obj
 0001:00005f00       ??1?$_Impl_vector@V?$CryStringT@D@@V?$allocator@V?$CryStringT@D@@@stlpmtx_std@@@priv@stlpmtx_std@@QEAA@XZ 0000000037506f00 f i LiveCreate.obj
 0001:00005f90       ?UnregisterController@CManager@LiveCreate@@UEAA_NPEAUIController@2@@Z 0000000037506f90 f   LiveCreate.obj
 0001:00006050       ?ConnectToPeer@CManager@LiveCreate@@UEAAPEAUSPeerLink@2@AEBUSPeerInfo@2@@Z 0000000037507050 f   LiveCreate.obj
 0001:00006250       ?AddPeer@CManager@LiveCreate@@UEAAPEAUSPeerLink@2@AEBUSPeerInfo@2@@Z 0000000037507250 f   LiveCreate.obj
 0001:00006280       ?OnReceive@CManager@LiveCreate@@IEAAXPEAXAEBUSNetMessage@2@@Z 0000000037507280 f   LiveCreate.obj
 0001:00006690       ?HandleNetEvents@CManager@LiveCreate@@IEAAXXZ 0000000037507690 f   LiveCreate.obj
 0001:000067d0       ?insert_unique@?$_Rb_tree@V?$CryStringT@D@@U?$less@V?$CryStringT@D@@@stlpmtx_std@@U?$pair@$$CBV?$CryStringT@D@@PEAUIController@LiveCreate@@@3@U?$_Select1st@U?$pair@$$CBV?$CryStringT@D@@PEAUIController@LiveCreate@@@stlpmtx_std@@@priv@3@U?$_MapTraitsT@U?$pair@$$CBV?$CryStringT@D@@PEAUIController@LiveCreate@@@stlpmtx_std@@@63@V?$allocator@U?$pair@$$CBV?$CryStringT@D@@PEAUIController@LiveCreate@@@stlpmtx_std@@@3@@priv@stlpmtx_std@@QEAA?AU?$_Rb_tree_iterator@U?$pair@$$CBV?$CryStringT@D@@PEAUIController@LiveCreate@@@stlpmtx_std@@U?$_MapTraitsT@U?$pair@$$CBV?$CryStringT@D@@PEAUIController@LiveCreate@@@stlpmtx_std@@@priv@2@@23@U423@AEBU?$pair@$$CBV?$CryStringT@D@@PEAUIController@LiveCreate@@@3@@Z 00000000375077d0 f i LiveCreate.obj
 0001:00006c30       ??1CManager@LiveCreate@@UEAA@XZ 0000000037507c30 f   LiveCreate.obj
 0001:00006f00       ??_ECManager@LiveCreate@@W7EAAPEAXI@Z 0000000037507f00 f i LiveCreate.obj
 0001:00006f10       ?Update@CManager@LiveCreate@@UEAAXXZ 0000000037507f10 f   LiveCreate.obj
 0001:00007010       ??_ECManager@LiveCreate@@UEAAPEAXI@Z 0000000037508010 f i LiveCreate.obj
 0001:00007010       ??_GCManager@LiveCreate@@UEAAPEAXI@Z 0000000037508010 f i LiveCreate.obj
 0001:00007040       ??$?APEBD@?$map@V?$CryStringT@D@@PEAUIController@LiveCreate@@U?$less@V?$CryStringT@D@@@stlpmtx_std@@V?$allocator@U?$pair@$$CBV?$CryStringT@D@@PEAUIController@LiveCreate@@@stlpmtx_std@@@5@@stlpmtx_std@@QEAAAEAPEAUIController@LiveCreate@@AEBQEBD@Z 0000000037508040 f i LiveCreate.obj
 0001:00007270       ?RegisterController@CManager@LiveCreate@@UEAA_NPEAUIController@2@@Z 0000000037508270 f   LiveCreate.obj
 0001:00007350       ??0CManager@LiveCreate@@QEAA@PEAUISystem@@@Z 0000000037508350 f   LiveCreate.obj
 0001:00007760       ?GetDisplayName@CameraController@LiveCreate@@UEAAPEBDXZ 0000000037508760 f   LiveCreateCtrl_Camera.obj
 0001:00007770       ?GetUniqueName@CameraController@LiveCreate@@UEAAPEBDXZ 0000000037508770 f   LiveCreateCtrl_Camera.obj
 0001:00007780       ?GetDescription@CameraController@LiveCreate@@UEAAPEBDXZ 0000000037508780 f   LiveCreateCtrl_Camera.obj
 0001:00007790       ?OnEndSendToPeers@CameraController@LiveCreate@@UEAAXXZ 0000000037508790 f   LiveCreateCtrl_Camera.obj
 0001:00007790       ?OnEndSendToPeers@CommonController@LiveCreate@@UEAAXXZ 0000000037508790 f   LiveCreateCtrl_Common.obj
 0001:00007790       ?OnEndSendToPeers@ScreenshotController@LiveCreate@@UEAAXXZ 0000000037508790 f   LiveCreateCtrl_Screenshot.obj
 0001:000077a0       ?CommitData@CameraController@LiveCreate@@UEAAXPEBDPEAXH@Z 00000000375087a0 f   LiveCreateCtrl_Camera.obj
 0001:00007850       ??0SViewParams@@QEAA@XZ    0000000037508850 f i LiveCreateCtrl_Camera.obj
 0001:00007910       ??_GCameraController@LiveCreate@@UEAAPEAXI@Z 0000000037508910 f i LiveCreateCtrl_Camera.obj
 0001:00007910       ??_ECameraController@LiveCreate@@UEAAPEAXI@Z 0000000037508910 f i LiveCreateCtrl_Camera.obj
 0001:00007950       ??4SViewParams@@QEAAAEAU0@AEBU0@@Z 0000000037508950 f i LiveCreateCtrl_Camera.obj
 0001:00007b10       ??0CameraController@LiveCreate@@QEAA@XZ 0000000037508b10 f   LiveCreateCtrl_Camera.obj
 0001:00007b70       ?OnReceive@CameraController@LiveCreate@@UEAAXPEAUSPeerLink@2@AEBUSDataSync@IController@2@@Z 0000000037508b70 f   LiveCreateCtrl_Camera.obj
 0001:00007da0       ?OnSend@CameraController@LiveCreate@@UEAA_NPEAUSPeerLink@2@AEAUSDataSync@IController@2@@Z 0000000037508da0 f   LiveCreateCtrl_Camera.obj
 0001:00007fd0       ?OnUpdate@CameraController@LiveCreate@@UEAAXXZ 0000000037508fd0 f   LiveCreateCtrl_Camera.obj
 0001:00008da0       ?SetEnabled@CommonController@LiveCreate@@UEAAX_N@Z 0000000037509da0 f   LiveCreateCtrl_Common.obj
 0001:00008db0       ?IsEnabled@CommonController@LiveCreate@@UEAA_NXZ 0000000037509db0 f   LiveCreateCtrl_Common.obj
 0001:00008dc0       ?NeedsToSend@CommonController@LiveCreate@@UEAA_NXZ 0000000037509dc0 f   LiveCreateCtrl_Common.obj
 0001:00008dd0       ?OnReceive@CommonController@LiveCreate@@UEAAXPEAUSPeerLink@2@AEBUSDataSync@IController@2@@Z 0000000037509dd0 f   LiveCreateCtrl_Common.obj
 0001:00008de0       ?CommitData@CommonController@LiveCreate@@UEAAXPEBDPEAXH@Z 0000000037509de0 f   LiveCreateCtrl_Common.obj
 0001:00008df0       ??0CommonController@LiveCreate@@QEAA@XZ 0000000037509df0 f   LiveCreateCtrl_Common.obj
 0001:00008e10       ??1CommonController@LiveCreate@@UEAA@XZ 0000000037509e10 f   LiveCreateCtrl_Common.obj
 0001:00008e20       ??_EIController@LiveCreate@@UEAAPEAXI@Z 0000000037509e20 f i LiveCreateCtrl_Common.obj
 0001:00008e20       ??_GCommonController@LiveCreate@@UEAAPEAXI@Z 0000000037509e20 f i LiveCreateCtrl_Common.obj
 0001:00008e20       ??_ECommonController@LiveCreate@@UEAAPEAXI@Z 0000000037509e20 f i LiveCreateCtrl_Common.obj
 0001:00008e20       ??_GIController@LiveCreate@@UEAAPEAXI@Z 0000000037509e20 f i LiveCreateCtrl_Common.obj
 0001:00008e50       ?GetDisplayName@CVarController@LiveCreate@@UEAAPEBDXZ 0000000037509e50 f   LiveCreateCtrl_CVar.obj
 0001:00008e60       ?GetUniqueName@CVarController@LiveCreate@@UEAAPEBDXZ 0000000037509e60 f   LiveCreateCtrl_CVar.obj
 0001:00008e70       ?GetDescription@CVarController@LiveCreate@@UEAAPEBDXZ 0000000037509e70 f   LiveCreateCtrl_CVar.obj
 0001:00008e80       ?OnRegistered@CVarController@LiveCreate@@UEAAXPEAUIManager@2@@Z 0000000037509e80 f   LiveCreateCtrl_CVar.obj
 0001:00008eb0       ?OnUnregistered@CVarController@LiveCreate@@UEAAXPEAUIManager@2@@Z 0000000037509eb0 f   LiveCreateCtrl_CVar.obj
 0001:00008ef0       ??_EIConsoleVarSink@@UEAAPEAXI@Z 0000000037509ef0 f i LiveCreateCtrl_CVar.obj
 0001:00008ef0       ??_GIConsoleVarSink@@UEAAPEAXI@Z 0000000037509ef0 f i LiveCreateCtrl_CVar.obj
 0001:00008f20       ?_M_compute_next_size@?$_Impl_vector@UCVarData@CVarController@LiveCreate@@V?$allocator@UCVarData@CVarController@LiveCreate@@@stlpmtx_std@@@priv@stlpmtx_std@@AEAA_K_K@Z 0000000037509f20 f i LiveCreateCtrl_CVar.obj
 0001:00008fb0       ??$__find@PEAV?$CryStringT@D@@V1@@priv@stlpmtx_std@@YAPEAV?$CryStringT@D@@PEAV2@0AEBV2@AEBUrandom_access_iterator_tag@1@@Z 0000000037509fb0 f i LiveCreateCtrl_CVar.obj
 0001:00008fb0       ??$__find@PEAV?$CryStringT@D@@PEAD@priv@stlpmtx_std@@YAPEAV?$CryStringT@D@@PEAV2@0AEBQEADAEBUrandom_access_iterator_tag@1@@Z 0000000037509fb0 f i LiveCreateCtrl_CVar.obj
 0001:00009190       ?OnSend@CVarController@LiveCreate@@UEAA_NPEAUSPeerLink@2@AEAUSDataSync@IController@2@@Z 000000003750a190 f   LiveCreateCtrl_CVar.obj
 0001:00009330       ??$__copy@PEAV?$CryStringT@D@@PEAV1@_J@priv@stlpmtx_std@@YAPEAV?$CryStringT@D@@PEAV2@00AEBUrandom_access_iterator_tag@1@PEA_J@Z 000000003750a330 f i LiveCreateCtrl_CVar.obj
 0001:00009420       ?_M_create_node@?$_Rb_tree@V?$CryStringT@D@@U?$less@V?$CryStringT@D@@@stlpmtx_std@@V1@U?$_Identity@V?$CryStringT@D@@@priv@3@U?$_SetTraitsT@V?$CryStringT@D@@@53@V?$allocator@V?$CryStringT@D@@@3@@priv@stlpmtx_std@@IEAAPEAU_Rb_tree_node_base@23@AEBV?$CryStringT@D@@@Z 000000003750a420 f i LiveCreateCtrl_CVar.obj
 0001:000094a0       ?push_back@?$_Impl_vector@UCVarData@CVarController@LiveCreate@@V?$allocator@UCVarData@CVarController@LiveCreate@@@stlpmtx_std@@@priv@stlpmtx_std@@QEAAXAEBUCVarData@CVarController@LiveCreate@@@Z 000000003750a4a0 f i LiveCreateCtrl_CVar.obj
 0001:000095e0       ?insert_unique@?$_Rb_tree@V?$CryStringT@D@@U?$less@V?$CryStringT@D@@@stlpmtx_std@@V1@U?$_Identity@V?$CryStringT@D@@@priv@3@U?$_SetTraitsT@V?$CryStringT@D@@@53@V?$allocator@V?$CryStringT@D@@@3@@priv@stlpmtx_std@@QEAA?AU?$pair@U?$_Rb_tree_iterator@V?$CryStringT@D@@U?$_SetTraitsT@V?$CryStringT@D@@@priv@stlpmtx_std@@@priv@stlpmtx_std@@_N@3@AEBV?$CryStringT@D@@@Z 000000003750a5e0 f i LiveCreateCtrl_CVar.obj
 0001:00009870       ?OnReceive@CVarController@LiveCreate@@UEAAXPEAUSPeerLink@2@AEBUSDataSync@IController@2@@Z 000000003750a870 f   LiveCreateCtrl_CVar.obj
 0001:000099b0       ?_M_clear_after_move@?$_Impl_vector@V?$CryStringT@D@@V?$allocator@V?$CryStringT@D@@@stlpmtx_std@@@priv@stlpmtx_std@@AEAAXXZ 000000003750a9b0 f i LiveCreateCtrl_CVar.obj
 0001:00009a30       ?OnUpdate@CVarController@LiveCreate@@UEAAXXZ 000000003750aa30 f   LiveCreateCtrl_CVar.obj
 0001:00009bd0       ?_M_erase@?$_Impl_vector@V?$CryStringT@D@@V?$allocator@V?$CryStringT@D@@@stlpmtx_std@@@priv@stlpmtx_std@@AEAAPEAV?$CryStringT@D@@PEAV4@0AEBU__false_type@3@@Z 000000003750abd0 f i LiveCreateCtrl_CVar.obj
 0001:00009c90       ?_M_insert_overflow_aux@?$_Impl_vector@V?$CryStringT@D@@V?$allocator@V?$CryStringT@D@@@stlpmtx_std@@@priv@stlpmtx_std@@AEAAXPEAV?$CryStringT@D@@AEBV4@AEBU__false_type@3@_K_N@Z 000000003750ac90 f i LiveCreateCtrl_CVar.obj
 0001:00009e80       ??0CVarController@LiveCreate@@QEAA@XZ 000000003750ae80 f   LiveCreateCtrl_CVar.obj
 0001:0000a070       ??_ECVarController@LiveCreate@@WBA@EAAPEAXI@Z 000000003750b070 f i LiveCreateCtrl_CVar.obj
 0001:0000a080       ??1CVarController@LiveCreate@@UEAA@XZ 000000003750b080 f   LiveCreateCtrl_CVar.obj
 0001:0000a130       ?push_back@?$_Impl_vector@V?$CryStringT@D@@V?$allocator@V?$CryStringT@D@@@stlpmtx_std@@@priv@stlpmtx_std@@QEAAXAEBV?$CryStringT@D@@@Z 000000003750b130 f i LiveCreateCtrl_CVar.obj
 0001:0000a1b0       ??_ECVarController@LiveCreate@@UEAAPEAXI@Z 000000003750b1b0 f i LiveCreateCtrl_CVar.obj
 0001:0000a1b0       ??_GCVarController@LiveCreate@@UEAAPEAXI@Z 000000003750b1b0 f i LiveCreateCtrl_CVar.obj
 0001:0000a1e0       ?OnAfterVarChange@CVarController@LiveCreate@@UEAAXPEAUICVar@@@Z 000000003750b1e0 f   LiveCreateCtrl_CVar.obj
 0001:0000a580       ?OnEndSendToPeers@CVarController@LiveCreate@@UEAAXXZ 000000003750b580 f   LiveCreateCtrl_CVar.obj
 0001:0000a5b0       ?CommitData@CVarController@LiveCreate@@UEAAXPEBDPEAXH@Z 000000003750b5b0 f   LiveCreateCtrl_CVar.obj
 0001:0000a960       ?GetDisplayName@EntitiesController@LiveCreate@@UEAAPEBDXZ 000000003750b960 f   LiveCreateCtrl_Entities.obj
 0001:0000a970       ?GetUniqueName@EntitiesController@LiveCreate@@UEAAPEBDXZ 000000003750b970 f   LiveCreateCtrl_Entities.obj
 0001:0000a980       ?GetDescription@EntitiesController@LiveCreate@@UEAAPEBDXZ 000000003750b980 f   LiveCreateCtrl_Entities.obj
 0001:0000a990       ??$__copy_backward@PEAUSTransformData@EntitiesController@LiveCreate@@PEAU123@_J@priv@stlpmtx_std@@YAPEAUSTransformData@EntitiesController@LiveCreate@@PEAU234@00AEBUrandom_access_iterator_tag@1@PEA_J@Z 000000003750b990 f i LiveCreateCtrl_Entities.obj
 0001:0000abd0       ??$__fill@PEAUSTransformData@EntitiesController@LiveCreate@@U123@_J@priv@stlpmtx_std@@YAXPEAUSTransformData@EntitiesController@LiveCreate@@0AEBU234@AEBUrandom_access_iterator_tag@1@PEA_J@Z 000000003750bbd0 f i LiveCreateCtrl_Entities.obj
 0001:0000ae00       ?_M_compute_next_size@?$_Impl_vector@USTransformData@EntitiesController@LiveCreate@@V?$allocator@USTransformData@EntitiesController@LiveCreate@@@stlpmtx_std@@@priv@stlpmtx_std@@AEAA_K_K@Z 000000003750be00 f i LiveCreateCtrl_Entities.obj
 0001:0000ae90       ??$__copy@PEAUSTransformData@EntitiesController@LiveCreate@@PEAU123@_J@priv@stlpmtx_std@@YAPEAUSTransformData@EntitiesController@LiveCreate@@PEAU234@00AEBUrandom_access_iterator_tag@1@PEA_J@Z 000000003750be90 f i LiveCreateCtrl_Entities.obj
 0001:0000b0c0       ?OnSend@EntitiesController@LiveCreate@@UEAA_NPEAUSPeerLink@2@AEAUSDataSync@IController@2@@Z 000000003750c0c0 f   LiveCreateCtrl_Entities.obj
 0001:0000b710       ??$__copy_backward@PEAV?$CryStringT@D@@PEAV1@_J@priv@stlpmtx_std@@YAPEAV?$CryStringT@D@@PEAV2@00AEBUrandom_access_iterator_tag@1@PEA_J@Z 000000003750c710 f i LiveCreateCtrl_Entities.obj
 0001:0000b800       ??$__fill@PEAV?$CryStringT@D@@V1@_J@priv@stlpmtx_std@@YAXPEAV?$CryStringT@D@@0AEBV2@AEBUrandom_access_iterator_tag@1@PEA_J@Z 000000003750c800 f i LiveCreateCtrl_Entities.obj
 0001:0000b8e0       ?_M_insert_overflow@?$_Impl_vector@IV?$allocator@I@stlpmtx_std@@@priv@stlpmtx_std@@AEAAXPEAIAEBIAEBU__true_type@3@_K_N@Z 000000003750c8e0 f i LiveCreateCtrl_Entities.obj
 0001:0000ba50       ??$__uninitialized_fill_n@PEAUSTransformData@EntitiesController@LiveCreate@@_KU123@@priv@stlpmtx_std@@YAPEAUSTransformData@EntitiesController@LiveCreate@@PEAU234@_KAEBU234@@Z 000000003750ca50 f i LiveCreateCtrl_Entities.obj
 0001:0000bb00       ?_M_fill_insert_aux@?$_Impl_vector@IV?$allocator@I@stlpmtx_std@@@priv@stlpmtx_std@@AEAAXPEAI_KAEBIAEBU__false_type@3@@Z 000000003750cb00 f i LiveCreateCtrl_Entities.obj
 0001:0000bc90       ?_M_fill_insert_aux@?$_Impl_vector@DV?$allocator@D@stlpmtx_std@@@priv@stlpmtx_std@@AEAAXPEAD_KAEBDAEBU__false_type@3@@Z 000000003750cc90 f i LiveCreateCtrl_Entities.obj
 0001:0000bdd0       ??$__ucopy_ptrs@PEAUSTransformData@EntitiesController@LiveCreate@@PEAU123@@priv@stlpmtx_std@@YAPEAUSTransformData@EntitiesController@LiveCreate@@PEAU234@00AEBU__false_type@1@@Z 000000003750cdd0 f i LiveCreateCtrl_Entities.obj
 0001:0000be80       ?_M_fill_insert_aux@?$_Impl_vector@USTransformData@EntitiesController@LiveCreate@@V?$allocator@USTransformData@EntitiesController@LiveCreate@@@stlpmtx_std@@@priv@stlpmtx_std@@AEAAXPEAUSTransformData@EntitiesController@LiveCreate@@_KAEBU456@AEBU__false_type@3@@Z 000000003750ce80 f i LiveCreateCtrl_Entities.obj
 0001:0000c060       ?_M_fill_insert_aux@?$_Impl_vector@V?$CryStringT@D@@V?$allocator@V?$CryStringT@D@@@stlpmtx_std@@@priv@stlpmtx_std@@AEAAXPEAV?$CryStringT@D@@_KAEBV4@AEBU__false_type@3@@Z 000000003750d060 f i LiveCreateCtrl_Entities.obj
 0001:0000c290       ?_M_insert_overflow_aux@?$_Impl_vector@USTransformData@EntitiesController@LiveCreate@@V?$allocator@USTransformData@EntitiesController@LiveCreate@@@stlpmtx_std@@@priv@stlpmtx_std@@AEAAXPEAUSTransformData@EntitiesController@LiveCreate@@AEBU456@AEBU__false_type@3@_K_N@Z 000000003750d290 f i LiveCreateCtrl_Entities.obj
 0001:0000c400       ?clear@?$vector@USTransformData@EntitiesController@LiveCreate@@V?$allocator@USTransformData@EntitiesController@LiveCreate@@@stlpmtx_std@@@stlpmtx_std@@QEAAXXZ 000000003750d400 f i LiveCreateCtrl_Entities.obj
 0001:0000c450       ?push_back@?$_Impl_vector@USTransformData@EntitiesController@LiveCreate@@V?$allocator@USTransformData@EntitiesController@LiveCreate@@@stlpmtx_std@@@priv@stlpmtx_std@@QEAAXAEBUSTransformData@EntitiesController@LiveCreate@@@Z 000000003750d450 f i LiveCreateCtrl_Entities.obj
 0001:0000c5f0       ??0EntitiesController@LiveCreate@@QEAA@XZ 000000003750d5f0 f   LiveCreateCtrl_Entities.obj
 0001:0000c6a0       ??1EntitiesController@LiveCreate@@UEAA@XZ 000000003750d6a0 f   LiveCreateCtrl_Entities.obj
 0001:0000c720       ??_GEntitiesController@LiveCreate@@UEAAPEAXI@Z 000000003750d720 f i LiveCreateCtrl_Entities.obj
 0001:0000c720       ??_EEntitiesController@LiveCreate@@UEAAPEAXI@Z 000000003750d720 f i LiveCreateCtrl_Entities.obj
 0001:0000c750       ?OnUpdate@EntitiesController@LiveCreate@@UEAAXXZ 000000003750d750 f   LiveCreateCtrl_Entities.obj
 0001:0000cee0       ?OnEndSendToPeers@EntitiesController@LiveCreate@@UEAAXXZ 000000003750dee0 f   LiveCreateCtrl_Entities.obj
 0001:0000cf70       ?CommitData@EntitiesController@LiveCreate@@UEAAXPEBDPEAXH@Z 000000003750df70 f   LiveCreateCtrl_Entities.obj
 0001:0000d520       ?OnReceive@EntitiesController@LiveCreate@@UEAAXPEAUSPeerLink@2@AEBUSDataSync@IController@2@@Z 000000003750e520 f   LiveCreateCtrl_Entities.obj
 0001:0000e200       ?GetDisplayName@ExecuteConsoleStringController@LiveCreate@@UEAAPEBDXZ 000000003750f200 f   LiveCreateCtrl_ExecuteConsoleString.obj
 0001:0000e210       ?GetUniqueName@ExecuteConsoleStringController@LiveCreate@@UEAAPEBDXZ 000000003750f210 f   LiveCreateCtrl_ExecuteConsoleString.obj
 0001:0000e220       ?GetDescription@ExecuteConsoleStringController@LiveCreate@@UEAAPEBDXZ 000000003750f220 f   LiveCreateCtrl_ExecuteConsoleString.obj
 0001:0000e230       ?OnSend@ExecuteConsoleStringController@LiveCreate@@UEAA_NPEAUSPeerLink@2@AEAUSDataSync@IController@2@@Z 000000003750f230 f   LiveCreateCtrl_ExecuteConsoleString.obj
 0001:0000e360       ??1ExecuteConsoleStringController@LiveCreate@@UEAA@XZ 000000003750f360 f   LiveCreateCtrl_ExecuteConsoleString.obj
 0001:0000e3e0       ?erase@?$_Impl_vector@USConsoleString@ExecuteConsoleStringController@LiveCreate@@V?$allocator@USConsoleString@ExecuteConsoleStringController@LiveCreate@@@stlpmtx_std@@@priv@stlpmtx_std@@QEAAPEAUSConsoleString@ExecuteConsoleStringController@LiveCreate@@PEAU456@0@Z 000000003750f3e0 f i LiveCreateCtrl_ExecuteConsoleString.obj
 0001:0000e3e0       ?erase@?$_Impl_vector@USChangedFileName@FileChangeNotifyController@LiveCreate@@V?$allocator@USChangedFileName@FileChangeNotifyController@LiveCreate@@@stlpmtx_std@@@priv@stlpmtx_std@@QEAAPEAUSChangedFileName@FileChangeNotifyController@LiveCreate@@PEAU456@0@Z 000000003750f3e0 f i LiveCreateCtrl_FileChangeNotify.obj
 0001:0000e3e0       ?erase@?$_Impl_vector@UCVarData@CVarController@LiveCreate@@V?$allocator@UCVarData@CVarController@LiveCreate@@@stlpmtx_std@@@priv@stlpmtx_std@@QEAAPEAUCVarData@CVarController@LiveCreate@@PEAU456@0@Z 000000003750f3e0 f i LiveCreateCtrl_CVar.obj
 0001:0000e3e0       ?erase@?$_Impl_vector@IV?$allocator@I@stlpmtx_std@@@priv@stlpmtx_std@@QEAAPEAIPEAI0@Z 000000003750f3e0 f i LiveCreateCtrl_Entities.obj
 0001:0000e460       ??_EExecuteConsoleStringController@LiveCreate@@UEAAPEAXI@Z 000000003750f460 f i LiveCreateCtrl_ExecuteConsoleString.obj
 0001:0000e460       ??_GExecuteConsoleStringController@LiveCreate@@UEAAPEAXI@Z 000000003750f460 f i LiveCreateCtrl_ExecuteConsoleString.obj
 0001:0000e490       ??0ExecuteConsoleStringController@LiveCreate@@QEAA@XZ 000000003750f490 f   LiveCreateCtrl_ExecuteConsoleString.obj
 0001:0000e510       ?OnReceive@ExecuteConsoleStringController@LiveCreate@@UEAAXPEAUSPeerLink@2@AEBUSDataSync@IController@2@@Z 000000003750f510 f   LiveCreateCtrl_ExecuteConsoleString.obj
 0001:0000e940       ?CommitData@ExecuteConsoleStringController@LiveCreate@@UEAAXPEBDPEAXH@Z 000000003750f940 f   LiveCreateCtrl_ExecuteConsoleString.obj
 0001:0000eb00       ?OnUpdate@ExecuteConsoleStringController@LiveCreate@@UEAAXXZ 000000003750fb00 f   LiveCreateCtrl_ExecuteConsoleString.obj
 0001:0000ec00       ?OnEndSendToPeers@ExecuteConsoleStringController@LiveCreate@@UEAAXXZ 000000003750fc00 f   LiveCreateCtrl_ExecuteConsoleString.obj
 0001:0000ec00       ?OnEndSendToPeers@FileChangeNotifyController@LiveCreate@@UEAAXXZ 000000003750fc00 f   LiveCreateCtrl_FileChangeNotify.obj
 0001:0000ec30       ?GetDisplayName@FileChangeNotifyController@LiveCreate@@UEAAPEBDXZ 000000003750fc30 f   LiveCreateCtrl_FileChangeNotify.obj
 0001:0000ec40       ?GetUniqueName@FileChangeNotifyController@LiveCreate@@UEAAPEBDXZ 000000003750fc40 f   LiveCreateCtrl_FileChangeNotify.obj
 0001:0000ec50       ?GetDescription@FileChangeNotifyController@LiveCreate@@UEAAPEBDXZ 000000003750fc50 f   LiveCreateCtrl_FileChangeNotify.obj
 0001:0000ec60       ?OnSend@FileChangeNotifyController@LiveCreate@@UEAA_NPEAUSPeerLink@2@AEAUSDataSync@IController@2@@Z 000000003750fc60 f   LiveCreateCtrl_FileChangeNotify.obj
 0001:0000ed90       ?ToUnixPath@PathUtil@@YA?AV?$CryStringT@D@@AEBV2@@Z 000000003750fd90 f i LiveCreateCtrl_FileChangeNotify.obj
 0001:0000eec0       ?CommitData@FileChangeNotifyController@LiveCreate@@UEAAXPEBDPEAXH@Z 000000003750fec0 f   LiveCreateCtrl_FileChangeNotify.obj
 0001:0000f080       ?AddSlash@PathUtil@@YA?AV?$CryStringT@D@@AEBV2@@Z 0000000037510080 f i LiveCreateCtrl_FileChangeNotify.obj
 0001:0000f220       ?MakeGamePath@PathUtil@@YA?AV?$CryStringT@D@@AEBV2@@Z 0000000037510220 f i LiveCreateCtrl_FileChangeNotify.obj
 0001:0000f460       ??0FileChangeNotifyController@LiveCreate@@QEAA@XZ 0000000037510460 f   LiveCreateCtrl_FileChangeNotify.obj
 0001:0000f4e0       ??_EFileChangeNotifyController@LiveCreate@@UEAAPEAXI@Z 00000000375104e0 f i LiveCreateCtrl_FileChangeNotify.obj
 0001:0000f4e0       ??_GFileChangeNotifyController@LiveCreate@@UEAAPEAXI@Z 00000000375104e0 f i LiveCreateCtrl_FileChangeNotify.obj
 0001:0000f560       ?OnUpdate@FileChangeNotifyController@LiveCreate@@UEAAXXZ 0000000037510560 f   LiveCreateCtrl_FileChangeNotify.obj
 0001:0000f920       ?OnReceive@FileChangeNotifyController@LiveCreate@@UEAAXPEAUSPeerLink@2@AEBUSDataSync@IController@2@@Z 0000000037510920 f   LiveCreateCtrl_FileChangeNotify.obj
 0001:0000fe40       ?GetDisplayName@ScreenshotController@LiveCreate@@UEAAPEBDXZ 0000000037510e40 f   LiveCreateCtrl_Screenshot.obj
 0001:0000fe50       ?GetUniqueName@ScreenshotController@LiveCreate@@UEAAPEBDXZ 0000000037510e50 f   LiveCreateCtrl_Screenshot.obj
 0001:0000fe60       ?GetDescription@ScreenshotController@LiveCreate@@UEAAPEBDXZ 0000000037510e60 f   LiveCreateCtrl_Screenshot.obj
 0001:0000fe70       ?OnUpdate@ScreenshotController@LiveCreate@@UEAAXXZ 0000000037510e70 f   LiveCreateCtrl_Screenshot.obj
 0001:0000fed0       ?Format@?$CryStringT@D@@QEAAAEAV1@PEBDZZ 0000000037510ed0 f i LiveCreateCtrl_Screenshot.obj
 0001:0000ff60       ?clear@?$CryStringT@D@@QEAAXXZ 0000000037510f60 f i LiveCreateCtrl_Screenshot.obj
 0001:0000ffd0       ?OnSend@ScreenshotController@LiveCreate@@UEAA_NPEAUSPeerLink@2@AEAUSDataSync@IController@2@@Z 0000000037510fd0 f   LiveCreateCtrl_Screenshot.obj
 0001:00010110       ?AddSlash@PathUtil@@YA?AV?$CryStringT@D@@PEBD@Z 0000000037511110 f i LiveCreateCtrl_Screenshot.obj
 0001:000101f0       ?OnReceive@ScreenshotController@LiveCreate@@UEAAXPEAUSPeerLink@2@AEBUSDataSync@IController@2@@Z 00000000375111f0 f   LiveCreateCtrl_Screenshot.obj
 0001:00010d00       ?CommitData@ScreenshotController@LiveCreate@@UEAAXPEBDPEAXH@Z 0000000037511d00 f   LiveCreateCtrl_Screenshot.obj
 0001:00010d60       ??0ScreenshotController@LiveCreate@@QEAA@XZ 0000000037511d60 f   LiveCreateCtrl_Screenshot.obj
 0001:00010e10       ??1ScreenshotController@LiveCreate@@UEAA@XZ 0000000037511e10 f   LiveCreateCtrl_Screenshot.obj
 0001:00010e90       ??_EScreenshotController@LiveCreate@@UEAAPEAXI@Z 0000000037511e90 f i LiveCreateCtrl_Screenshot.obj
 0001:00010e90       ??_GScreenshotController@LiveCreate@@UEAAPEAXI@Z 0000000037511e90 f i LiveCreateCtrl_Screenshot.obj
 0001:00010ec0       ??_ECryRunnable@@UEAAPEAXI@Z 0000000037511ec0 f i LiveCreateFileSync.obj
 0001:00010ec0       ??_GCryRunnable@@UEAAPEAXI@Z 0000000037511ec0 f i LiveCreateFileSync.obj
 0001:00010ef0       ?MatchWildcard@PathUtil@@YA_NPEBD0@Z 0000000037511ef0 f i LiveCreateFileSync.obj
 0001:00010fe0       ?Cancel@?$CrySimpleThread@VNetPeerServerAcceptThread@LiveCreate@@@@UEAAXXZ 0000000037511fe0 f i LiveCreateNetwork.obj
 0001:00010fe0       ?Cancel@?$CrySimpleThread@VFileSyncManager@LiveCreate@@@@UEAAXXZ 0000000037511fe0 f i LiveCreateFileSync.obj
 0001:00010fe0       ?Cancel@?$CrySimpleThread@VNetPeerCommThread@LiveCreate@@@@UEAAXXZ 0000000037511fe0 f i LiveCreateNetwork.obj
 0001:00011010       ?IsFileSyncGroupDone@FileSyncManager@LiveCreate@@QEAA_NH@Z 0000000037512010 f   LiveCreateFileSync.obj
 0001:000110b0       ??1SFileItem@FileSyncManager@LiveCreate@@QEAA@XZ 00000000375120b0 f i LiveCreateFileSync.obj
 0001:00011150       ?IsFileIgnored@FileSyncManager@LiveCreate@@QEAA_NPEBD@Z 0000000037512150 f   LiveCreateFileSync.obj
 0001:00011280       ?Run@?$CrySimpleThread@VFileSyncManager@LiveCreate@@@@UEAAXXZ 0000000037512280 f i LiveCreateFileSync.obj
 0001:00011280       ?Run@?$CrySimpleThread@VNetPeerServerAcceptThread@LiveCreate@@@@UEAAXXZ 0000000037512280 f i LiveCreateNetwork.obj
 0001:00011280       ?Run@?$CrySimpleThread@VNetPeerCommThread@LiveCreate@@@@UEAAXXZ 0000000037512280 f i LiveCreateNetwork.obj
 0001:000112a0       ?RunThis@?$CrySimpleThread@VNetPeerServerAcceptThread@LiveCreate@@@@CAIPEAX@Z 00000000375122a0 f i LiveCreateNetwork.obj
 0001:000112a0       ?RunThis@?$CrySimpleThread@VNetPeerCommThread@LiveCreate@@@@CAIPEAX@Z 00000000375122a0 f i LiveCreateNetwork.obj
 0001:000112a0       ?RunThis@?$CrySimpleThread@VFileSyncManager@LiveCreate@@@@CAIPEAX@Z 00000000375122a0 f i LiveCreateFileSync.obj
 0001:000112e0       ??0SFileItem@FileSyncManager@LiveCreate@@QEAA@PEBD0H0@Z 00000000375122e0 f i LiveCreateFileSync.obj
 0001:000113c0       ?_M_erase@?$_Impl_vector@USFileItem@FileSyncManager@LiveCreate@@V?$allocator@USFileItem@FileSyncManager@LiveCreate@@@stlpmtx_std@@@priv@stlpmtx_std@@AEAAPEAUSFileItem@FileSyncManager@LiveCreate@@PEAU456@AEBU__false_type@3@@Z 00000000375123c0 f i LiveCreateFileSync.obj
 0001:00011480       ??$__uninitialized_fill_n@PEAUSFileItem@FileSyncManager@LiveCreate@@_KU123@@priv@stlpmtx_std@@YAPEAUSFileItem@FileSyncManager@LiveCreate@@PEAU234@_KAEBU234@@Z 0000000037512480 f i LiveCreateFileSync.obj
 0001:00011510       ?_M_erase@?$_Impl_vector@USFileItem@FileSyncManager@LiveCreate@@V?$allocator@USFileItem@FileSyncManager@LiveCreate@@@stlpmtx_std@@@priv@stlpmtx_std@@AEAAPEAUSFileItem@FileSyncManager@LiveCreate@@PEAU456@0AEBU__false_type@3@@Z 0000000037512510 f i LiveCreateFileSync.obj
 0001:000115f0       ?_M_insert_overflow_aux@?$_Impl_vector@USFileItem@FileSyncManager@LiveCreate@@V?$allocator@USFileItem@FileSyncManager@LiveCreate@@@stlpmtx_std@@@priv@stlpmtx_std@@AEAAXPEAUSFileItem@FileSyncManager@LiveCreate@@AEBU456@AEBU__false_type@3@_K_N@Z 00000000375125f0 f i LiveCreateFileSync.obj
 0001:00011890       ??1FileSyncManager@LiveCreate@@UEAA@XZ 0000000037512890 f   LiveCreateFileSync.obj
 0001:000119a0       ??_EFileSyncManager@LiveCreate@@W7EAAPEAXI@Z 00000000375129a0 f i LiveCreateFileSync.obj
 0001:000119b0       ?ProcessNextFile@FileSyncManager@LiveCreate@@AEAA_NXZ 00000000375129b0 f   LiveCreateFileSync.obj
 0001:00012070       ?Run@FileSyncManager@LiveCreate@@UEAAXXZ 0000000037513070 f   LiveCreateFileSync.obj
 0001:000120c0       ??_GFileSyncManager@LiveCreate@@UEAAPEAXI@Z 00000000375130c0 f i LiveCreateFileSync.obj
 0001:000120c0       ??_EFileSyncManager@LiveCreate@@UEAAPEAXI@Z 00000000375130c0 f i LiveCreateFileSync.obj
 0001:000120f0       ?push_back@?$_Impl_vector@USFileItem@FileSyncManager@LiveCreate@@V?$allocator@USFileItem@FileSyncManager@LiveCreate@@@stlpmtx_std@@@priv@stlpmtx_std@@QEAAXAEBUSFileItem@FileSyncManager@LiveCreate@@@Z 00000000375130f0 f i LiveCreateFileSync.obj
 0001:000121a0       ??0FileSyncManager@LiveCreate@@QEAA@XZ 00000000375131a0 f   LiveCreateFileSync.obj
 0001:00012c10       ?AbortSync@FileSyncManager@LiveCreate@@QEAAXXZ 0000000037513c10 f   LiveCreateFileSync.obj
 0001:00012c70       ?AddFile@FileSyncManager@LiveCreate@@QEAA_NPEBD0H0@Z 0000000037513c70 f   LiveCreateFileSync.obj
 0001:00012d50       ?Create@NetSocket@LiveCreate@@QEAA_NW4EType@12@_K_N@Z 0000000037513d50 f   LiveCreateNetSocket.obj
 0001:00012f10       ?Bind@NetSocket@LiveCreate@@QEAA_NG@Z 0000000037513f10 f   LiveCreateNetSocket.obj
 0001:00013000       ?Listen@NetSocket@LiveCreate@@QEAA_NI@Z 0000000037514000 f   LiveCreateNetSocket.obj
 0001:00013070       ?Accept@NetSocket@LiveCreate@@QEAA_KPEAUsockaddr@@AEAH@Z 0000000037514070 f   LiveCreateNetSocket.obj
 0001:000130b0       ?Close@NetSocket@LiveCreate@@QEAAXXZ 00000000375140b0 f   LiveCreateNetSocket.obj
 0001:00013110       ?IsLocalAddress@NetSocket@LiveCreate@@QEAA_NPEBD@Z 0000000037514110 f   LiveCreateNetSocket.obj
 0001:000131e0       ?IsConnected@NetSocket@LiveCreate@@QEAA_NXZ 00000000375141e0 f   LiveCreateNetSocket.obj
 0001:000131f0       ?IsShutdown@NetSocket@LiveCreate@@QEAA_NXZ 00000000375141f0 f   LiveCreateNetSocket.obj
 0001:00013200       ?Connect@NetSocket@LiveCreate@@QEAA_NPEBDG@Z 0000000037514200 f   LiveCreateNetSocket.obj
 0001:00013450       ?Validate@NetSocket@LiveCreate@@QEAA_NXZ 0000000037514450 f   LiveCreateNetSocket.obj
 0001:00013680       ?HasRecvData@NetSocket@LiveCreate@@QEAA_NXZ 0000000037514680 f   LiveCreateNetSocket.obj
 0001:00013770       ?SendData@NetSocket@LiveCreate@@QEAAHPEBEI@Z 0000000037514770 f   LiveCreateNetSocket.obj
 0001:00013890       ?ReceiveData@NetSocket@LiveCreate@@QEAAHPEAEI@Z 0000000037514890 f   LiveCreateNetSocket.obj
 0001:00013a10       ??_EINetSocketObserver@LiveCreate@@UEAAPEAXI@Z 0000000037514a10 f i LiveCreateNetwork.obj
 0001:00013a10       ??_GINetSocketObserver@LiveCreate@@UEAAPEAXI@Z 0000000037514a10 f i LiveCreateNetwork.obj
 0001:00013a40       ?NetGetTimeMsec@LiveCreate@@YAHXZ 0000000037514a40 f   LiveCreateNetwork.obj
 0001:00013a50       ?CreateAndConnectSocket@NetPeerCommThread@LiveCreate@@QEAA_NPEBDH_K@Z 0000000037514a50 f   LiveCreateNetwork.obj
 0001:00013b00       ?Start@NetPeer@LiveCreate@@QEAA_NII@Z 0000000037514b00 f   LiveCreateNetwork.obj
 0001:00013b40       ?OnPeerConnected@NetPeer@LiveCreate@@IEAAXPEAUNetPeerConnection@2@@Z 0000000037514b40 f   LiveCreateNetwork.obj
 0001:00013bb0       ?Stop@NetPeer@LiveCreate@@QEAAXXZ 0000000037514bb0 f   LiveCreateNetwork.obj
 0001:00013bc0       ?_M_compute_next_size@?$_Impl_vector@USNetEvent@LiveCreate@@V?$allocator@USNetEvent@LiveCreate@@@stlpmtx_std@@@priv@stlpmtx_std@@AEAA_K_K@Z 0000000037514bc0 f i LiveCreateNetwork.obj
 0001:00013c50       ?_M_set@?$_Impl_vector@USFileItem@FileSyncManager@LiveCreate@@V?$allocator@USFileItem@FileSyncManager@LiveCreate@@@stlpmtx_std@@@priv@stlpmtx_std@@AEAAXPEAUSFileItem@FileSyncManager@LiveCreate@@00@Z 0000000037514c50 f i LiveCreateFileSync.obj
 0001:00013c50       ?_M_set@?$_Impl_vector@USNetMessage@LiveCreate@@V?$allocator@USNetMessage@LiveCreate@@@stlpmtx_std@@@priv@stlpmtx_std@@AEAAXPEAUSNetMessage@LiveCreate@@00@Z 0000000037514c50 f i LiveCreateNetwork.obj
 0001:00013c50       ?_M_set@?$_Impl_vector@USChangedFileName@FileChangeNotifyController@LiveCreate@@V?$allocator@USChangedFileName@FileChangeNotifyController@LiveCreate@@@stlpmtx_std@@@priv@stlpmtx_std@@AEAAXPEAUSChangedFileName@FileChangeNotifyController@LiveCreate@@00@Z 0000000037514c50 f i LiveCreateCtrl_FileChangeNotify.obj
 0001:00013c50       ?_M_set@?$_Impl_vector@USConsoleString@ExecuteConsoleStringController@LiveCreate@@V?$allocator@USConsoleString@ExecuteConsoleStringController@LiveCreate@@@stlpmtx_std@@@priv@stlpmtx_std@@AEAAXPEAUSConsoleString@ExecuteConsoleStringController@LiveCreate@@00@Z 0000000037514c50 f i LiveCreateCtrl_ExecuteConsoleString.obj
 0001:00013c50       ?_M_set@?$_Impl_vector@PEAXV?$allocator@PEAX@stlpmtx_std@@@priv@stlpmtx_std@@AEAAXPEAPEAX00@Z 0000000037514c50 f i LiveCreate.obj
 0001:00013c50       ?_M_set@?$_Impl_vector@V?$CryStringT@D@@V?$allocator@V?$CryStringT@D@@@stlpmtx_std@@@priv@stlpmtx_std@@AEAAXPEAV?$CryStringT@D@@00@Z 0000000037514c50 f i LiveCreateCtrl_CVar.obj
 0001:00013c50       ?_M_set@?$_Impl_vector@UCVarData@CVarController@LiveCreate@@V?$allocator@UCVarData@CVarController@LiveCreate@@@stlpmtx_std@@@priv@stlpmtx_std@@AEAAXPEAUCVarData@CVarController@LiveCreate@@00@Z 0000000037514c50 f i LiveCreateCtrl_CVar.obj
 0001:00013c50       ?_M_set@?$_Impl_vector@USTransformData@EntitiesController@LiveCreate@@V?$allocator@USTransformData@EntitiesController@LiveCreate@@@stlpmtx_std@@@priv@stlpmtx_std@@AEAAXPEAUSTransformData@EntitiesController@LiveCreate@@00@Z 0000000037514c50 f i LiveCreateCtrl_Entities.obj
 0001:00013c50       ?_M_set@?$_Impl_vector@USNetEvent@LiveCreate@@V?$allocator@USNetEvent@LiveCreate@@@stlpmtx_std@@@priv@stlpmtx_std@@AEAAXPEAUSNetEvent@LiveCreate@@00@Z 0000000037514c50 f i LiveCreateNetwork.obj
 0001:00013c50       ?_M_set@?$_Impl_vector@IV?$allocator@I@stlpmtx_std@@@priv@stlpmtx_std@@AEAAXPEAI00@Z 0000000037514c50 f i LiveCreateCtrl_Entities.obj
 0001:00013ce0       ??4SNetEvent@LiveCreate@@QEAAAEAU01@AEBU01@@Z 0000000037514ce0 f i LiveCreateNetwork.obj
 0001:00013d50       ?IsConnectedTo@NetPeer@LiveCreate@@QEAA_NPEBD@Z 0000000037514d50 f   LiveCreateNetwork.obj
 0001:00013df0       ?GetPeerInfo@NetPeer@LiveCreate@@QEAA_NPEAXAEAUSPeerInfo@2@@Z 0000000037514df0 f   LiveCreateNetwork.obj
 0001:00013ea0       ?DisconnectFromPeer@NetPeer@LiveCreate@@QEAA_NPEAX@Z 0000000037514ea0 f   LiveCreateNetwork.obj
 0001:00014050       ?DisconnectFromAllPeers@NetPeer@LiveCreate@@QEAAXXZ 0000000037515050 f   LiveCreateNetwork.obj
 0001:00014230       ?IsConnectedToAnyPeer@NetPeer@LiveCreate@@QEAA_NXZ 0000000037515230 f   LiveCreateNetwork.obj
 0001:000142a0       ??1?$CrySimpleThread@VNetPeerCommThread@LiveCreate@@@@UEAA@XZ 00000000375152a0 f i LiveCreateNetwork.obj
 0001:000142a0       ??1?$CrySimpleThread@VFileSyncManager@LiveCreate@@@@UEAA@XZ 00000000375152a0 f i LiveCreateFileSync.obj
 0001:000142a0       ??1?$CrySimpleThread@VNetPeerServerAcceptThread@LiveCreate@@@@UEAA@XZ 00000000375152a0 f i LiveCreateNetwork.obj
 0001:00014370       ??_E?$CrySimpleThread@VNetPeerServerAcceptThread@LiveCreate@@@@W7EAAPEAXI@Z 0000000037515370 f i LiveCreateNetwork.obj
 0001:00014370       ??_E?$CrySimpleThread@VFileSyncManager@LiveCreate@@@@W7EAAPEAXI@Z 0000000037515370 f i LiveCreateFileSync.obj
 0001:00014370       ??_E?$CrySimpleThread@VNetPeerCommThread@LiveCreate@@@@W7EAAPEAXI@Z 0000000037515370 f i LiveCreateNetwork.obj
 0001:00014380       ?Start@?$CrySimpleThread@VFileSyncManager@LiveCreate@@@@UEAAXAEAVFileSyncManager@LiveCreate@@IPEBDH@Z 0000000037515380 f i LiveCreateFileSync.obj
 0001:00014380       ?Start@?$CrySimpleThread@VNetPeerServerAcceptThread@LiveCreate@@@@UEAAXAEAVNetPeerServerAcceptThread@LiveCreate@@IPEBDH@Z 0000000037515380 f i LiveCreateNetwork.obj
 0001:00014380       ?Start@?$CrySimpleThread@VNetPeerCommThread@LiveCreate@@@@UEAAXAEAVNetPeerCommThread@LiveCreate@@IPEBDH@Z 0000000037515380 f i LiveCreateNetwork.obj
 0001:000143a0       ?RunRunnable@?$CrySimpleThread@VFileSyncManager@LiveCreate@@@@CAIPEAX@Z 00000000375153a0 f i LiveCreateFileSync.obj
 0001:000143a0       ?RunRunnable@?$CrySimpleThread@VNetPeerCommThread@LiveCreate@@@@CAIPEAX@Z 00000000375153a0 f i LiveCreateNetwork.obj
 0001:000143a0       ?RunRunnable@?$CrySimpleThread@VNetPeerServerAcceptThread@LiveCreate@@@@CAIPEAX@Z 00000000375153a0 f i LiveCreateNetwork.obj
 0001:000143e0       ?Start@?$CrySimpleThread@VFileSyncManager@LiveCreate@@@@UEAAXIPEBDHH@Z 00000000375153e0 f i LiveCreateFileSync.obj
 0001:000143e0       ?Start@?$CrySimpleThread@VNetPeerServerAcceptThread@LiveCreate@@@@UEAAXIPEBDHH@Z 00000000375153e0 f i LiveCreateNetwork.obj
 0001:000143e0       ?Start@?$CrySimpleThread@VNetPeerCommThread@LiveCreate@@@@UEAAXIPEBDHH@Z 00000000375153e0 f i LiveCreateNetwork.obj
 0001:00014400       ??_E?$CrySimpleThread@VNetPeerServerAcceptThread@LiveCreate@@@@UEAAPEAXI@Z 0000000037515400 f i LiveCreateNetwork.obj
 0001:00014400       ??_G?$CrySimpleThread@VNetPeerCommThread@LiveCreate@@@@UEAAPEAXI@Z 0000000037515400 f i LiveCreateNetwork.obj
 0001:00014400       ??_G?$CrySimpleThread@VNetPeerServerAcceptThread@LiveCreate@@@@UEAAPEAXI@Z 0000000037515400 f i LiveCreateNetwork.obj
 0001:00014400       ??_G?$CrySimpleThread@VFileSyncManager@LiveCreate@@@@UEAAPEAXI@Z 0000000037515400 f i LiveCreateFileSync.obj
 0001:00014400       ??_E?$CrySimpleThread@VFileSyncManager@LiveCreate@@@@UEAAPEAXI@Z 0000000037515400 f i LiveCreateFileSync.obj
 0001:00014400       ??_E?$CrySimpleThread@VNetPeerCommThread@LiveCreate@@@@UEAAPEAXI@Z 0000000037515400 f i LiveCreateNetwork.obj
 0001:00014430       ?_M_insert_overflow@?$_Impl_vector@USNetMessage@LiveCreate@@V?$allocator@USNetMessage@LiveCreate@@@stlpmtx_std@@@priv@stlpmtx_std@@AEAAXPEAUSNetMessage@LiveCreate@@AEBU45@AEBU__true_type@3@_K_N@Z 0000000037515430 f i LiveCreateNetwork.obj
 0001:000145c0       ??0?$CryThread@VNetPeerCommThread@LiveCreate@@@@QEAA@XZ 00000000375155c0 f i LiveCreateNetwork.obj
 0001:000145c0       ??0?$CryThread@VNetPeerServerAcceptThread@LiveCreate@@@@QEAA@XZ 00000000375155c0 f i LiveCreateNetwork.obj
 0001:000145c0       ??0?$CryThread@VFileSyncManager@LiveCreate@@@@QEAA@XZ 00000000375155c0 f i LiveCreateFileSync.obj
 0001:00014650       ??_E?$CryThread@VFileSyncManager@LiveCreate@@@@W7EAAPEAXI@Z 0000000037515650 f i LiveCreateFileSync.obj
 0001:00014650       ??_E?$CryThread@VNetPeerCommThread@LiveCreate@@@@W7EAAPEAXI@Z 0000000037515650 f i LiveCreateNetwork.obj
 0001:00014650       ??_E?$CryThread@VNetPeerServerAcceptThread@LiveCreate@@@@W7EAAPEAXI@Z 0000000037515650 f i LiveCreateNetwork.obj
 0001:00014660       ??_E?$CryThread@VFileSyncManager@LiveCreate@@@@UEAAPEAXI@Z 0000000037515660 f i LiveCreateFileSync.obj
 0001:00014660       ??_E?$CryThread@VNetPeerServerAcceptThread@LiveCreate@@@@UEAAPEAXI@Z 0000000037515660 f i LiveCreateNetwork.obj
 0001:00014660       ??_G?$CryThread@VFileSyncManager@LiveCreate@@@@UEAAPEAXI@Z 0000000037515660 f i LiveCreateFileSync.obj
 0001:00014660       ??_E?$CryThread@VNetPeerCommThread@LiveCreate@@@@UEAAPEAXI@Z 0000000037515660 f i LiveCreateNetwork.obj
 0001:00014660       ??_G?$CryThread@VNetPeerCommThread@LiveCreate@@@@UEAAPEAXI@Z 0000000037515660 f i LiveCreateNetwork.obj
 0001:00014660       ??_G?$CryThread@VNetPeerServerAcceptThread@LiveCreate@@@@UEAAPEAXI@Z 0000000037515660 f i LiveCreateNetwork.obj
 0001:000146b0       ?push_back@?$_Impl_vector@USNetMessage@LiveCreate@@V?$allocator@USNetMessage@LiveCreate@@@stlpmtx_std@@@priv@stlpmtx_std@@QEAAXAEBUSNetMessage@LiveCreate@@@Z 00000000375156b0 f i LiveCreateNetwork.obj
 0001:00014730       ??$__copy_ptrs@PEAUSNetEvent@LiveCreate@@PEAU12@@priv@stlpmtx_std@@YAPEAUSNetEvent@LiveCreate@@PEAU23@00AEBU__false_type@1@@Z 0000000037515730 f i LiveCreateNetwork.obj
 0001:00014800       ?DeleteDisconnectedPeers@NetPeer@LiveCreate@@QEAAXXZ 0000000037515800 f   LiveCreateNetwork.obj
 0001:000149b0       ?AddSendMessage@NetPeerCommThread@LiveCreate@@QEAAXAEBUSNetMessage@2@@Z 00000000375159b0 f   LiveCreateNetwork.obj
 0001:00014a00       ?SendMessageA@NetPeer@LiveCreate@@QEAA_NPEAXAEBUSNetMessage@2@@Z 0000000037515a00 f   LiveCreateNetwork.obj
 0001:00014a70       ?SendConnectMessage@NetPeer@LiveCreate@@IEAAXPEAUNetPeerConnection@2@@Z 0000000037515a70 f   LiveCreateNetwork.obj
 0001:00014c70       ?SendInfoMessage@NetPeer@LiveCreate@@IEAAXPEAUNetPeerConnection@2@@Z 0000000037515c70 f   LiveCreateNetwork.obj
 0001:000153e0       ?_M_clear_after_move@?$_Impl_vector@USNetEvent@LiveCreate@@V?$allocator@USNetEvent@LiveCreate@@@stlpmtx_std@@@priv@stlpmtx_std@@AEAAXXZ 00000000375163e0 f i LiveCreateNetwork.obj
 0001:00015460       ??$__uninitialized_fill_n@PEAUSNetEvent@LiveCreate@@_KU12@@priv@stlpmtx_std@@YAPEAUSNetEvent@LiveCreate@@PEAU23@_KAEBU23@@Z 0000000037516460 f i LiveCreateNetwork.obj
 0001:00015510       ??$__ucopy_ptrs@PEAUSNetEvent@LiveCreate@@PEAU12@@priv@stlpmtx_std@@YAPEAUSNetEvent@LiveCreate@@PEAU23@00AEBU__false_type@1@@Z 0000000037516510 f i LiveCreateNetwork.obj
 0001:000155d0       ??1?$_Impl_vector@USNetEvent@LiveCreate@@V?$allocator@USNetEvent@LiveCreate@@@stlpmtx_std@@@priv@stlpmtx_std@@QEAA@XZ 00000000375165d0 f i LiveCreateNetwork.obj
 0001:00015660       ?erase@?$_Impl_vector@USNetEvent@LiveCreate@@V?$allocator@USNetEvent@LiveCreate@@@stlpmtx_std@@@priv@stlpmtx_std@@QEAAPEAUSNetEvent@LiveCreate@@PEAU45@@Z 0000000037516660 f i LiveCreateNetwork.obj
 0001:000156f0       ?_M_insert_overflow_aux@?$_Impl_vector@USNetEvent@LiveCreate@@V?$allocator@USNetEvent@LiveCreate@@@stlpmtx_std@@@priv@stlpmtx_std@@AEAAXPEAUSNetEvent@LiveCreate@@AEBU45@AEBU__false_type@3@_K_N@Z 00000000375166f0 f i LiveCreateNetwork.obj
 0001:00015860       ?PopEvent@NetEventQueue@LiveCreate@@QEAA_NAEAUSNetEvent@2@@Z 0000000037516860 f   LiveCreateNetwork.obj
 0001:000158d0       ??1NetPeerServerAcceptThread@LiveCreate@@UEAA@XZ 00000000375168d0 f i LiveCreateNetwork.obj
 0001:00015950       ??0NetPeerCommThread@LiveCreate@@QEAA@XZ 0000000037516950 f   LiveCreateNetwork.obj
 0001:00015a70       ??_ENetPeerCommThread@LiveCreate@@WJI@EAAPEAXI@Z 0000000037516a70 f i LiveCreateNetwork.obj
 0001:00015a80       ??_ENetPeerCommThread@LiveCreate@@W7EAAPEAXI@Z 0000000037516a80 f i LiveCreateNetwork.obj
 0001:00015a90       ??1NetPeerCommThread@LiveCreate@@UEAA@XZ 0000000037516a90 f i LiveCreateNetwork.obj
 0001:00015b50       ??1NetPeer@LiveCreate@@UEAA@XZ 0000000037516b50 f   LiveCreateNetwork.obj
 0001:00015bc0       ?ConnectToPeer@NetPeer@LiveCreate@@QEAAPEAXPEBDH_K@Z 0000000037516bc0 f   LiveCreateNetwork.obj
 0001:00015eb0       ?OnPeerConnectionAccepted@NetPeer@LiveCreate@@IEAAXPEBDH_K@Z 0000000037516eb0 f   LiveCreateNetwork.obj
 0001:00015fa0       ??0NetPeerServerAcceptThread@LiveCreate@@QEAA@XZ 0000000037516fa0 f   LiveCreateNetwork.obj
 0001:00016080       ??_ENetPeerServerAcceptThread@LiveCreate@@W7EAAPEAXI@Z 0000000037517080 f i LiveCreateNetwork.obj
 0001:00016090       ??_ENetPeerServerAcceptThread@LiveCreate@@UEAAPEAXI@Z 0000000037517090 f i LiveCreateNetwork.obj
 0001:00016090       ??_GNetPeerServerAcceptThread@LiveCreate@@UEAAPEAXI@Z 0000000037517090 f i LiveCreateNetwork.obj
 0001:000160c0       ??_GNetPeerCommThread@LiveCreate@@UEAAPEAXI@Z 00000000375170c0 f i LiveCreateNetwork.obj
 0001:000160c0       ??_ENetPeerCommThread@LiveCreate@@UEAAPEAXI@Z 00000000375170c0 f i LiveCreateNetwork.obj
 0001:000160f0       ??0NetPeer@LiveCreate@@QEAA@XZ 00000000375170f0 f   LiveCreateNetwork.obj
 0001:00016190       ??_ENetPeer@LiveCreate@@UEAAPEAXI@Z 0000000037517190 f i LiveCreateNetwork.obj
 0001:00016190       ??_GNetPeer@LiveCreate@@UEAAPEAXI@Z 0000000037517190 f i LiveCreateNetwork.obj
 0001:000161c0       ?push_back@?$_Impl_vector@USNetEvent@LiveCreate@@V?$allocator@USNetEvent@LiveCreate@@@stlpmtx_std@@@priv@stlpmtx_std@@QEAAXAEBUSNetEvent@LiveCreate@@@Z 00000000375171c0 f i LiveCreateNetwork.obj
 0001:00016280       ?Run@NetPeerServerAcceptThread@LiveCreate@@UEAAXXZ 0000000037517280 f   LiveCreateNetwork.obj
 0001:00016650       ?OnSocketConnected@NetPeerCommThread@LiveCreate@@UEAAXPEAUNetSocket@2@@Z 0000000037517650 f   LiveCreateNetwork.obj
 0001:00016780       ?Run@NetPeerCommThread@LiveCreate@@UEAAXXZ 0000000037517780 f   LiveCreateNetwork.obj
 0001:00017270       ?Update@NetPeer@LiveCreate@@QEAAXXZ 0000000037518270 f   LiveCreateNetwork.obj
 0001:00018130       ?SetProfile@PlatformHandlerBase@LiveCreate@@UEAAXPEAUSProfile@2@@Z 0000000037519130 f   PlatformHandlerBase.obj
 0001:00018140       ?GetProfile@PlatformHandlerBase@LiveCreate@@UEBAPEAUSProfile@2@XZ 0000000037519140 f   PlatformHandlerBase.obj
 0001:00018150       ?SetEnabled@PlatformHandlerBase@LiveCreate@@UEAAX_N@Z 0000000037519150 f   PlatformHandlerBase.obj
 0001:00018160       ?IsEnabled@PlatformHandlerBase@LiveCreate@@UEAA_NXZ 0000000037519160 f   PlatformHandlerBase.obj
 0001:00018170       ?IsFileSyncEnabled@PlatformHandlerBase@LiveCreate@@UEAA_NXZ 0000000037519170 f   PlatformHandlerBase.obj
 0001:00018180       ?SetFlags@PlatformHandlerBase@LiveCreate@@UEAAXI@Z 0000000037519180 f   PlatformHandlerBase.obj
 0001:00018190       ?SetFlag@PlatformHandlerBase@LiveCreate@@UEAAXI@Z 0000000037519190 f   PlatformHandlerBase.obj
 0001:000181a0       ?IsFlagSet@PlatformHandlerBase@LiveCreate@@UEAA_NI@Z 00000000375191a0 f   PlatformHandlerBase.obj
 0001:000181b0       ?UnsetFlag@PlatformHandlerBase@LiveCreate@@UEAAXI@Z 00000000375191b0 f   PlatformHandlerBase.obj
 0001:000181c0       ?GetFlags@PlatformHandlerBase@LiveCreate@@UEAAIXZ 00000000375191c0 f   PlatformHandlerBase.obj
 0001:000181d0       ?GetInfo@PlatformHandlerBase@LiveCreate@@UEAAAEBUSPeerInfo@2@XZ 00000000375191d0 f   PlatformHandlerBase.obj
 0001:000181e0       ?GrabScreenshot@PlatformHandlerBase@LiveCreate@@UEAA_NXZ 00000000375191e0 f   PlatformHandlerBase.obj
 0001:00018240       ??_EIPlatformHandler@LiveCreate@@UEAAPEAXI@Z 0000000037519240 f i PlatformHandlerBase.obj
 0001:00018240       ??_GIPlatformHandler@LiveCreate@@UEAAPEAXI@Z 0000000037519240 f i PlatformHandlerBase.obj
 0001:00018270       ?SetInfo@PlatformHandlerBase@LiveCreate@@UEAAXAEBUSPeerInfo@2@@Z 0000000037519270 f   PlatformHandlerBase.obj
 0001:000182d0       ?GetGameBuildInfoCount@PlatformHandlerBase@LiveCreate@@UEAAHXZ 00000000375192d0 f   PlatformHandlerBase.obj
 0001:000182f0       ?GetGameBuildInfoAt@PlatformHandlerBase@LiveCreate@@UEAAPEAUSGameBuildInfo@2@H@Z 00000000375192f0 f   PlatformHandlerBase.obj
 0001:00018300       ??0PlatformHandlerBase@LiveCreate@@QEAA@PEBUIManager@1@@Z 0000000037519300 f   PlatformHandlerBase.obj
 0001:000183a0       ?ParseBuildInfo@PlatformHandlerBase@LiveCreate@@QEAA_NPEBDAEAUSGameBuildInfo@2@@Z 00000000375193a0 f   PlatformHandlerBase.obj
 0001:00018a50       ?DeleteGameBuilds@PlatformHandlerBase@LiveCreate@@QEAAXXZ 0000000037519a50 f   PlatformHandlerBase.obj
 0001:00018b80       ??1PlatformHandlerBase@LiveCreate@@UEAA@XZ 0000000037519b80 f   PlatformHandlerBase.obj
 0001:00018be0       ??_EPlatformHandlerBase@LiveCreate@@UEAAPEAXI@Z 0000000037519be0 f i PlatformHandlerBase.obj
 0001:00018be0       ??_GPlatformHandlerBase@LiveCreate@@UEAAPEAXI@Z 0000000037519be0 f i PlatformHandlerBase.obj
 0001:00018c60       ?GetPlatformName@PlatformHandlerFactory_EditorPC@LiveCreate@@UEAAPEBDXZ 0000000037519c60 f   PlatformHandler_EditorPC.obj
 0001:00018c70       ?CreatePlatformHandlerInstance@PlatformHandlerFactory_EditorPC@LiveCreate@@UEAAPEAUIPlatformHandler@2@PEBUIManager@2@QEBUSPeerInfo@2@@Z 0000000037519c70 f   PlatformHandler_EditorPC.obj
 0001:00018ce0       ?GetPlatformName@PlatformHandlerFactory_GamePC@LiveCreate@@UEAAPEBDXZ 0000000037519ce0 f   PlatformHandler_GamePC.obj
 0001:00018cf0       ?CreatePlatformHandlerInstance@PlatformHandlerFactory_GamePC@LiveCreate@@UEAAPEAUIPlatformHandler@2@PEBUIManager@2@QEBUSPeerInfo@2@@Z 0000000037519cf0 f   PlatformHandler_GamePC.obj
 0001:00018d60       ??_GPlatformHandler_EditorPC@LiveCreate@@UEAAPEAXI@Z 0000000037519d60 f i PlatformHandler_EditorPC.obj
 0001:00018d60       ??_EPlatformHandler_GamePC@LiveCreate@@UEAAPEAXI@Z 0000000037519d60 f i PlatformHandler_GamePC.obj
 0001:00018d60       ??_GPlatformHandler_GamePC@LiveCreate@@UEAAPEAXI@Z 0000000037519d60 f i PlatformHandler_GamePC.obj
 0001:00018d60       ??_EPlatformHandler_EditorPC@LiveCreate@@UEAAPEAXI@Z 0000000037519d60 f i PlatformHandler_EditorPC.obj
 0001:00018da0       ?GetPlatformName@PlatformHandlerFactory_PS3@LiveCreate@@UEAAPEBDXZ 0000000037519da0 f   PlatformHandler_PS3.obj
 0001:00018db0       ?FindTargetInfoByName@PlatformHandlerFactory_PS3@LiveCreate@@QEAAPEAUPS3TargetInfo@@PEBD@Z 0000000037519db0 f   PlatformHandler_PS3.obj
 0001:00018e40       ?ConnectToTargetByName@PlatformHandlerFactory_PS3@LiveCreate@@QEAA_NPEBD@Z 0000000037519e40 f   PlatformHandler_PS3.obj
 0001:00018ee0       ?FindMachineAddressByName@PlatformHandlerFactory_PS3@LiveCreate@@UEAA_NPEBDPEADI@Z 0000000037519ee0 f   PlatformHandler_PS3.obj
 0001:00018f50       ?Launch@PlatformHandler_PS3@LiveCreate@@UEAA_NPEBD00@Z 0000000037519f50 f   PlatformHandler_PS3.obj
 0001:00018f90       ?Reset@PlatformHandler_PS3@LiveCreate@@UEAA_NW4EResetMode@SProfile@2@@Z 0000000037519f90 f   PlatformHandler_PS3.obj
 0001:00018fc0       ?CopyFileFrom@PlatformHandler_PS3@LiveCreate@@UEAA_NPEBD0@Z 0000000037519fc0 f   PlatformHandler_PS3.obj
 0001:00018ff0       ?EraseFile@PlatformHandler_PS3@LiveCreate@@UEAA_NPEBD@Z 0000000037519ff0 f   PlatformHandler_PS3.obj
 0001:00018ff0       ?EraseFolder@PlatformHandler_PS3@LiveCreate@@UEAA_NPEBD@Z 0000000037519ff0 f   PlatformHandler_PS3.obj
 0001:00019020       ?IsOn@PlatformHandler_PS3@LiveCreate@@UEAA_NXZ 000000003751a020 f   PlatformHandler_PS3.obj
 0001:00019040       ?ExtractTimeUTC64@LiveCreate@@YAX_KAEAUSDateTime@1@@Z 000000003751a040 f   PlatformHandler_PS3.obj
 0001:00019140       ?NextScanFolderEntry@PlatformHandler_PS3@LiveCreate@@UEAA_NPEAXPEAUSScanFolderEntry@2@@Z 000000003751a140 f   PlatformHandler_PS3.obj
 0001:00019230       ?SearchForGameBuilds@PlatformHandler_PS3@LiveCreate@@UEAA_NXZ 000000003751a230 f   PlatformHandler_PS3.obj
 0001:00019240       ?GrabScreenshot@PlatformHandler_PS3@LiveCreate@@UEAA_NXZ 000000003751a240 f   PlatformHandler_PS3.obj
 0001:00019250       ??0PlatformHandlerFactory_PS3@LiveCreate@@QEAA@XZ 000000003751a250 f   PlatformHandler_PS3.obj
 0001:000192c0       ?CreatePlatformHandlerInstance@PlatformHandlerFactory_PS3@LiveCreate@@UEAAPEAUIPlatformHandler@2@PEBUIManager@2@QEBUSPeerInfo@2@@Z 000000003751a2c0 f   PlatformHandler_PS3.obj
 0001:000193a0       ?GatherPlatforms@PlatformHandlerFactory_PS3@LiveCreate@@UEAAIPEAUSPeerInfo@2@I@Z 000000003751a3a0 f   PlatformHandler_PS3.obj
 0001:000194d0       ??_GPlatformHandler_PS3@LiveCreate@@UEAAPEAXI@Z 000000003751a4d0 f i PlatformHandler_PS3.obj
 0001:000194d0       ??_EPlatformHandler_PS3@LiveCreate@@UEAAPEAXI@Z 000000003751a4d0 f i PlatformHandler_PS3.obj
 0001:00019510       ??_GPlatformHandlerFactory_PS3@LiveCreate@@UEAAPEAXI@Z 000000003751a510 f i PlatformHandler_PS3.obj
 0001:00019510       ??_EPlatformHandlerFactory_PS3@LiveCreate@@UEAAPEAXI@Z 000000003751a510 f i PlatformHandler_PS3.obj
 0001:00019580       ?EndScanFolder@PlatformHandler_PS3@LiveCreate@@UEAAXPEAX@Z 000000003751a580 f   PlatformHandler_PS3.obj
 0001:000195e0       ?BeginScanFolder@PlatformHandler_PS3@LiveCreate@@UEAAPEAXPEBD@Z 000000003751a5e0 f   PlatformHandler_PS3.obj
 0001:00019760       ?CopyFileTo@PlatformHandler_PS3@LiveCreate@@UEAA_NPEBD0@Z 000000003751a760 f   PlatformHandler_PS3.obj
 0001:00019d10       ?GetPlatformName@PlatformHandlerFactory_X360@LiveCreate@@UEAAPEBDXZ 000000003751ad10 f   PlatformHandler_X360.obj
 0001:00019d20       ?GatherPlatforms@PlatformHandlerFactory_X360@LiveCreate@@UEAAIPEAUSPeerInfo@2@I@Z 000000003751ad20 f   PlatformHandler_X360.obj
 0001:00019e10       ?FindMachineAddressByName@PlatformHandlerFactory_X360@LiveCreate@@UEAA_NPEBDPEADI@Z 000000003751ae10 f   PlatformHandler_X360.obj
 0001:00019ee0       ?CopyFileTimeToDateTime@LiveCreate@@YAXAEAU_FILETIME@@AEAUSDateTime@1@@Z 000000003751aee0 f   PlatformHandler_X360.obj
 0001:00019f50       ?SetAsDefaultConsole@PlatformHandler_X360@LiveCreate@@IEAA_NXZ 000000003751af50 f   PlatformHandler_X360.obj
 0001:00019fe0       ?Launch@PlatformHandler_X360@LiveCreate@@UEAA_NPEBD00@Z 000000003751afe0 f   PlatformHandler_X360.obj
 0001:0001a080       ?Reset@PlatformHandler_X360@LiveCreate@@UEAA_NW4EResetMode@SProfile@2@@Z 000000003751b080 f   PlatformHandler_X360.obj
 0001:0001a0e0       ?GrabScreenshot@PlatformHandler_X360@LiveCreate@@UEAA_NXZ 000000003751b0e0 f   PlatformHandler_X360.obj
 0001:0001a110       ?EraseFile@PlatformHandler_X360@LiveCreate@@UEAA_NPEBD@Z 000000003751b110 f   PlatformHandler_X360.obj
 0001:0001a150       ?EraseFolder@PlatformHandler_X360@LiveCreate@@UEAA_NPEBD@Z 000000003751b150 f   PlatformHandler_X360.obj
 0001:0001a190       ?GetFileModificationTime@PlatformHandler_X360@LiveCreate@@UEAA_KPEBD@Z 000000003751b190 f   PlatformHandler_X360.obj
 0001:0001a1f0       ?IsOn@PlatformHandler_X360@LiveCreate@@UEAA_NXZ 000000003751b1f0 f   PlatformHandler_X360.obj
 0001:0001a220       ?NextScanFolderEntry@PlatformHandler_X360@LiveCreate@@UEAA_NPEAXPEAUSScanFolderEntry@2@@Z 000000003751b220 f   PlatformHandler_X360.obj
 0001:0001a320       ?replace@?$CryStringT@D@@QEAAAEAV1@PEBD0@Z 000000003751b320 f i PlatformHandler_X360.obj
 0001:0001a550       ?erase@?$vector@PEAUSX360WalkDir@PlatformHandler_X360@LiveCreate@@V?$allocator@PEAUSX360WalkDir@PlatformHandler_X360@LiveCreate@@@stlpmtx_std@@@stlpmtx_std@@QEAAPEAPEAUSX360WalkDir@PlatformHandler_X360@LiveCreate@@PEAPEAU345@@Z 000000003751b550 f i PlatformHandler_X360.obj
 0001:0001a5b0       ?ToDosPath@PathUtil@@YA?AV?$CryStringT@D@@AEBV2@@Z 000000003751b5b0 f i PlatformHandler_X360.obj
 0001:0001a6e0       ??_EPlatformHandler_X360@LiveCreate@@UEAAPEAXI@Z 000000003751b6e0 f i PlatformHandler_X360.obj
 0001:0001a6e0       ??_GPlatformHandler_X360@LiveCreate@@UEAAPEAXI@Z 000000003751b6e0 f i PlatformHandler_X360.obj
 0001:0001a760       ?EndScanFolder@PlatformHandler_X360@LiveCreate@@UEAAXPEAX@Z 000000003751b760 f   PlatformHandler_X360.obj
 0001:0001a820       ?CopyFileTo@PlatformHandler_X360@LiveCreate@@UEAA_NPEBD0@Z 000000003751b820 f   PlatformHandler_X360.obj
 0001:0001ac90       ?CopyFileFrom@PlatformHandler_X360@LiveCreate@@UEAA_NPEBD0@Z 000000003751bc90 f   PlatformHandler_X360.obj
 0001:0001b210       ?BeginScanFolder@PlatformHandler_X360@LiveCreate@@UEAAPEAXPEBD@Z 000000003751c210 f   PlatformHandler_X360.obj
 0001:0001b440       ?SearchForGameBuildsRecursive@PlatformHandler_X360@LiveCreate@@IEAA_NPEBD@Z 000000003751c440 f   PlatformHandler_X360.obj
 0001:0001c460       ?SearchForGameBuilds@PlatformHandler_X360@LiveCreate@@UEAA_NXZ 000000003751d460 f   PlatformHandler_X360.obj
 0001:0001c4a0       ??0PlatformHandler_X360@LiveCreate@@QEAA@PEBUIManager@1@@Z 000000003751d4a0 f   PlatformHandler_X360.obj
 0001:0001c960       ??0PlatformHandlerFactory_X360@LiveCreate@@QEAA@XZ 000000003751d960 f   PlatformHandler_X360.obj
 0001:0001c990       ?CreatePlatformHandlerInstance@PlatformHandlerFactory_X360@LiveCreate@@UEAAPEAUIPlatformHandler@2@PEBUIManager@2@QEBUSPeerInfo@2@@Z 000000003751d990 f   PlatformHandler_X360.obj
 0001:0001c9f0       ?DeInitialize@?$Node_Alloc_Lock@$00$00@@SAXXZ 000000003751d9f0 f i StdAfx.obj
 0001:0001ca58       __WSAFDIsSet               000000003751da58 f   Ws2_32:WS2_32.dll
 0001:0001ca5e       __imp_load_DmGetAltAddress 000000003751da5e     xbdm:xbdm.DLL
 0001:0001ca6a       __tailMerge_xbdm_DLL       000000003751da6a     xbdm:xbdm.DLL
 0001:0001cae3       DmGetAltAddress            000000003751dae3 f   xbdm:xbdm.DLL
 0001:0001cae9       __imp_load_DmGetXboxName   000000003751dae9     xbdm:xbdm.DLL
 0001:0001caf5       DmGetXboxName              000000003751daf5 f   xbdm:xbdm.DLL
 0001:0001cafb       __imp_load_DmSetXboxNameNoRegister 000000003751dafb     xbdm:xbdm.DLL
 0001:0001cb07       DmSetXboxNameNoRegister    000000003751db07 f   xbdm:xbdm.DLL
 0001:0001cb0d       __imp_load_DmReboot        000000003751db0d     xbdm:xbdm.DLL
 0001:0001cb19       DmReboot                   000000003751db19 f   xbdm:xbdm.DLL
 0001:0001cb1f       __imp_load_DmSetTitleEx    000000003751db1f     xbdm:xbdm.DLL
 0001:0001cb2b       DmSetTitleEx               000000003751db2b f   xbdm:xbdm.DLL
 0001:0001cb31       __imp_load_DmDeleteFile    000000003751db31     xbdm:xbdm.DLL
 0001:0001cb3d       DmDeleteFile               000000003751db3d f   xbdm:xbdm.DLL
 0001:0001cb43       __imp_load_DmGetFileAttributes 000000003751db43     xbdm:xbdm.DLL
 0001:0001cb4f       DmGetFileAttributes        000000003751db4f f   xbdm:xbdm.DLL
 0001:0001cb55       __imp_load_DmGetSystemTime 000000003751db55     xbdm:xbdm.DLL
 0001:0001cb61       DmGetSystemTime            000000003751db61 f   xbdm:xbdm.DLL
 0001:0001cb67       __imp_load_DmWalkDir       000000003751db67     xbdm:xbdm.DLL
 0001:0001cb73       DmWalkDir                  000000003751db73 f   xbdm:xbdm.DLL
 0001:0001cb79       __imp_load_DmCloseDir      000000003751db79     xbdm:xbdm.DLL
 0001:0001cb85       DmCloseDir                 000000003751db85 f   xbdm:xbdm.DLL
 0001:0001cb8b       __imp_load_DmSendFileA     000000003751db8b     xbdm:xbdm.DLL
 0001:0001cb97       DmSendFileA                000000003751db97 f   xbdm:xbdm.DLL
 0001:0001cb9d       __imp_load_DmMkdir         000000003751db9d     xbdm:xbdm.DLL
 0001:0001cba9       DmMkdir                    000000003751dba9 f   xbdm:xbdm.DLL
 0001:0001cbaf       __imp_load_DmReceiveFileA  000000003751dbaf     xbdm:xbdm.DLL
 0001:0001cbbb       DmReceiveFileA             000000003751dbbb f   xbdm:xbdm.DLL
 0001:0001cbc1       __imp_load_DmReadFilePartial 000000003751dbc1     xbdm:xbdm.DLL
 0001:0001cbcd       DmReadFilePartial          000000003751dbcd f   xbdm:xbdm.DLL
 0001:0001cbd4       _purecall                  000000003751dbd4 f   MSVCRT:MSVCR100.dll
 0001:0001cbda       memcpy                     000000003751dbda f   MSVCRT:MSVCR100.dll
 0001:0001cbe0       memset                     000000003751dbe0 f   MSVCRT:MSVCR100.dll
 0001:0001cc00       __chkstk                   000000003751dc00 f   MSVCRT:chkstk.obj
 0001:0001cc00       _alloca_probe              000000003751dc00     MSVCRT:chkstk.obj
 0001:0001cc50       _onexit                    000000003751dc50 f   MSVCRT:atonexit.obj
 0001:0001cd00       atexit                     000000003751dd00 f   MSVCRT:atonexit.obj
 0001:0001cd18       ?what@exception@std@@UEBAPEBDXZ 000000003751dd18 f   MSVCRT:MSVCR100.dll
 0001:0001cd80       _CRT_INIT                  000000003751dd80 f   MSVCRT:crtdll.obj
 0001:0001d118       _DllMainCRTStartup         000000003751e118 f   MSVCRT:crtdll.obj
 0001:0001d170       __security_check_cookie    000000003751e170 f   MSVCRT:amdsecgs.obj
 0001:0001d190       __C_specific_handler       000000003751e190 f   MSVCRT:MSVCR100.dll
 0001:0001d196       _unlock                    000000003751e196 f   MSVCRT:MSVCR100.dll
 0001:0001d19c       __dllonexit                000000003751e19c f   MSVCRT:MSVCR100.dll
 0001:0001d1a2       _lock                      000000003751e1a2 f   MSVCRT:MSVCR100.dll
 0001:0001d1a8       __clean_type_info_names    000000003751e1a8 f   MSVCRT:tncleanup.obj
 0001:0001d1b4       _RTC_Initialize            000000003751e1b4 f   MSVCRT:_initsect_.obj
 0001:0001d1ec       _RTC_Terminate             000000003751e1ec f   MSVCRT:_initsect_.obj
 0001:0001d230       _ValidateImageBase         000000003751e230 f   MSVCRT:pesect.obj
 0001:0001d260       _FindPESection             000000003751e260 f   MSVCRT:pesect.obj
 0001:0001d2b0       _IsNonwritableInCurrentImage 000000003751e2b0 f   MSVCRT:pesect.obj
 0001:0001d2f2       _initterm                  000000003751e2f2 f   MSVCRT:MSVCR100.dll
 0001:0001d2f8       _initterm_e                000000003751e2f8 f   MSVCRT:MSVCR100.dll
 0001:0001d2fe       _amsg_exit                 000000003751e2fe f   MSVCRT:MSVCR100.dll
 0001:0001d304       __CppXcptFilter            000000003751e304 f   MSVCRT:MSVCR100.dll
 0001:0001d30c       __security_init_cookie     000000003751e30c f   MSVCRT:gs_support.obj
 0001:0001d3c0       __report_gsfailure         000000003751e3c0 f   MSVCRT:gs_report.obj
 0001:0001d50a       __clean_type_info_names_internal 000000003751e50a f   MSVCRT:MSVCR100.dll
 0001:0001d510       __crt_debugger_hook        000000003751e510 f   MSVCRT:MSVCR100.dll
 0001:0001d516       RtlVirtualUnwind           000000003751e516 f   kernel32:KERNEL32.dll
 0001:0001d51c       RtlLookupFunctionEntry     000000003751e51c f   kernel32:KERNEL32.dll
 0001:0001d524       __GSHandlerCheckCommon     000000003751e524 f   MSVCRT:gshandler.obj
 0001:0001d588       __GSHandlerCheck           000000003751e588 f   MSVCRT:gshandler.obj
 0001:0001d7c0       ??__Fs_dummyMemReplay@?1??CryGetIMemReplay@@YAPEAUIMemReplay@@XZ@YAXXZ 000000003751e7c0 f i CryLiveCreate.obj
 0001:0001d7e0       ??__Fp@?1??CreateClassInstance@CFactory@CEngineModule_CryLiveCreate@@UEBA?AV?$shared_ptr@UICryUnknown@@@boost@@XZ@YAXXZ 000000003751e7e0 f i CryLiveCreate.obj
 0002:00000000       __imp_CreateEventA         000000003751f000     kernel32:KERNEL32.dll
 0002:00000008       __imp_CloseHandle          000000003751f008     kernel32:KERNEL32.dll
 0002:00000010       __imp_WaitForSingleObject  000000003751f010     kernel32:KERNEL32.dll
 0002:00000018       __imp_CreateMutexA         000000003751f018     kernel32:KERNEL32.dll
 0002:00000020       __imp_ReleaseMutex         000000003751f020     kernel32:KERNEL32.dll
 0002:00000028       __imp_InitializeCriticalSection 000000003751f028     kernel32:KERNEL32.dll
 0002:00000030       __imp_DeleteCriticalSection 000000003751f030     kernel32:KERNEL32.dll
 0002:00000038       __imp_EnterCriticalSection 000000003751f038     kernel32:KERNEL32.dll
 0002:00000040       __imp_LeaveCriticalSection 000000003751f040     kernel32:KERNEL32.dll
 0002:00000048       __imp_CreateSemaphoreA     000000003751f048     kernel32:KERNEL32.dll
 0002:00000050       __imp_GetCurrentThreadId   000000003751f050     kernel32:KERNEL32.dll
 0002:00000058       __imp_ResumeThread         000000003751f058     kernel32:KERNEL32.dll
 0002:00000060       __imp_LoadLibraryA         000000003751f060     kernel32:KERNEL32.dll
 0002:00000068       __imp_GetProcAddress       000000003751f068     kernel32:KERNEL32.dll
 0002:00000070       __imp_GetModuleHandleA     000000003751f070     kernel32:KERNEL32.dll
 0002:00000078       __imp_IsDebuggerPresent    000000003751f078     kernel32:KERNEL32.dll
 0002:00000080       __imp_Sleep                000000003751f080     kernel32:KERNEL32.dll
 0002:00000088       __imp_LocalAlloc           000000003751f088     kernel32:KERNEL32.dll
 0002:00000090       __imp_FreeLibrary          000000003751f090     kernel32:KERNEL32.dll
 0002:00000098       __imp_GetLastError         000000003751f098     kernel32:KERNEL32.dll
 0002:000000a0       __imp_SetErrorMode         000000003751f0a0     kernel32:KERNEL32.dll
 0002:000000a8       __imp_GetErrorMode         000000003751f0a8     kernel32:KERNEL32.dll
 0002:000000b0       __imp_GetSystemTime        000000003751f0b0     kernel32:KERNEL32.dll
 0002:000000b8       __imp_DeleteFileA          000000003751f0b8     kernel32:KERNEL32.dll
 0002:000000c0       __imp_GetTickCount         000000003751f0c0     kernel32:KERNEL32.dll
 0002:000000c8       __imp_FileTimeToSystemTime 000000003751f0c8     kernel32:KERNEL32.dll
 0002:000000d0       __imp_CreateDirectoryA     000000003751f0d0     kernel32:KERNEL32.dll
 0002:000000d8       __imp_GetEnvironmentVariableA 000000003751f0d8     kernel32:KERNEL32.dll
 0002:000000e0       __imp_DecodePointer        000000003751f0e0     kernel32:KERNEL32.dll
 0002:000000e8       __imp_QueryPerformanceCounter 000000003751f0e8     kernel32:KERNEL32.dll
 0002:000000f0       __imp_RtlCaptureContext    000000003751f0f0     kernel32:KERNEL32.dll
 0002:000000f8       __imp_RtlLookupFunctionEntry 000000003751f0f8     kernel32:KERNEL32.dll
 0002:00000100       __imp_RtlVirtualUnwind     000000003751f100     kernel32:KERNEL32.dll
 0002:00000108       __imp_SetUnhandledExceptionFilter 000000003751f108     kernel32:KERNEL32.dll
 0002:00000110       __imp_UnhandledExceptionFilter 000000003751f110     kernel32:KERNEL32.dll
 0002:00000118       __imp_GetCurrentProcess    000000003751f118     kernel32:KERNEL32.dll
 0002:00000120       __imp_TerminateProcess     000000003751f120     kernel32:KERNEL32.dll
 0002:00000128       __imp_GetSystemTimeAsFileTime 000000003751f128     kernel32:KERNEL32.dll
 0002:00000130       __imp_GetCurrentProcessId  000000003751f130     kernel32:KERNEL32.dll
 0002:00000138       __imp_EncodePointer        000000003751f138     kernel32:KERNEL32.dll
 0002:00000140       \177KERNEL32_NULL_THUNK_DATA 000000003751f140     kernel32:KERNEL32.dll
 0002:00000148       __imp_strnicmp             000000003751f148     MSVCRT:MSVCR100.dll
 0002:00000148       __imp__strnicmp            000000003751f148     MSVCRT:MSVCR100.dll
 0002:00000150       __imp___crt_debugger_hook  000000003751f150     MSVCRT:MSVCR100.dll
 0002:00000158       __imp___clean_type_info_names_internal 000000003751f158     MSVCRT:MSVCR100.dll
 0002:00000160       __imp___CppXcptFilter      000000003751f160     MSVCRT:MSVCR100.dll
 0002:00000168       __imp__amsg_exit           000000003751f168     MSVCRT:MSVCR100.dll
 0002:00000170       __imp__encoded_null        000000003751f170     MSVCRT:MSVCR100.dll
 0002:00000178       __imp_free                 000000003751f178     MSVCRT:MSVCR100.dll
 0002:00000180       __imp__initterm_e          000000003751f180     MSVCRT:MSVCR100.dll
 0002:00000188       __imp__initterm            000000003751f188     MSVCRT:MSVCR100.dll
 0002:00000190       __imp__purecall            000000003751f190     MSVCRT:MSVCR100.dll
 0002:00000198       __imp_memcpy               000000003751f198     MSVCRT:MSVCR100.dll
 0002:000001a0       __imp_memmove              000000003751f1a0     MSVCRT:MSVCR100.dll
 0002:000001a8       __imp_memset               000000003751f1a8     MSVCRT:MSVCR100.dll
 0002:000001b0       __imp__beginthreadex       000000003751f1b0     MSVCRT:MSVCR100.dll
 0002:000001b8       __imp_sscanf_s             000000003751f1b8     MSVCRT:MSVCR100.dll
 0002:000001c0       __imp_sprintf              000000003751f1c0     MSVCRT:MSVCR100.dll
 0002:000001c8       __imp_strcspn              000000003751f1c8     MSVCRT:MSVCR100.dll
 0002:000001d0       __imp_strchr               000000003751f1d0     MSVCRT:MSVCR100.dll
 0002:000001d8       __imp_exit                 000000003751f1d8     MSVCRT:MSVCR100.dll
 0002:000001e0       __imp__set_invalid_parameter_handler 000000003751f1e0     MSVCRT:MSVCR100.dll
 0002:000001e8       __imp__set_purecall_handler 000000003751f1e8     MSVCRT:MSVCR100.dll
 0002:000001f0       __imp_??0exception@std@@QEAA@AEBQEBDH@Z 000000003751f1f0     MSVCRT:MSVCR100.dll
 0002:000001f8       __imp_?what@exception@std@@UEBAPEBDXZ 000000003751f1f8     MSVCRT:MSVCR100.dll
 0002:00000200       __imp_??1exception@std@@UEAA@XZ 000000003751f200     MSVCRT:MSVCR100.dll
 0002:00000208       __imp_stricmp              000000003751f208     MSVCRT:MSVCR100.dll
 0002:00000208       __imp_strcmpi              000000003751f208     MSVCRT:MSVCR100.dll
 0002:00000208       __imp__stricmp             000000003751f208     MSVCRT:MSVCR100.dll
 0002:00000210       __imp_abort                000000003751f210     MSVCRT:MSVCR100.dll
 0002:00000218       __imp_puts                 000000003751f218     MSVCRT:MSVCR100.dll
 0002:00000220       __imp_strncmp              000000003751f220     MSVCRT:MSVCR100.dll
 0002:00000228       __imp_strncpy_s            000000003751f228     MSVCRT:MSVCR100.dll
 0002:00000230       __imp_strcpy_s             000000003751f230     MSVCRT:MSVCR100.dll
 0002:00000238       __imp_fclose               000000003751f238     MSVCRT:MSVCR100.dll
 0002:00000240       __imp_fread                000000003751f240     MSVCRT:MSVCR100.dll
 0002:00000248       __imp_ftell                000000003751f248     MSVCRT:MSVCR100.dll
 0002:00000250       __imp_fseek                000000003751f250     MSVCRT:MSVCR100.dll
 0002:00000258       __imp_fopen                000000003751f258     MSVCRT:MSVCR100.dll
 0002:00000260       __imp__vscprintf           000000003751f260     MSVCRT:MSVCR100.dll
 0002:00000268       __imp__vsnprintf           000000003751f268     MSVCRT:MSVCR100.dll
 0002:00000268       __imp_vsnprintf            000000003751f268     MSVCRT:MSVCR100.dll
 0002:00000270       __imp_sprintf_s            000000003751f270     MSVCRT:MSVCR100.dll
 0002:00000278       __imp__endthreadex         000000003751f278     MSVCRT:MSVCR100.dll
 0002:00000280       __imp_strspn               000000003751f280     MSVCRT:MSVCR100.dll
 0002:00000288       __imp_atoi                 000000003751f288     MSVCRT:MSVCR100.dll
 0002:00000290       __imp_strstr               000000003751f290     MSVCRT:MSVCR100.dll
 0002:00000298       __imp_printf               000000003751f298     MSVCRT:MSVCR100.dll
 0002:000002a0       __imp___C_specific_handler 000000003751f2a0     MSVCRT:MSVCR100.dll
 0002:000002a8       __imp__unlock              000000003751f2a8     MSVCRT:MSVCR100.dll
 0002:000002b0       __imp___dllonexit          000000003751f2b0     MSVCRT:MSVCR100.dll
 0002:000002b8       __imp__lock                000000003751f2b8     MSVCRT:MSVCR100.dll
 0002:000002c0       __imp__onexit              000000003751f2c0     MSVCRT:MSVCR100.dll
 0002:000002c8       __imp__malloc_crt          000000003751f2c8     MSVCRT:MSVCR100.dll
 0002:000002d0       \177MSVCR100_NULL_THUNK_DATA 000000003751f2d0     MSVCRT:MSVCR100.dll
 0002:000002d8       __imp_MessageBoxA          000000003751f2d8     user32:USER32.dll
 0002:000002e0       \177USER32_NULL_THUNK_DATA 000000003751f2e0     user32:USER32.dll
 0002:000002e8       __imp_select               000000003751f2e8     Ws2_32:WS2_32.dll
 0002:000002f0       __imp___WSAFDIsSet         000000003751f2f0     Ws2_32:WS2_32.dll
 0002:000002f8       __imp_connect              000000003751f2f8     Ws2_32:WS2_32.dll
 0002:00000300       __imp_gethostname          000000003751f300     Ws2_32:WS2_32.dll
 0002:00000308       __imp_gethostbyname        000000003751f308     Ws2_32:WS2_32.dll
 0002:00000310       __imp_inet_addr            000000003751f310     Ws2_32:WS2_32.dll
 0002:00000318       __imp_send                 000000003751f318     Ws2_32:WS2_32.dll
 0002:00000320       __imp_accept               000000003751f320     Ws2_32:WS2_32.dll
 0002:00000328       __imp_listen               000000003751f328     Ws2_32:WS2_32.dll
 0002:00000330       __imp_htonl                000000003751f330     Ws2_32:WS2_32.dll
 0002:00000338       __imp_htons                000000003751f338     Ws2_32:WS2_32.dll
 0002:00000340       __imp_bind                 000000003751f340     Ws2_32:WS2_32.dll
 0002:00000348       __imp_socket               000000003751f348     Ws2_32:WS2_32.dll
 0002:00000350       __imp_setsockopt           000000003751f350     Ws2_32:WS2_32.dll
 0002:00000358       __imp_closesocket          000000003751f358     Ws2_32:WS2_32.dll
 0002:00000360       __imp_ioctlsocket          000000003751f360     Ws2_32:WS2_32.dll
 0002:00000368       __imp_recv                 000000003751f368     Ws2_32:WS2_32.dll
 0002:00000370       __imp_ntohl                000000003751f370     Ws2_32:WS2_32.dll
 0002:00000378       \177WS2_32_NULL_THUNK_DATA 000000003751f378     Ws2_32:WS2_32.dll
 0002:00000380       __xc_a                     000000003751f380     MSVCRT:cinitexe.obj
 0002:000003e0       __xc_z                     000000003751f3e0     MSVCRT:cinitexe.obj
 0002:000003e8       __xi_a                     000000003751f3e8     MSVCRT:cinitexe.obj
 0002:000003f8       __xi_z                     000000003751f3f8     MSVCRT:cinitexe.obj
 0002:00000420       ??_C@_0BO@ELGNHIIF@?$CBCRY_LIVECREATE_ANYONE_THERE?$DP?$AA@ 000000003751f420     CryLiveCreate.obj
 0002:00000440       ??_C@_0BA@FELBPFAN@255?4255?4255?4255?$AA@ 000000003751f440     CryLiveCreate.obj
 0002:00000450       ??_7IMemReplay@@6B@        000000003751f450     CryLiveCreate.obj
 0002:00000580       ??_7CrySimpleThreadSelf@@6B@ 000000003751f580     CryLiveCreate.obj
 0002:00000588       ??_C@_0DJ@DLJMMMP@Could?5not?5access?5CrySystem?4dll?5?$CI@ 000000003751f588     CryLiveCreate.obj
 0002:000005c8       ??_C@_0P@NHEMOHAI@Memory?5Manager?$AA@ 000000003751f5c8     CryLiveCreate.obj
 0002:000005d8       ??_C@_0O@FFDHMLKN@CrySystem?4dll?$AA@ 000000003751f5d8     CryLiveCreate.obj
 0002:000005e8       ??_C@_0BO@JDKBDPNB@CryGetIMemoryManagerInterface?$AA@ 000000003751f5e8     CryLiveCreate.obj
 0002:00000608       ??_C@_0BB@PNKHDABP@CrySystemCrtFree?$AA@ 000000003751f608     CryLiveCreate.obj
 0002:00000620       ??_C@_0BB@MFMFBMDO@CrySystemCrtSize?$AA@ 000000003751f620     CryLiveCreate.obj
 0002:00000638       ??_C@_0BD@BBIFHONI@CrySystemCrtMalloc?$AA@ 000000003751f638     CryLiveCreate.obj
 0002:00000650       ??_C@_0O@LCCIKADF@CryGetMemSize?$AA@ 000000003751f650     CryLiveCreate.obj
 0002:00000660       ??_C@_07CKAGCLEE@CryFree?$AA@ 000000003751f660     CryLiveCreate.obj
 0002:00000668       ??_C@_0L@FICCDMFO@CryRealloc?$AA@ 000000003751f668     CryLiveCreate.obj
 0002:00000678       ??_C@_09MCKPOEAK@CryMalloc?$AA@ 000000003751f678     CryLiveCreate.obj
 0002:00000688       ?iid@?1??IID@IEngineModule@@CAAEBUCryGUID@@XZ@4U3@B 000000003751f688     CryLiveCreate.obj
 0002:00000698       ??_7ICryFactory@@6B@       000000003751f698     CryLiveCreate.obj
 0002:000006c8       ??_7ISystemEventListener@@6B@ 000000003751f6c8     CryLiveCreate.obj
 0002:000006d8       ??_7ICryUnknown@@6B@       000000003751f6d8     CryLiveCreate.obj
 0002:000006f8       ??_C@_02DKCKIIND@?$CFs?$AA@ 000000003751f6f8     CryLiveCreate.obj
 0002:00000700       ?iid@?1??IID@ICryUnknown@@CAAEBUCryGUID@@XZ@4U3@B 000000003751f700     CryLiveCreate.obj
 0002:00000710       ??_7CDummyMemReplay@@6B@   000000003751f710     CryLiveCreate.obj
 0002:00000840       ??_C@_0BD@PJOKHJBB@Pure?5function?5call?$AA@ 000000003751f840     CryLiveCreate.obj
 0002:00000858       ??_C@_0CL@LKHBOBAH@Invalid?5parameter?5detected?5in?5CR@ 000000003751f858     CryLiveCreate.obj
 0002:00000888       ??_C@_0BO@HAMEIFMK@Critical?5Section?5hanging?5lock?$AA@ 000000003751f888     CryLiveCreate.obj
 0002:000008a8       ??_7CSystemEventListner_LiveCreate@@6B@ 000000003751f8a8     CryLiveCreate.obj
 0002:000008b8       ??_C@_0DM@BDLAIJDG@Missing?5NULL?5LiveCreate?5implemen@ 000000003751f8b8     CryLiveCreate.obj
 0002:000008f8       ??_C@_0O@DAPGGCLB@CryLiveCreate?$AA@ 000000003751f8f8     CryLiveCreate.obj
 0002:00000908       ??_7CEngineModule_CryLiveCreate@@6B@ 000000003751f908     CryLiveCreate.obj
 0002:00000940       ??_C@_09BHIABECK@CryEngine?$AA@ 000000003751f940     CryLiveCreate.obj
 0002:0000094c       ??_C@_06ICGJLFIM@string?$AA@ 000000003751f94c     CryLiveCreate.obj
 0002:00000958       ??_7CFactory@CEngineModule_CryLiveCreate@@6B@ 000000003751f958     CryLiveCreate.obj
 0002:00000988       ??_7bad_alloc@std@@6B@     000000003751f988     CryLiveCreate.obj
 0002:00000998       ??_C@_0P@GHFPNOJB@bad?5allocation?$AA@ 000000003751f998     CryLiveCreate.obj
 0002:000009a8       ??_C@_0BL@FPNMKCO@EngineModule_CryLiveCreate?$AA@ 000000003751f9a8     CryLiveCreate.obj
 0002:000009c8       ?cid@?1??GetClassID@CFactory@CEngineModule_CryLiveCreate@@UEBAAEBUCryGUID@@XZ@4U4@B 000000003751f9c8     CryLiveCreate.obj
 0002:000009d8       ??_7sp_counted_base@detail@boost@@6B@ 000000003751f9d8     CryLiveCreate.obj
 0002:000009f8       ??_7?$sp_counted_impl_p@VCEngineModule_CryLiveCreate@@@detail@boost@@6B@ 000000003751f9f8     CryLiveCreate.obj
 0002:00000a18       ??_C@_0BN@FOKPCDPC@Boost?5threw?5an?5exception?3?5?$CFs?$AA@ 000000003751fa18     CryLiveCreate.obj
 0002:00000a38       ??_C@_01IHBHIGKO@?0?$AA@   000000003751fa38     CryLiveCreate.obj
 0002:00000a3c       ??_C@_03IPCHNKJI@PS3?$AA@  000000003751fa3c     LiveCreate.obj
 0002:00000a40       ??_C@_04CMIAHEHG@X360?$AA@ 000000003751fa40     LiveCreate.obj
 0002:00000a48       ??_C@_08DKHDPPEE@EditorPC?$AA@ 000000003751fa48     LiveCreate.obj
 0002:00000a54       ??_C@_06PKCFDBDC@GamePC?$AA@ 000000003751fa54     LiveCreate.obj
 0002:00000a60       ??_7IObserver@FileSyncManager@LiveCreate@@6B@ 000000003751fa60     LiveCreate.obj
 0002:00000a80       ??_7IManager@LiveCreate@@6B@ 000000003751fa80     LiveCreate.obj
 0002:00000c00       ??_7IPlatformHandlerFactory@LiveCreate@@6B@ 000000003751fc00     LiveCreate.obj
 0002:00000c28       ??_C@_0L@PHNBOBLE@Init?5done?4?$AA@ 000000003751fc28     LiveCreate.obj
 0002:00000c40       ??_C@_0EC@CPHNADBN@Initializing?5listening?5at?5port?3?5@ 000000003751fc40     LiveCreate.obj
 0002:00000c88       ??_C@_0BE@PCAECBPN@Shutdown?5completed?4?$AA@ 000000003751fc88     LiveCreate.obj
 0002:00000ca0       ??_C@_0M@PILEMGMH@Shutdown?4?4?4?$AA@ 000000003751fca0     LiveCreate.obj
 0002:00000cb0       ??_C@_0N@EFGMCLPD@lc_enablelog?$AA@ 000000003751fcb0     LiveCreate.obj
 0002:00000cc0       ??_C@_0DP@KJJFNDEN@Could?5not?5allocate?5memory?5for?5se@ 000000003751fcc0     LiveCreate.obj
 0002:00000d00       ??_C@_08BABJIOEM@filename?$AA@ 000000003751fd00     LiveCreate.obj
 0002:00000d10       ??_C@_0BD@NFLLDKOP@file_change_notify?$AA@ 000000003751fd10     LiveCreate.obj
 0002:00000d28       ??_C@_0P@PCJPAHLM@out?5of?5memory?6?$AA@ 000000003751fd28     LiveCreate.obj
 0002:00000d38       ??_C@_06NBFPPGEG@vector?$AA@ 000000003751fd38     LiveCreate.obj
 0002:00000d40       ??_7CNullManager@LiveCreate@@6B@ 000000003751fd40     LiveCreate.obj
 0002:00000ec0       ??_7PlatformHandlerFactory_EditorPC@LiveCreate@@6B@ 000000003751fec0     LiveCreate.obj
 0002:00000ee8       ??_7PlatformHandlerFactory_GamePC@LiveCreate@@6B@ 000000003751fee8     LiveCreate.obj
 0002:00000f10       ??_C@_07MCNDKCLD@?$FLLC?$FN?5?$CFs?$AA@ 000000003751ff10     LiveCreate.obj
 0002:00000f18       ??_C@_09LGJOJGI@NO?5PEERS?$CB?$AA@ 000000003751ff18     LiveCreate.obj
 0002:00000f28       ??_C@_0CG@LPGJEDDC@Sync?3?5SendControllerData?5for?5pee@ 000000003751ff28     LiveCreate.obj
 0002:00000f50       ??_C@_0BC@DCMMDGPL@Sync?5peer?5?$CD?$CFd?3?5?$CFd?$AA@ 000000003751ff50     LiveCreate.obj
 0002:00000f70       ??_C@_0EA@KIPFILOC@Could?5not?5find?5a?5proper?5platform@ 000000003751ff70     LiveCreate.obj
 0002:00000fb0       ??_C@_0BI@GMFNHKPF@Searching?5platform?5?8?$CFs?8?$AA@ 000000003751ffb0     LiveCreate.obj
 0002:00000fc8       ??_C@_0CJ@HPKKIDPF@Finding?5IP?5from?5platform?5handler@ 000000003751ffc8     LiveCreate.obj
 0002:00000ff8       ??_C@_0CD@BFAEHCHE@Finding?5IP?5from?5connections?3?5?$CFs?5@ 000000003751fff8     LiveCreate.obj
 0002:00001020       ??_C@_0CG@IKKDFEMP@Peer?5added?5and?5connection?5set?5?8?$CF@ 0000000037520020     LiveCreate.obj
 0002:00001048       ??_C@_0CG@MMANFLAF@Peer?5IP?3?8?$CFs?8?5connected?0?5platform@ 0000000037520048     LiveCreate.obj
 0002:00001070       ??_C@_0CG@FJBJLCKB@CManager?3?3OnConnected?5NULL?5conne@ 0000000037520070     LiveCreate.obj
 0002:00001098       ??_C@_0CB@JLGNLNBJ@Peer?5link?5net?5connection?5closed?4@ 0000000037520098     LiveCreate.obj
 0002:000010c0       ??_C@_0DE@KENCAIDB@No?5peer?5link?5found?5on?5peer?5disco@ 00000000375200c0     LiveCreate.obj
 0002:000010f8       ??_C@_0DA@KJCBDEBG@CManager?3?3OnDisconnected?$CIHPeerCo@ 00000000375200f8     LiveCreate.obj
 0002:00001128       ??_C@_0CC@ILBOOLOK@Added?5peer?5link?5for?5connection?5?$CF@ 0000000037520128     LiveCreate.obj
 0002:00001150       ??_C@_0BG@BACEKDGF@Created?5link?5for?5?8?$CFs?8?$AA@ 0000000037520150     LiveCreate.obj
 0002:00001170       ??_C@_0EL@IFGPEOHK@Created?5link?5for?5target?5?8?$CFs?8?5for@ 0000000037520170     LiveCreate.obj
 0002:000011c0       ??_C@_0CA@DKNGMKNB@Cannot?5create?5peer?5link?5to?5?8?$CFs?8?$AA@ 00000000375201c0     LiveCreate.obj
 0002:000011e0       ??_C@_0CL@FNDPKDPO@Cannot?5create?5platform?5handler?5f@ 00000000375201e0     LiveCreate.obj
 0002:00001210       ??_C@_0EN@BNFODFPD@Found?5link?5for?5target?5?8?$CFs?8?5with?5@ 0000000037520210     LiveCreate.obj
 0002:00001260       ??_C@_0CD@DJCKPONN@Peer?5presented?5itself?5?$CIaddress?5?$CF@ 0000000037520260     LiveCreate.obj
 0002:00001288       ??_C@_0DL@MACJOJJN@CManager?3?3ConnectToPeer1?3?5Connec@ 0000000037520288     LiveCreate.obj
 0002:000012c8       ??_C@_0CL@GBMDKGBI@Peer?5is?5already?5connected?5or?5con@ 00000000375202c8     LiveCreate.obj
 0002:000012f8       ??_C@_0DL@KEMJJCGD@CManager?3?3ConnectToPeer2?3?5Connec@ 00000000375202f8     LiveCreate.obj
 0002:00001340       ??_C@_0EE@PHPBEJEA@A?5controller?5message?5arrived?5ctr@ 0000000037520340     LiveCreate.obj
 0002:00001390       ??_C@_0EB@JNEOPIAH@Could?5not?5get?5peer?5info?5on?5CMana@ 0000000037520390     LiveCreate.obj
 0002:000013e0       ??_C@_0GH@GJNDJCIP@Peer?5says?5Hello?$CB?5platform?3?8?$CFs?8?5t@ 00000000375203e0     LiveCreate.obj
 0002:00001448       ??_C@_0CK@OFAKAHLN@Peer?5info?5came?5from?5?8?$CFd?8?5?$CItarget@ 0000000037520448     LiveCreate.obj
 0002:00001478       ??_C@_0DH@ONOFMBEH@Handling?5message?5?$CItype?3?$CFd?5id?3?$CFd?5@ 0000000037520478     LiveCreate.obj
 0002:000014b0       ??_C@_0BG@KDFIJDAM@Deleting?5sync?5data?5?$CFp?$AA@ 00000000375204b0     LiveCreate.obj
 0002:000014c8       ??_7CManager@LiveCreate@@6BIObserver@FileSyncManager@1@@ 00000000375204c8     LiveCreate.obj
 0002:000014f0       ??_7CManager@LiveCreate@@6BIManager@1@@ 00000000375204f0     LiveCreate.obj
 0002:00001670       ??_C@_0CM@FJIPJBC@Enables?5CryLiveCreate?5specific?5l@ 0000000037520670     LiveCreate.obj
 0002:0000169c       ??_C@_06HPGEIPLA@?$DMnull?$DO?$AA@ 000000003752069c     LiveCreateCtrl_Camera.obj
 0002:000016a8       ??_C@_07KAALEJHI@?$DMlocal?$DO?$AA@ 00000000375206a8     LiveCreateCtrl_Camera.obj
 0002:000016b0       ??_7CameraController@LiveCreate@@6B@ 00000000375206b0     LiveCreateCtrl_Camera.obj
 0002:00001738       ??_C@_06JCBBMBIP@Camera?$AA@ 0000000037520738     LiveCreateCtrl_Camera.obj
 0002:00001740       ??_C@_06FNKMPIBD@camera?$AA@ 0000000037520740     LiveCreateCtrl_Camera.obj
 0002:00001750       ??_C@_0EJ@EOGCMENC@This?5controller?5syncs?5the?5camera@ 0000000037520750     LiveCreateCtrl_Camera.obj
 0002:0000179c       ??_C@_04JNABKDKF@sync?$AA@ 000000003752079c     LiveCreateCtrl_Camera.obj
 0002:000017a8       ??_C@_09HPKLLIJF@direction?$AA@ 00000000375207a8     LiveCreateCtrl_Camera.obj
 0002:000017b8       ??_C@_08OAGMDKAF@position?$AA@ 00000000375207b8     LiveCreateCtrl_Camera.obj
 0002:000017c4       __real@40000000            00000000375207c4     LiveCreateCtrl_Camera.obj
 0002:000017c8       __real@3f800000            00000000375207c8     LiveCreateCtrl_Camera.obj
 0002:000017d0       ??_C@_0CI@IOKCCNHB@Deleting?5Reference?5Counted?5Objec@ 00000000375207d0     LiveCreateCtrl_Camera.obj
 0002:00001800       __mask@@NegFloat@          0000000037520800     LiveCreateCtrl_Camera.obj
 0002:00001810       __real@bf800000            0000000037520810     LiveCreateCtrl_Camera.obj
 0002:00001814       __real@3727c5ac            0000000037520814     LiveCreateCtrl_Camera.obj
 0002:00001818       __real@3f3504f3            0000000037520818     LiveCreateCtrl_Camera.obj
 0002:00001820       ??_C@_0DJ@GDJPDHPN@?$FLcamera?$FN?5Received?5enable?$CI?$CFd?$CJ?5pos@ 0000000037520820     LiveCreateCtrl_Camera.obj
 0002:00001860       ??_C@_0DJ@JNAMLABP@?$FLcamera?$FN?5Sending?5enabled?$CI?$CFd?$CJ?5pos@ 0000000037520860     LiveCreateCtrl_Camera.obj
 0002:000018a0       ??_C@_0BB@IPNBLGKE@g_detachCamera?50?$AA@ 00000000375208a0     LiveCreateCtrl_Camera.obj
 0002:000018b8       ??_C@_0CC@OPCBPOOK@e_ObjectLayersActivationPhysics?5@ 00000000375208b8     LiveCreateCtrl_Camera.obj
 0002:000018e0       ??_C@_0BL@CEIAODEJ@e_ObjectLayersActivation?51?$AA@ 00000000375208e0     LiveCreateCtrl_Camera.obj
 0002:00001900       ??_C@_0BC@EIOHGPLF@mov_NoCutscenes?50?$AA@ 0000000037520900     LiveCreateCtrl_Camera.obj
 0002:00001918       ??_C@_0N@DDKOBKOA@p_fly_mode?50?$AA@ 0000000037520918     LiveCreateCtrl_Camera.obj
 0002:00001928       ??_C@_0O@ONLCLDBI@AI_NoUpdate?50?$AA@ 0000000037520928     LiveCreateCtrl_Camera.obj
 0002:00001938       ??_C@_0BC@FOKHPPMN@AI_IgnorePlayer?50?$AA@ 0000000037520938     LiveCreateCtrl_Camera.obj
 0002:00001950       ??_C@_08FPPDEJEI@sys_ai?51?$AA@ 0000000037520950     LiveCreateCtrl_Camera.obj
 0002:00001960       ??_C@_0M@IMNJGFFB@g_godMode?50?$AA@ 0000000037520960     LiveCreateCtrl_Camera.obj
 0002:00001970       ??_C@_0EA@MHHLFPJL@Disabling?5camera?5sync?0?5exiting?5f@ 0000000037520970     LiveCreateCtrl_Camera.obj
 0002:000019b0       ??_C@_0BB@JGMKIHOF@g_detachCamera?51?$AA@ 00000000375209b0     LiveCreateCtrl_Camera.obj
 0002:000019c8       ??_C@_0CC@PGDKMPKL@e_ObjectLayersActivationPhysics?5@ 00000000375209c8     LiveCreateCtrl_Camera.obj
 0002:000019f0       ??_C@_0BL@DNJLNCAI@e_ObjectLayersActivation?50?$AA@ 00000000375209f0     LiveCreateCtrl_Camera.obj
 0002:00001a10       ??_C@_0BC@FBPMFOPE@mov_NoCutscenes?51?$AA@ 0000000037520a10     LiveCreateCtrl_Camera.obj
 0002:00001a28       ??_C@_0N@CKLFCLKB@p_fly_mode?51?$AA@ 0000000037520a28     LiveCreateCtrl_Camera.obj
 0002:00001a38       ??_C@_0O@PEKJICFJ@AI_NoUpdate?51?$AA@ 0000000037520a38     LiveCreateCtrl_Camera.obj
 0002:00001a48       ??_C@_0BC@EHLMMOIM@AI_IgnorePlayer?51?$AA@ 0000000037520a48     LiveCreateCtrl_Camera.obj
 0002:00001a60       ??_C@_08EGOIHIAJ@sys_ai?50?$AA@ 0000000037520a60     LiveCreateCtrl_Camera.obj
 0002:00001a70       ??_C@_0M@JFMCFEBA@g_godMode?51?$AA@ 0000000037520a70     LiveCreateCtrl_Camera.obj
 0002:00001a80       ??_C@_0CP@OLKCGBJH@Enabling?5camera?5sync?0?5entering?5f@ 0000000037520a80     LiveCreateCtrl_Camera.obj
 0002:00001ab0       __real@3d4ccccd            0000000037520ab0     LiveCreateCtrl_Camera.obj
 0002:00001ab4       __real@38d1b717            0000000037520ab4     LiveCreateCtrl_Camera.obj
 0002:00001ac0       ??_7IController@LiveCreate@@6B@ 0000000037520ac0     LiveCreateCtrl_Common.obj
 0002:00001b50       ??_7CommonController@LiveCreate@@6B@ 0000000037520b50     LiveCreateCtrl_Common.obj
 0002:00001bd8       ??_7IConsoleVarSink@@6B@   0000000037520bd8     LiveCreateCtrl_CVar.obj
 0002:00001bf0       ??_C@_04JMPEMAGG@CVar?$AA@ 0000000037520bf0     LiveCreateCtrl_CVar.obj
 0002:00001bf8       ??_C@_04PNAHEAFM@cvar?$AA@ 0000000037520bf8     LiveCreateCtrl_CVar.obj
 0002:00001c00       ??_C@_0CM@HALPGDCA@This?5controller?5syncs?5the?5consol@ 0000000037520c00     LiveCreateCtrl_CVar.obj
 0002:00001c30       ??_C@_0CB@NLOKMCHG@?$FLcvar?$FN?5Sending?5cvar?3?5?8?$CFs?8?5?$DN?5?8?$CFs?8@ 0000000037520c30     LiveCreateCtrl_CVar.obj
 0002:00001c58       ??_C@_0BI@MPDEOKIL@?$FLcvar?$FN?5Sending?5?$CFd?5cvars?$AA@ 0000000037520c58     LiveCreateCtrl_CVar.obj
 0002:00001c70       ??_C@_0CC@MKCJFMLF@?$FLcvar?$FN?5Received?5cvar?3?5?8?$CFs?8?5?$DN?5?8?$CFs@ 0000000037520c70     LiveCreateCtrl_CVar.obj
 0002:00001c98       ??_C@_0BJ@HALLNPGN@?$FLcvar?$FN?5Received?5?$CFd?5cvars?$AA@ 0000000037520c98     LiveCreateCtrl_CVar.obj
 0002:00001cb8       ??_C@_0BK@INNOOEPG@?$FLcvar?$FN?5Receiving?5?$CFd?5cvars?$AA@ 0000000037520cb8     LiveCreateCtrl_CVar.obj
 0002:00001cd8       ??_C@_0CP@HNHELJFH@?$FLcvar?$FN?5Receiving?5cvars?5?$CIdatasize@ 0000000037520cd8     LiveCreateCtrl_CVar.obj
 0002:00001d08       ??_C@_0CB@KOMFMLLG@?$FLcvar?$FN?5Setting?5cvar?3?5?8?$CFs?8?5?$DN?5?8?$CFs?8@ 0000000037520d08     LiveCreateCtrl_CVar.obj
 0002:00001d30       ??_C@_0BI@IKOLDELO@?$FLcvar?$FN?5Setting?5?$CFd?5cvars?$AA@ 0000000037520d30     LiveCreateCtrl_CVar.obj
 0002:00001d48       ??_C@_08JGBOOFEC@sys_spec?$AA@ 0000000037520d48     LiveCreateCtrl_CVar.obj
 0002:00001d58       ??_C@_0O@FFOHGDOH@r_debuglights?$AA@ 0000000037520d58     LiveCreateCtrl_CVar.obj
 0002:00001d68       ??_7CVarController@LiveCreate@@6BIConsoleVarSink@@@ 0000000037520d68     LiveCreateCtrl_CVar.obj
 0002:00001d80       ??_7CVarController@LiveCreate@@6BCommonController@1@@ 0000000037520d80     LiveCreateCtrl_CVar.obj
 0002:00001e08       ??_C@_0CL@GGNOGCML@CVar?5?$CFs?5not?5allowed?5to?5sync?5with@ 0000000037520e08     LiveCreateCtrl_CVar.obj
 0002:00001e38       ??_C@_0BB@FFLAAGB@disallowed_cvars?$AA@ 0000000037520e38     LiveCreateCtrl_CVar.obj
 0002:00001e50       ??_C@_0N@KMCDGBNI@cvar_changed?$AA@ 0000000037520e50     LiveCreateCtrl_CVar.obj
 0002:00001e60       ??_C@_08HPDMGIEC@Entities?$AA@ 0000000037520e60     LiveCreateCtrl_Entities.obj
 0002:00001e70       ??_C@_08PNMNOKOB@entities?$AA@ 0000000037520e70     LiveCreateCtrl_Entities.obj
 0002:00001e80       ??_C@_0FN@IJALLDCF@This?5controller?5syncs?5the?5entiti@ 0000000037520e80     LiveCreateCtrl_Entities.obj
 0002:00001ee0       ??_C@_0CD@LDOKKKIA@?$FLEntity?$FN?5Sent?5deleted?5entity?5id?5@ 0000000037520ee0     LiveCreateCtrl_Entities.obj
 0002:00001f08       ??_C@_0CA@KMGJBMPB@?$FLEntity?$FN?5Sending?5?$CFd?5deleted?5ids?$AA@ 0000000037520f08     LiveCreateCtrl_Entities.obj
 0002:00001f28       ??_C@_0CE@JOOPOGFL@?$FLEntity?$FN?5Sent?5xml?5buffer?5of?5size@ 0000000037520f28     LiveCreateCtrl_Entities.obj
 0002:00001f50       ??_C@_0CJ@LGFBNDIK@?$FLEntity?$FN?5Sending?5?$CFd?5entity?5prope@ 0000000037520f50     LiveCreateCtrl_Entities.obj
 0002:00001f80       ??_C@_0CG@FNDHPMOC@?$FLEntity?$FN?5Sending?5?$CFd?5entity?5trans@ 0000000037520f80     LiveCreateCtrl_Entities.obj
 0002:00001fb0       ??_7EntitiesController@LiveCreate@@6B@ 0000000037520fb0     LiveCreateCtrl_Entities.obj
 0002:00002038       ??_C@_0BE@KJPNLNKK@Delete?5entity?5id?5?$CFd?$AA@ 0000000037521038     LiveCreateCtrl_Entities.obj
 0002:00002050       ??_C@_0CE@JBAIKDCE@?$FLEntity?$FN?5Doing?5entities?5deletion@ 0000000037521050     LiveCreateCtrl_Entities.obj
 0002:00002078       ??_C@_0BP@LCFCMIJN@?$FLEntity?$FN?5Entity?5props?5were?5set?$AA@ 0000000037521078     LiveCreateCtrl_Entities.obj
 0002:00002098       ??_C@_0CE@PIIHPLFB@?$FLEntity?$FN?5Loading?5?$CFd?5ents?5props?5s@ 0000000037521098     LiveCreateCtrl_Entities.obj
 0002:000020c0       ??_C@_0CD@EFAGLFGD@Set?5entity?5props?5for?5id?3?$CFd?5Xml?$CI?$CF@ 00000000375210c0     LiveCreateCtrl_Entities.obj
 0002:000020e8       ??_C@_08BLPBAEMP@EntityId?$AA@ 00000000375210e8     LiveCreateCtrl_Entities.obj
 0002:000020f8       ??_C@_0DD@BFAGDKNP@?$FLEntity?$FN?5Parsing?5entities?5proper@ 00000000375210f8     LiveCreateCtrl_Entities.obj
 0002:00002130       ??_C@_0DA@BEIPKBDJ@?$FLEntity?$FN?5Doing?5entities?5property@ 0000000037521130     LiveCreateCtrl_Entities.obj
 0002:00002160       ??_C@_0CM@GIAICLCL@?$FLEntity?$FN?5Entity?5transform?5was?5se@ 0000000037521160     LiveCreateCtrl_Entities.obj
 0002:00002190       ??_C@_0EC@DIMHAPAD@Set?5entity?5xform?5for?5id?3?$CFd?5P?$CI?$CFf?5@ 0000000037521190     LiveCreateCtrl_Entities.obj
 0002:000021d8       ??_C@_0CL@CAEEKBH@?$FLEntity?$FN?5Could?5not?5find?5entity?5w@ 00000000375211d8     LiveCreateCtrl_Entities.obj
 0002:00002208       ??_C@_0CF@BOGAGOBL@?$FLEntity?$FN?5Doing?5entities?5transfor@ 0000000037521208     LiveCreateCtrl_Entities.obj
 0002:00002230       ??_C@_0BG@MLLKANMC@Delete?5entity?3?5id?$CI?$CFd?$CJ?$AA@ 0000000037521230     LiveCreateCtrl_Entities.obj
 0002:00002248       ??_C@_0BB@FAIIKBDL@entities_deleted?$AA@ 0000000037521248     LiveCreateCtrl_Entities.obj
 0002:00002260       ??_C@_0CC@FPHDINDN@Adding?5entity?5properties?3?5xml?$CI?$CFs@ 0000000037521260     LiveCreateCtrl_Entities.obj
 0002:00002288       ??_C@_0BE@BJHAALGF@entities_properties?$AA@ 0000000037521288     LiveCreateCtrl_Entities.obj
 0002:000022a0       ??_C@_0EC@DCNDDHFM@Adding?5entity?5xform?3?5id?3?$CFd?5P?$CI?$CFf?5@ 00000000375212a0     LiveCreateCtrl_Entities.obj
 0002:000022e8       ??_C@_0BD@OBOMKHAI@entities_transform?$AA@ 00000000375212e8     LiveCreateCtrl_Entities.obj
 0002:00002300       ??_C@_0BK@INGHJKHN@Recv?5deleted?5entity?5id?5?$CFd?$AA@ 0000000037521300     LiveCreateCtrl_Entities.obj
 0002:00002320       ??_C@_0CI@FIJLHFII@?$FLEntity?$FN?5Received?5?$CFd?5deleted?5ent@ 0000000037521320     LiveCreateCtrl_Entities.obj
 0002:00002348       ??_C@_0DH@EIEKMNBM@Recv?5entity?5props?3?5xml?5len?5?$CFd?0?5s@ 0000000037521348     LiveCreateCtrl_Entities.obj
 0002:00002380       ??_C@_0BB@KENKNNIE@Read?5xmlSize?3?5?$CFd?$AA@ 0000000037521380     LiveCreateCtrl_Entities.obj
 0002:00002398       ??_C@_0CG@MLKHKGHC@?$FLEntity?$FN?5Received?5?$CFd?5entity?5prop@ 0000000037521398     LiveCreateCtrl_Entities.obj
 0002:000023c0       ??_C@_0EA@MAMLJDIK@Recv?5entity?5xform?3?5id?3?$CFd?5P?$CI?$CFf?5?$CFf@ 00000000375213c0     LiveCreateCtrl_Entities.obj
 0002:00002400       ??_C@_0CH@JDLNLPIP@?$FLEntity?$FN?5Received?5?$CFd?5entity?5tran@ 0000000037521400     LiveCreateCtrl_Entities.obj
 0002:00002428       ??_C@_0BF@LIJACADB@ExecuteConsoleString?$AA@ 0000000037521428     LiveCreateCtrl_ExecuteConsoleString.obj
 0002:00002440       ??_C@_0BE@LMACFFID@exec_console_string?$AA@ 0000000037521440     LiveCreateCtrl_ExecuteConsoleString.obj
 0002:00002458       ??_C@_0CN@MBEKNENA@This?5controller?5executes?5command@ 0000000037521458     LiveCreateCtrl_ExecuteConsoleString.obj
 0002:00002488       ??_C@_0CB@IGBNKDJC@?$FLcmd?$FN?5Sending?5console?5string?$CI?$CFs?$CJ@ 0000000037521488     LiveCreateCtrl_ExecuteConsoleString.obj
 0002:000024b0       ??_7ExecuteConsoleStringController@LiveCreate@@6B@ 00000000375214b0     LiveCreateCtrl_ExecuteConsoleString.obj
 0002:00002538       ??_C@_0BH@PGIJIPOB@?$FLcmd?$FN?5Received?5cmd?$CI?$CFs?$CJ?$AA@ 0000000037521538     LiveCreateCtrl_ExecuteConsoleString.obj
 0002:00002550       ??_C@_0CA@LNBCALBA@?$FLcmd?$FN?5Exec?5console?5string?3?5?8?$CFs?8?$AA@ 0000000037521550     LiveCreateCtrl_ExecuteConsoleString.obj
 0002:00002570       ??_C@_0BB@OCMELCLO@FileChangeNotify?$AA@ 0000000037521570     LiveCreateCtrl_FileChangeNotify.obj
 0002:00002590       ??_C@_0EC@MHNJGALA@This?5controller?5notifies?5file?5ch@ 0000000037521590     LiveCreateCtrl_FileChangeNotify.obj
 0002:000025d8       ??_C@_0CE@GIDJBDJF@?$FLfilechange?$FN?5Sending?5filechange?$CI@ 00000000375215d8     LiveCreateCtrl_FileChangeNotify.obj
 0002:000025fc       ??_C@_01KMDKNFGN@?1?$AA@   00000000375215fc     LiveCreateCtrl_FileChangeNotify.obj
 0002:00002600       ??_7FileChangeNotifyController@LiveCreate@@6B@ 0000000037521600     LiveCreateCtrl_FileChangeNotify.obj
 0002:00002688       ??_C@_0BK@OEANLPOM@?$FLfilechange?$FN?5Reload?3?5?8?$CFs?8?$AA@ 0000000037521688     LiveCreateCtrl_FileChangeNotify.obj
 0002:000026a4       ??_C@_02JDPG@rb?$AA@       00000000375216a4     LiveCreateCtrl_FileChangeNotify.obj
 0002:000026a8       ??_C@_03INEHOLBK@mtl?$AA@  00000000375216a8     LiveCreateCtrl_FileChangeNotify.obj
 0002:000026b0       ??_C@_0CM@NFIIJKKD@?$FLfilechange?$FN?5File?5changed?3?5?8?$CFs?8?5@ 00000000375216b0     LiveCreateCtrl_FileChangeNotify.obj
 0002:000026e0       ??_C@_0BL@LAMAEDOK@?$FLfilechange?$FN?5Received?5?$CI?$CFs?$CJ?$AA@ 00000000375216e0     LiveCreateCtrl_FileChangeNotify.obj
 0002:00002700       ??_C@_0L@KKOCHHLN@Screenshot?$AA@ 0000000037521700     LiveCreateCtrl_Screenshot.obj
 0002:00002710       ??_C@_0L@CMHOPIGK@screenshot?$AA@ 0000000037521710     LiveCreateCtrl_Screenshot.obj
 0002:00002720       ??_C@_0EM@GBLPBLKG@This?5controller?5takes?5screenshot@ 0000000037521720     LiveCreateCtrl_Screenshot.obj
 0002:00002770       ??_C@_0CA@CJJPECAB@Screenshot?5is?5ready?5to?5be?5sent?4?$AA@ 0000000037521770     LiveCreateCtrl_Screenshot.obj
 0002:00002790       ??_C@_0CE@BKBOLMA@?$FLscreenshot?$FN?5Sending?5screenshot?$CI@ 0000000037521790     LiveCreateCtrl_Screenshot.obj
 0002:000027b8       ??_C@_0BJ@KOLJLNPB@Saved?5screenshot?5to?5?8?$CFs?8?$AA@ 00000000375217b8     LiveCreateCtrl_Screenshot.obj
 0002:000027d8       ??_C@_0CE@MDAKMPFD@user?1screenshots?1ScreenShot?$CF?44d?4@ 00000000375217d8     LiveCreateCtrl_Screenshot.obj
 0002:00002800       ??_C@_0BC@JHMNMMHA@r_getscreenshot?52?$AA@ 0000000037521800     LiveCreateCtrl_Screenshot.obj
 0002:00002818       ??_C@_0DO@CCJNPPDO@Cannot?5copy?5screenshot?5file?$CB?5Bad@ 0000000037521818     LiveCreateCtrl_Screenshot.obj
 0002:00002858       ??_C@_0CL@NIANLGEP@?$FLscreenshot?$FN?5Copy?5screen?5from?5?$CI?$CF@ 0000000037521858     LiveCreateCtrl_Screenshot.obj
 0002:00002888       ??_C@_0L@FMNOOCIE@?1app_home?1?$AA@ 0000000037521888     LiveCreateCtrl_Screenshot.obj
 0002:00002898       ??_C@_0BN@BADLHLEP@?$CFs_?$CFd?9?$CFd?9?$CFd__?$CFd_?$CFd_?$CFd_?$CFd?4tga?$AA@ 0000000037521898     LiveCreateCtrl_Screenshot.obj
 0002:000028b8       ??_C@_05LIDBDCIK@USER?2?$AA@ 00000000375218b8     LiveCreateCtrl_Screenshot.obj
 0002:000028c0       ??_C@_0BL@MCJDPJCM@?$FLscreenshot?$FN?5Received?5?$CI?$CFs?$CJ?$AA@ 00000000375218c0     LiveCreateCtrl_Screenshot.obj
 0002:000028e0       ??_7ScreenshotController@LiveCreate@@6B@ 00000000375218e0     LiveCreateCtrl_Screenshot.obj
 0002:00002968       ??_7CryRunnable@@6B@       0000000037521968     LiveCreateFileSync.obj
 0002:00002980       ??_C@_0BH@LGHILDHL@Runaway?5thread?5?$CFp?5?8?$CFs?8?$AA@ 0000000037521980     LiveCreateFileSync.obj
 0002:00002998       ??_7FileSyncManager@LiveCreate@@6BCrySimpleThreadSelf@@@ 0000000037521998     LiveCreateFileSync.obj
 0002:000029a0       ??_7FileSyncManager@LiveCreate@@6BCryRunnable@@@ 00000000375219a0     LiveCreateFileSync.obj
 0002:000029d0       ??_C@_0BJ@GFCDLFOH@Deleting?5temp?5file?3?5?8?$CFs?8?$AA@ 00000000375219d0     LiveCreateFileSync.obj
 0002:000029f0       ??_C@_0CF@GNKJNOLB@Copy?5?$CItarget?3?5?$CFs?5?$FL?$CFs?$FN?$CJ?3?5?8?$CFs?8?5to?5@ 00000000375219f0     LiveCreateFileSync.obj
 0002:00002a18       ??_C@_0CB@PAPOLKLE@Skipping?5platform?5?8?$CFs?8?5?$CI?$CFs?5only?$CJ@ 0000000037521a18     LiveCreateFileSync.obj
 0002:00002a40       ??_C@_0BE@MMMNAGJJ@LiveCreate_FileSync?$AA@ 0000000037521a40     LiveCreateFileSync.obj
 0002:00002a58       ??_C@_08IHFGNGMO@Editor?2?$CK?$AA@ 0000000037521a58     LiveCreateFileSync.obj
 0002:00002a68       ??_C@_08NBOBAAMH@Editor?1?$CK?$AA@ 0000000037521a68     LiveCreateFileSync.obj
 0002:00002a74       ??_C@_05KKOCDBFP@?$CK?4psd?$AA@ 0000000037521a74     LiveCreateFileSync.obj
 0002:00002a7c       ??_C@_05PBEEJEFO@?$CK?4max?$AA@ 0000000037521a7c     LiveCreateFileSync.obj
 0002:00002a84       ??_C@_05GAHOCCM@?$CK?4tif?$AA@ 0000000037521a84     LiveCreateFileSync.obj
 0002:00002a8c       ??_C@_05GIOEPHGE@?$CK?4bmp?$AA@ 0000000037521a8c     LiveCreateFileSync.obj
 0002:00002a94       ??_C@_05PKPOKHBI@?$CK?4bai?$AA@ 0000000037521a94     LiveCreateFileSync.obj
 0002:00002a9c       ??_C@_05MIMIMFJK@?$CK?4bak?$AA@ 0000000037521a9c     LiveCreateFileSync.obj
 0002:00002aa4       ??_C@_06GLOHMMNK@?$CK$tmp?$CK?$AA@ 0000000037521aa4     LiveCreateFileSync.obj
 0002:00002aac       ??_C@_06FEPPMCDC@?$CK?4tmp$?$AA@ 0000000037521aac     LiveCreateFileSync.obj
 0002:00002ab4       ??_C@_05BNJGPPCH@?$CK?4tmp?$AA@ 0000000037521ab4     LiveCreateFileSync.obj
 0002:00002abc       ??_C@_05BGOAMPAF@?$CK?4cry?$AA@ 0000000037521abc     LiveCreateFileSync.obj
 0002:00002ac4       ??_C@_05KBCCOJHJ@?$CK?4lyr?$AA@ 0000000037521ac4     LiveCreateFileSync.obj
 0002:00002ad0       ??_C@_0CB@KMLCFMIK@Deleting?5ignored?5temp?5file?3?5?8?$CFs?8@ 0000000037521ad0     LiveCreateFileSync.obj
 0002:00002af8       ??_C@_0BJ@FMJCDNF@Failed?5to?5create?5socket?4?$AA@ 0000000037521af8     LiveCreateNetSocket.obj
 0002:00002b18       ??_C@_0CC@KPDLIPBK@Failed?5to?5set?5TCP_NODELAY?5option@ 0000000037521b18     LiveCreateNetSocket.obj
 0002:00002b40       ??_C@_0DA@MOFGJACN@Failed?5to?5set?5socket?5to?5asynchro@ 0000000037521b40     LiveCreateNetSocket.obj
 0002:00002b70       ??_C@_0CD@GENCCHLH@Failed?5to?5set?5SO_REUSEADDR?5optio@ 0000000037521b70     LiveCreateNetSocket.obj
 0002:00002b98       ??_C@_0CA@ENMALPJE@Successfully?5bound?5socket?5to?5?$CFd?$AA@ 0000000037521b98     LiveCreateNetSocket.obj
 0002:00002bb8       ??_C@_0CO@ICEJELC@Could?5not?5bind?5socket?5to?5port?5?$CFd@ 0000000037521bb8     LiveCreateNetSocket.obj
 0002:00002be8       ??_C@_0DJ@MBPJPBPG@Cannot?5listen?5for?5incoming?5conne@ 0000000037521be8     LiveCreateNetSocket.obj
 0002:00002c28       ??_C@_0P@MGCLGBJJ@Socket?5closed?4?$AA@ 0000000037521c28     LiveCreateNetSocket.obj
 0002:00002c38       ??_C@_0BJ@JFCKEEOG@Get?5host?5by?5name?5failed?4?$AA@ 0000000037521c38     LiveCreateNetSocket.obj
 0002:00002c58       ??_C@_0CE@MFPKNILP@Error?5when?5getting?5local?5host?5na@ 0000000037521c58     LiveCreateNetSocket.obj
 0002:00002c80       ??_C@_0CA@KDPDNBOB@Successfully?5connected?5to?5?$CFs?3?$CFd?$AA@ 0000000037521c80     LiveCreateNetSocket.obj
 0002:00002ca0       ??_C@_0CD@NMDHPMLG@Failed?5to?5connect?0?5reason?5code?3?5@ 0000000037521ca0     LiveCreateNetSocket.obj
 0002:00002cc8       ??_C@_0BD@FHNMKEBB@Already?5connected?4?$AA@ 0000000037521cc8     LiveCreateNetSocket.obj
 0002:00002ce0       ??_C@_0O@HFCDDHBI@Is?5connected?4?$AA@ 0000000037521ce0     LiveCreateNetSocket.obj
 0002:00002cf0       ??_C@_0N@HMIINEON@Would?5block?4?$AA@ 0000000037521cf0     LiveCreateNetSocket.obj
 0002:00002d00       ??_C@_0BI@BPFBDIEN@Connecting?5to?5?$CFs?3?$CFd?5?4?4?4?$AA@ 0000000037521d00     LiveCreateNetSocket.obj
 0002:00002d18       ??_C@_0BH@FEJLNBAE@Reconnecting?5socket?4?4?4?$AA@ 0000000037521d18     LiveCreateNetSocket.obj
 0002:00002d30       ??_C@_0BN@JBKPGPJB@Validate?3?5We?5need?5reconnect?4?$AA@ 0000000037521d30     LiveCreateNetSocket.obj
 0002:00002d50       ??_C@_0DF@HHMDKJIL@Validate?3?5Failed?5to?5select?5socke@ 0000000037521d50     LiveCreateNetSocket.obj
 0002:00002d88       ??_C@_0BI@BJNPHCCD@Validate?3?5Is?5connected?4?$AA@ 0000000037521d88     LiveCreateNetSocket.obj
 0002:00002da0       ??_C@_0CP@HLACFNGF@Validate?3?5Failed?5to?5select?5socke@ 0000000037521da0     LiveCreateNetSocket.obj
 0002:00002dd0       ??_C@_0EF@EEAAJNCO@Failed?5to?5select?5socket?5when?5che@ 0000000037521dd0     LiveCreateNetSocket.obj
 0002:00002e18       ??_C@_0CF@KBLBLBKK@Send?3?5Failed?5to?5send?4?5Not?5connec@ 0000000037521e18     LiveCreateNetSocket.obj
 0002:00002e40       ??_C@_0CB@EIJHBAAJ@Send?3?5Failed?5to?5send?0?5reason?3?5?$CFd@ 0000000037521e40     LiveCreateNetSocket.obj
 0002:00002e68       ??_C@_0BC@OPNFDKPA@Failed?5to?5receive?$AA@ 0000000037521e68     LiveCreateNetSocket.obj
 0002:00002e80       ??_C@_0CO@FAIPGMF@recv?3?5failed?5to?5receive?5package?4@ 0000000037521e80     LiveCreateNetSocket.obj
 0002:00002eb0       ??_C@_0DL@MMAMGGMI@recv?3?5failed?5to?5receive?5package?4@ 0000000037521eb0     LiveCreateNetSocket.obj
 0002:00002ef0       ??_7INetSocketObserver@LiveCreate@@6B@ 0000000037521ef0     LiveCreateNetwork.obj
 0002:00002f00       ??_C@_0CL@FFDEGLBC@Connection?5did?5not?5succeeded?5for@ 0000000037521f00     LiveCreateNetwork.obj
 0002:00002f30       ??_C@_0BP@PBLIDAIA@OnPeerConnected?3?5Peer?5is?5NULL?$CB?$AA@ 0000000037521f30     LiveCreateNetwork.obj
 0002:00002f50       ??_C@_0CI@EGHNCDCC@OnPeerConnected?3?5Peer?5connected?5@ 0000000037521f50     LiveCreateNetwork.obj
 0002:00002f78       ??_C@_0DE@LEHOJCFB@OnPeerDisconnected?3?5Disconnectin@ 0000000037521f78     LiveCreateNetwork.obj
 0002:00002fb0       ??_C@_08FOJKHHJA@?$CFd?4?$CFd?4?$CFd?$AA@ 0000000037521fb0     LiveCreateNetwork.obj
 0002:00002fc0       ??_C@_0CB@FNJFGKDG@Peer?5comm?5thread?5already?5stopped@ 0000000037521fc0     LiveCreateNetwork.obj
 0002:00002fe8       ??_C@_0BN@LNJEMIJA@Peer?5scheduled?5for?5removing?4?$AA@ 0000000037521fe8     LiveCreateNetwork.obj
 0002:00003008       ??_C@_0BH@BBIHKAPI@Wait?5for?5thread?4?4?4?$CI?$CFp?$CJ?$AA@ 0000000037522008     LiveCreateNetwork.obj
 0002:00003020       ??_C@_0CA@NHBPPCPB@Stopping?5peer?5connection?4?4?4?$CI?$CFp?$CJ?$AA@ 0000000037522020     LiveCreateNetwork.obj
 0002:00003040       ??_7?$CrySimpleThread@VFileSyncManager@LiveCreate@@@@6BCrySimpleThreadSelf@@@ 0000000037522040     LiveCreateFileSync.obj
 0002:00003040       ??_7?$CrySimpleThread@VNetPeerCommThread@LiveCreate@@@@6BCrySimpleThreadSelf@@@ 0000000037522040     LiveCreateNetwork.obj
 0002:00003040       ??_7?$CrySimpleThread@VNetPeerServerAcceptThread@LiveCreate@@@@6BCrySimpleThreadSelf@@@ 0000000037522040     LiveCreateNetwork.obj
 0002:00003048       ??_7?$CrySimpleThread@VNetPeerServerAcceptThread@LiveCreate@@@@6BCryRunnable@@@ 0000000037522048     LiveCreateNetwork.obj
 0002:00003048       ??_7?$CrySimpleThread@VFileSyncManager@LiveCreate@@@@6BCryRunnable@@@ 0000000037522048     LiveCreateFileSync.obj
 0002:00003048       ??_7?$CrySimpleThread@VNetPeerCommThread@LiveCreate@@@@6BCryRunnable@@@ 0000000037522048     LiveCreateNetwork.obj
 0002:00003078       ??_7?$CryThread@VNetPeerCommThread@LiveCreate@@@@6BCrySimpleThreadSelf@@@ 0000000037522078     LiveCreateNetwork.obj
 0002:00003078       ??_7?$CryThread@VNetPeerServerAcceptThread@LiveCreate@@@@6BCrySimpleThreadSelf@@@ 0000000037522078     LiveCreateNetwork.obj
 0002:00003078       ??_7?$CryThread@VFileSyncManager@LiveCreate@@@@6BCrySimpleThreadSelf@@@ 0000000037522078     LiveCreateFileSync.obj
 0002:00003080       ??_7?$CryThread@VNetPeerServerAcceptThread@LiveCreate@@@@6BCryRunnable@@@ 0000000037522080     LiveCreateNetwork.obj
 0002:00003080       ??_7?$CryThread@VNetPeerCommThread@LiveCreate@@@@6BCryRunnable@@@ 0000000037522080     LiveCreateNetwork.obj
 0002:00003080       ??_7?$CryThread@VFileSyncManager@LiveCreate@@@@6BCryRunnable@@@ 0000000037522080     LiveCreateFileSync.obj
 0002:000030b0       ??_C@_0BC@EKNPFJEB@Deleting?5peer?3?5?$CFs?$AA@ 00000000375220b0     LiveCreateNetwork.obj
 0002:000030d0       ??_C@_0FL@HGMMGPJN@Sending?5peer?5info?3?5platform?3?5?8?$CFs@ 00000000375220d0     LiveCreateNetwork.obj
 0002:00003130       ??_7NetPeerCommThread@LiveCreate@@6B@ 0000000037522130     LiveCreateNetwork.obj
 0002:00003140       ??_7NetPeerCommThread@LiveCreate@@6BCrySimpleThreadSelf@@@ 0000000037522140     LiveCreateNetwork.obj
 0002:00003148       ??_7NetPeerCommThread@LiveCreate@@6BCryRunnable@@@ 0000000037522148     LiveCreateNetwork.obj
 0002:00003178       ??_7NetPeer@LiveCreate@@6B@ 0000000037522178     LiveCreateNetwork.obj
 0002:00003180       ??_C@_0DH@NHIPDDH@No?5success?5on?5create?5and?5connect@ 0000000037522180     LiveCreateNetwork.obj
 0002:000031b8       ??_C@_0BC@LLIMECND@ConnectToPeer?3?5?$CFs?$AA@ 00000000375221b8     LiveCreateNetwork.obj
 0002:000031d0       ??_C@_0DI@CHEODAIP@Received?5accept?5request?5from?5?8?$CFs@ 00000000375221d0     LiveCreateNetwork.obj
 0002:00003208       ??_C@_0DK@DICDBION@Peer?5accepted?0?5initiating?5server@ 0000000037522208     LiveCreateNetwork.obj
 0002:00003248       ??_C@_0CI@OJJMNGI@Cannot?5accept?5a?5connection?5from?5@ 0000000037522248     LiveCreateNetwork.obj
 0002:00003270       ??_7NetPeerServerAcceptThread@LiveCreate@@6BCryRunnable@@@ 0000000037522270     LiveCreateNetwork.obj
 0002:000032a0       ??_7NetPeerServerAcceptThread@LiveCreate@@6BCrySimpleThreadSelf@@@ 00000000375222a0     LiveCreateNetwork.obj
 0002:000032a8       ??_C@_0BM@GBDIAICF@Accept?5peers?5thread?5closed?4?$AA@ 00000000375222a8     LiveCreateNetwork.obj
 0002:000032c8       ??_C@_0BL@EPEKIFMC@Listening?5on?5server?5socket?$AA@ 00000000375222c8     LiveCreateNetwork.obj
 0002:000032e8       ??_C@_0BP@DLKNLFFJ@Cannot?5listen?5on?5server?5socket?$AA@ 00000000375222e8     LiveCreateNetwork.obj
 0002:00003308       ??_C@_0CM@DPDPEHPL@Cannot?5bind?5server?5listen?5socket@ 0000000037522308     LiveCreateNetwork.obj
 0002:00003338       ??_C@_0CD@JJIKECGD@Cannot?5create?5server?5listen?5sock@ 0000000037522338     LiveCreateNetwork.obj
 0002:00003360       ??_C@_0BC@KGFBLBGL@LiveCreate_Server?$AA@ 0000000037522360     LiveCreateNetwork.obj
 0002:00003378       ??_C@_0BG@MONAJOJG@OnSocketConnected?5end?$AA@ 0000000037522378     LiveCreateNetwork.obj
 0002:00003390       ??_C@_0BJ@MAEJCDB@OnSocketConnected?5called?$AA@ 0000000037522390     LiveCreateNetwork.obj
 0002:000033b0       ??_C@_0BC@JJNJGKEE@Ended?5comm?5thread?$AA@ 00000000375223b0     LiveCreateNetwork.obj
 0002:000033c8       ??_C@_0CP@MNEFJKJA@Tried?5to?5send?5data?5of?5size?5?$CFd?5bu@ 00000000375223c8     LiveCreateNetwork.obj
 0002:000033f8       ??_C@_0CG@LAJJJCED@Sending?5message?5data?5size?5of?5?$CFd?5@ 00000000375223f8     LiveCreateNetwork.obj
 0002:00003420       ??_C@_0CE@PKJJIOCC@Sent?5header?5of?5size?5?$CFd?5?$CImust?5be?5@ 0000000037522420     LiveCreateNetwork.obj
 0002:00003450       ??_C@_0FE@CHIEANIL@Sending?5message?5header?5from?5send@ 0000000037522450     LiveCreateNetwork.obj
 0002:000034a8       ??_C@_0DC@FIBEKAB@Pushing?5new?5message?5to?5received?5@ 00000000375224a8     LiveCreateNetwork.obj
 0002:000034e0       ??_C@_0CP@MOMNFJDO@Could?5not?5allocate?5memory?5for?5me@ 00000000375224e0     LiveCreateNetwork.obj
 0002:00003510       ??_C@_0CL@FLPPDIEF@Received?5msg?5data?5of?5size?5?$CFd?$CB?5?$CIm@ 0000000037522510     LiveCreateNetwork.obj
 0002:00003540       ??_C@_0CA@NBJLICGK@Receiving?5message?5data?5?$CFd?5bytes?$AA@ 0000000037522540     LiveCreateNetwork.obj
 0002:00003560       ??_C@_0EO@FBKNNBPG@Got?5message?5header?5from?5peer?5han@ 0000000037522560     LiveCreateNetwork.obj
 0002:000035b0       ??_C@_0DC@DGOHMJDN@Received?5msg?5header?5data?5of?5size@ 00000000375225b0     LiveCreateNetwork.obj
 0002:000035e8       ??_C@_0CB@MDGLNBAN@Receiving?5from?5peer?5handle?5?$CFd?4?4?4@ 00000000375225e8     LiveCreateNetwork.obj
 0002:00003610       ??_C@_0DF@JCBCKAOO@Started?5peer?5communication?5threa@ 0000000037522610     LiveCreateNetwork.obj
 0002:00003648       ??_C@_0BE@EGKEFDML@LiveCreate_PeerComm?$AA@ 0000000037522648     LiveCreateNetwork.obj
 0002:00003660       ??_7IPlatformHandler@LiveCreate@@6B@ 0000000037522660     PlatformHandlerBase.obj
 0002:00003740       ??_C@_0CC@DHGOLEGJ@?$FLLC?$FN?5Set?5info?5?8?$CFs?8?5?8?$CFs?8?5?8?$CFs?8?5?8?$CFs@ 0000000037522740     PlatformHandlerBase.obj
 0002:00003770       ??_7PlatformHandlerBase@LiveCreate@@6B@ 0000000037522770     PlatformHandlerBase.obj
 0002:00003850       ??_C@_0M@GGNMBBGG@AssetBranch?$AA@ 0000000037522850     PlatformHandlerBase.obj
 0002:00003860       ??_C@_0L@GPNKJCPG@CodeBranch?$AA@ 0000000037522860     PlatformHandlerBase.obj
 0002:00003870       ??_C@_0BA@DECOJOPE@AssetChangelist?$AA@ 0000000037522870     PlatformHandlerBase.obj
 0002:00003880       ??_C@_0P@EFJLMFKL@CodeChangelist?$AA@ 0000000037522880     PlatformHandlerBase.obj
 0002:00003890       ??_C@_0BA@BEPPBH@BuildChangelist?$AA@ 0000000037522890     PlatformHandlerBase.obj
 0002:000038a0       ??_C@_0BI@DPHLIOHO@?$CFhd?1?$CFhd?1?$CFhd?3?$CFhd?3?$CFhd?3?$CFhd?$AA@ 00000000375228a0     PlatformHandlerBase.obj
 0002:000038b8       ??_C@_09PPOBAANA@BuildTime?$AA@ 00000000375228b8     PlatformHandlerBase.obj
 0002:000038c8       ??_C@_09BAAFKHBM@BuildName?$AA@ 00000000375228c8     PlatformHandlerBase.obj
 0002:000038d8       ??_C@_0M@PIEABBJI@BuildNumber?$AA@ 00000000375228d8     PlatformHandlerBase.obj
 0002:000038e8       ??_C@_0BM@GODNEFOE@Found?5build?5info?3?5?8?$CFs?8?$DN?8?$CFs?8?$AA@ 00000000375228e8     PlatformHandlerBase.obj
 0002:00003904       ??_C@_01NEMOKFLO@?$DN?$AA@ 0000000037522904     PlatformHandlerBase.obj
 0002:00003908       ??_C@_01EEMJAFIK@?6?$AA@   0000000037522908     PlatformHandlerBase.obj
 0002:00003910       ??_7PlatformHandler_GamePC@LiveCreate@@6B@ 0000000037522910     PlatformHandler_GamePC.obj
 0002:00003910       ??_7PlatformHandler_EditorPC@LiveCreate@@6B@ 0000000037522910     PlatformHandler_EditorPC.obj
 0002:000039f0       ??_7PlatformHandler_PS3@LiveCreate@@6B@ 00000000375229f0     PlatformHandler_PS3.obj
 0002:00003ad0       ??_C@_0O@LKOBEIKN@PS3?5Entry?3?5?$CFs?$AA@ 0000000037522ad0     PlatformHandler_PS3.obj
 0002:00003ae0       ??_C@_0CG@JMHAEBPP@?$FLLiveCreate?$FN?5Initializing?5PS3?5De@ 0000000037522ae0     PlatformHandler_PS3.obj
 0002:00003b10       ??_C@_0HM@HENNEAAI@?$FLLiveCreate?$FN?5Could?5not?5initializ@ 0000000037522b10     PlatformHandler_PS3.obj
 0002:00003b90       ??_7PlatformHandlerFactory_PS3@LiveCreate@@6B@ 0000000037522b90     PlatformHandler_PS3.obj
 0002:00003bb8       ??_C@_0CC@FJICKMOF@?$FLLC?$FN?5Cannot?5connect?5to?5target?3?5?$CF@ 0000000037522bb8     PlatformHandler_PS3.obj
 0002:00003be0       ??_C@_0DK@LIMDLHBC@Found?5?$CFd?5PS3?5consoles?5registered@ 0000000037522be0     PlatformHandler_PS3.obj
 0002:00003c20       ??_C@_0DO@KIAOJNCE@Discovered?5PS3?5console?3?5?$CFs?5with?5@ 0000000037522c20     PlatformHandler_PS3.obj
 0002:00003c60       ??_C@_0M@OAJHAIPD@Entries?3?5?$CFd?$AA@ 0000000037522c60     PlatformHandler_PS3.obj
 0002:00003c70       ??_C@_0O@EAEOJDKL@Begin?5scan?5?$CFs?$AA@ 0000000037522c70     PlatformHandler_PS3.obj
 0002:00003c80       ??_C@_0BE@GMNCKEIJ@Created?5PS3?5dir?3?5?$CFs?$AA@ 0000000037522c80     PlatformHandler_PS3.obj
 0002:00003c98       ??_C@_0DD@GNBDBNP@Cannot?5create?5PS3?5dir?3?5?$CFs?0?5error@ 0000000037522c98     PlatformHandler_PS3.obj
 0002:00003cd0       ??_C@_0M@JDDILGDP@End?5scan?5?$CFs?$AA@ 0000000037522cd0     PlatformHandler_PS3.obj
 0002:00003ce0       ??_C@_0BC@LIMHDPOP@Cannot?5parse?5?8?$CFs?8?$AA@ 0000000037522ce0     PlatformHandler_PS3.obj
 0002:00003cf8       ??_C@_0O@DDPIGMKO@BuildInfo?4txt?$AA@ 0000000037522cf8     PlatformHandler_PS3.obj
 0002:00003d08       ??_C@_0P@IOPMPLNM@Cannot?5scan?5?$CFs?$AA@ 0000000037522d08     PlatformHandler_PS3.obj
 0002:00003d18       ??_C@_0BJ@HAPGHECA@Launching?5game?3?5?$CFs?5?$CFs?5?$CFs?$AA@ 0000000037522d18     PlatformHandler_X360.obj
 0002:00003d40       ??_7PlatformHandler_X360@LiveCreate@@6B@ 0000000037522d40     PlatformHandler_X360.obj
 0002:00003e20       ??_C@_09CJFJMKEK@CopyTo?5?$CFs?$AA@ 0000000037522e20     PlatformHandler_X360.obj
 0002:00003e2c       ??_C@_02HDBGODGB@?2?2?$AA@ 0000000037522e2c     PlatformHandler_X360.obj
 0002:00003e30       ??_C@_01KICIPPFI@?2?$AA@   0000000037522e30     PlatformHandler_X360.obj
 0002:00003e38       ??_C@_0BG@BOANFGAO@CopyFrom?5?8?$CFs?8?5to?5?8?$CFs?8?$AA@ 0000000037522e38     PlatformHandler_X360.obj
 0002:00003e50       ??_C@_0BA@GPMKPMHG@Adding?5exe?5?8?$CFs?8?$AA@ 0000000037522e50     PlatformHandler_X360.obj
 0002:00003e60       ??_C@_0CJ@GIOKFDEN@Failed?5to?5open?3?5?$CFs?5file?5in?5the?5?$CF@ 0000000037522e60     PlatformHandler_X360.obj
 0002:00003e8c       ??_C@_03NJMKFCKF@xex?$AA@  0000000037522e8c     PlatformHandler_X360.obj
 0002:00003e90       ??_C@_09POLAKCBN@Entry?3?5?$CFs?$AA@ 0000000037522e90     PlatformHandler_X360.obj
 0002:00003e9c       ??_C@_04MDHFNGMD@xe?3?2?$AA@ 0000000037522e9c     PlatformHandler_X360.obj
 0002:00003ea8       ??_C@_08EJOALOPG@xbdm?4dll?$AA@ 0000000037522ea8     PlatformHandler_X360.obj
 0002:00003eb8       ??_C@_09ILCHEPKO@?2bin?2x64?2?$AA@ 0000000037522eb8     PlatformHandler_X360.obj
 0002:00003ec4       ??_C@_04PJGKJHDF@XEDK?$AA@ 0000000037522ec4     PlatformHandler_X360.obj
 0002:00003ed0       ??_7PlatformHandlerFactory_X360@LiveCreate@@6B@ 0000000037522ed0     PlatformHandler_X360.obj
 0002:00003f00       __sz_xbdm_DLL              0000000037522f00     xbdm:xbdm.DLL
 0002:00003f10       _pRawDllMain               0000000037522f10     MSVCRT:crtdll.obj
 0002:00003f10       _pDefaultRawDllMain        0000000037522f10     MSVCRT:crtdll.obj
 0002:00003f28       ??_C@_00CNPNBAHC@?$AA@     0000000037522f28     PS3TmHelperLib:PS3TmHelper.obj
 0002:00003f30       ??_C@_07OHKHACFK@0?40?40?40?$AA@ 0000000037522f30     PS3TmHelperLib:PS3TmHelper.obj
 0002:00003f38       ??_C@_0BK@JNJLPKIF@PS3TM?5notify?3?5Progress?5?$CFd?$AA@ 0000000037522f38     PS3TmHelperLib:PS3TmHelper.obj
 0002:00003f58       ??_C@_0BK@HOFLIKPA@PS3TM?5notify?3?5Finished?5?$CFd?$AA@ 0000000037522f58     PS3TmHelperLib:PS3TmHelper.obj
 0002:00003f78       ??_C@_0BG@BPDDGKNH@PS3TM?5notify?3?5Skipped?$AA@ 0000000037522f78     PS3TmHelperLib:PS3TmHelper.obj
 0002:00003f90       ??_C@_0BE@KNOPDBJB@PS3TM?5notify?3?5Error?$AA@ 0000000037522f90     PS3TmHelperLib:PS3TmHelper.obj
 0002:00003fa4       ??_C@_05MBDEGLCK@ERROR?$AA@ 0000000037522fa4     PS3TmHelperLib:PS3TmHelper.obj
 0002:00003fb0       ??_C@_0BB@PKDENBIC@INVALID_INSTANCE?$AA@ 0000000037522fb0     PS3TmHelperLib:PS3TmHelper.obj
 0002:00003fc8       ??_C@_0P@FCKDAKFC@INVALID_TARGET?$AA@ 0000000037522fc8     PS3TmHelperLib:PS3TmHelper.obj
 0002:00003fd8       ??_C@_0BB@LPLMBNBB@INVALID_GAMEPORT?$AA@ 0000000037522fd8     PS3TmHelperLib:PS3TmHelper.obj
 0002:00003ff0       ??_C@_0M@PCENNPGA@?$CFd?4?$CFd?4?$CFd?4?$CFd?$AA@ 0000000037522ff0     PS3TmHelperLib:PS3TmHelper.obj
 0002:00004000       ??_C@_0BD@NJMIMGEP@Could?5not?5scan?5dir?$AA@ 0000000037523000     PS3TmHelperLib:PS3TmHelper.obj
 0002:00004018       ??_C@_0BA@DOAKOOEK@ps3tmapix64?4dll?$AA@ 0000000037523018     PS3TmHelperLib:PS3TmDynApi.obj
 0002:00004028       ??_C@_0BD@IGNCBFMM@SNPS3GetTargetInfo?$AA@ 0000000037523028     PS3TmHelperLib:PS3TmDynApi.obj
 0002:00004040       ??_C@_0BF@ODKOBHGL@SNPS3InitTargetComms?$AA@ 0000000037523040     PS3TmHelperLib:PS3TmDynApi.obj
 0002:00004058       ??_C@_0BI@CCKNFGFN@SNPS3EnumerateTargetsEx?$AA@ 0000000037523058     PS3TmHelperLib:PS3TmDynApi.obj
 0002:00004070       ??_C@_0BG@GDOJLPJK@SNPS3CloseTargetComms?$AA@ 0000000037523070     PS3TmHelperLib:PS3TmDynApi.obj
 0002:00004088       ??_C@_0BG@BOFCLGEK@SNPS3GetDirectoryList?$AA@ 0000000037523088     PS3TmHelperLib:PS3TmDynApi.obj
 0002:000040a0       ??_C@_0BB@OPOJDHIG@SNPS3ProcessLoad?$AA@ 00000000375230a0     PS3TmHelperLib:PS3TmDynApi.obj
 0002:000040b8       ??_C@_0N@GDJCAKOK@SNPS3Connect?$AA@ 00000000375230b8     PS3TmHelperLib:PS3TmDynApi.obj
 0002:000040c8       ??_C@_0BN@MLGMKKEC@SNPS3RegisterTTYEventHandler?$AA@ 00000000375230c8     PS3TmHelperLib:PS3TmDynApi.obj
 0002:000040e8       ??_C@_0BN@ELNEOPP@SNPS3RegisterFTPEventHandler?$AA@ 00000000375230e8     PS3TmHelperLib:PS3TmDynApi.obj
 0002:00004108       ??_C@_0BA@JNLAJHMN@SNPS3Disconnect?$AA@ 0000000037523108     PS3TmHelperLib:PS3TmDynApi.obj
 0002:00004118       ??_C@_0BD@PJMMKGLL@SNPS3SetTargetInfo?$AA@ 0000000037523118     PS3TmHelperLib:PS3TmDynApi.obj
 0002:00004130       ??_C@_0L@KJHGCDDD@SNPS3Reset?$AA@ 0000000037523130     PS3TmHelperLib:PS3TmDynApi.obj
 0002:00004140       ??_C@_0N@MHLLABOB@SNPS3ResetEx?$AA@ 0000000037523140     PS3TmHelperLib:PS3TmDynApi.obj
 0002:00004150       ??_C@_0M@EBENCBHA@SNPS3Delete?$AA@ 0000000037523150     PS3TmHelperLib:PS3TmDynApi.obj
 0002:00004160       ??_C@_0BC@IAADHCAB@SNPS3DownloadFile?$AA@ 0000000037523160     PS3TmHelperLib:PS3TmDynApi.obj
 0002:00004178       ??_C@_0BD@EIOHPPON@SNPS3MakeDirectory?$AA@ 0000000037523178     PS3TmHelperLib:PS3TmDynApi.obj
 0002:00004190       ??_C@_0BA@BPODFJGA@SNPS3UploadFile?$AA@ 0000000037523190     PS3TmHelperLib:PS3TmDynApi.obj
 0002:000041a0       ??_C@_09DIGGBBHM@SNPS3Kick?$AA@ 00000000375231a0     PS3TmHelperLib:PS3TmDynApi.obj
 0002:000041b0       ??_C@_0BF@BOMMHPA@SNPS3CancelFTPEvents?$AA@ 00000000375231b0     PS3TmHelperLib:PS3TmDynApi.obj
 0002:000041c8       ??_C@_0BF@DNPIINAO@SNPS3CancelTTYEvents?$AA@ 00000000375231c8     PS3TmHelperLib:PS3TmDynApi.obj
 0002:000041e0       ??_C@_0BE@KCJIIADA@SNPS3GetPowerStatus?$AA@ 00000000375231e0     PS3TmHelperLib:PS3TmDynApi.obj
 0002:000041f8       ??_C@_0BG@BAJNDJJI@SNPS3GetConnectStatus?$AA@ 00000000375231f8     PS3TmHelperLib:PS3TmDynApi.obj
 0002:00004210       ??_C@_0BB@JPOCANBF@SNPS3ProcessList?$AA@ 0000000037523210     PS3TmHelperLib:PS3TmDynApi.obj
 0002:00004228       ??_C@_0BB@HJAOBANN@SNPS3ProcessInfo?$AA@ 0000000037523228     PS3TmHelperLib:PS3TmDynApi.obj
 0002:00004240       ??_C@_0BL@GGNNEPLN@SNPS3GetGamePortIPAddrData?$AA@ 0000000037523240     PS3TmHelperLib:PS3TmDynApi.obj
 0002:00004260       ??_C@_0CA@KNHGKIJ@SNPS3GetGamePortDebugIPAddrData?$AA@ 0000000037523260     PS3TmHelperLib:PS3TmDynApi.obj
 0002:00004280       ??_C@_0BH@FIGHAJEB@SNPS3GetConnectionInfo?$AA@ 0000000037523280     PS3TmHelperLib:PS3TmDynApi.obj
 0002:00004298       ??_C@_0BB@JJMOPHEC@SNPS3SetTimeouts?$AA@ 0000000037523298     PS3TmHelperLib:PS3TmDynApi.obj
 0002:000042b0       ??_C@_0BH@DKKDHIPI@SNPS3EnableVRAMCapture?$AA@ 00000000375232b0     PS3TmHelperLib:PS3TmDynApi.obj
 0002:000042c8       ??_C@_0BB@HNKNILKP@SNPS3VRAMCapture?$AA@ 00000000375232c8     PS3TmHelperLib:PS3TmDynApi.obj
 0002:000042e0       ??_C@_0BI@LJCDBDLB@SNPS3GetDirectoryListEx?$AA@ 00000000375232e0     PS3TmHelperLib:PS3TmDynApi.obj
 0002:00004350       __rtc_iaa                  0000000037523350     MSVCRT:_initsect_.obj
 0002:00004358       __rtc_izz                  0000000037523358     MSVCRT:_initsect_.obj
 0002:00004360       __rtc_taa                  0000000037523360     MSVCRT:_initsect_.obj
 0002:00004368       __rtc_tzz                  0000000037523368     MSVCRT:_initsect_.obj
 0002:00005e5c       __DELAY_IMPORT_DESCRIPTOR_xbdm_DLL 0000000037524e5c     xbdm:xbdm.DLL
 0002:00005e7c       __NULL_DELAY_IMPORT_DESCRIPTOR 0000000037524e7c     xbdm:xbdm.DLL
 0002:00005f10       \177xbdm_NULL_THUNK_DATA_DLN 0000000037524f10     xbdm:xbdm.DLL
 0002:00006008       \177xbdm_NULL_THUNK_DATA_DLB 0000000037525008     xbdm:xbdm.DLL
 0002:00006078       __IMPORT_DESCRIPTOR_KERNEL32 0000000037525078     kernel32:KERNEL32.dll
 0002:0000608c       __IMPORT_DESCRIPTOR_USER32 000000003752508c     user32:USER32.dll
 0002:000060a0       __IMPORT_DESCRIPTOR_WS2_32 00000000375250a0     Ws2_32:WS2_32.dll
 0002:000060b4       __IMPORT_DESCRIPTOR_MSVCR100 00000000375250b4     MSVCRT:MSVCR100.dll
 0002:000060c8       __NULL_IMPORT_DESCRIPTOR   00000000375250c8     kernel32:KERNEL32.dll
 0003:00000010       ?m_seed@CLCGRndGen@@0_KA   0000000037526010     CryLiveCreate.obj
 0003:00000020       ?sEmptyStringBuffer@?1??_emptyHeader@?$CryStringT@D@@KAPEAUStrHeader@2@XZ@4PAU32@A 0000000037526020     CryLiveCreate.obj
 0003:00000068       ?s_testNullImplCompile@LiveCreate@@3VCNullManager@1@A 0000000037526068     LiveCreate.obj
 0003:00000188       ?fVec3_Zero@?$Vec3Constants@M@@2U?$Vec3_tpl@M@@B 0000000037526188     StdAfx.obj
 0003:00000198       ?fVec3_One@?$Vec3Constants@M@@2U?$Vec3_tpl@M@@B 0000000037526198     StdAfx.obj
 0003:000001a8       ?fVec2_Zero@?$Vec2Constants@M@@2U?$Vec2_tpl@M@@A 00000000375261a8     StdAfx.obj
 0003:000001b0       ?fVec2_OneX@?$Vec2Constants@M@@2U?$Vec2_tpl@M@@A 00000000375261b0     StdAfx.obj
 0003:000001b8       ?fVec2_OneY@?$Vec2Constants@M@@2U?$Vec2_tpl@M@@A 00000000375261b8     StdAfx.obj
 0003:000001c0       ?fVec2_One@?$Vec2Constants@M@@2U?$Vec2_tpl@M@@A 00000000375261c0     StdAfx.obj
 0003:000001c8       _fltused                   00000000375261c8     MSVCRT:dllsupp.obj
 0003:000001d0       __native_dllmain_reason    00000000375261d0     MSVCRT:natstart.obj
 0003:000001d4       __native_vcclrit_reason    00000000375261d4     MSVCRT:natstart.obj
 0003:000001d8       __security_cookie          00000000375261d8     MSVCRT:gs_cookie.obj
 0003:000001e0       __security_cookie_complement 00000000375261e0     MSVCRT:gs_cookie.obj
 0003:000001e8       __imp_DmGetAltAddress      00000000375261e8     xbdm:xbdm.DLL
 0003:000001f0       __imp_DmGetXboxName        00000000375261f0     xbdm:xbdm.DLL
 0003:000001f8       __imp_DmSetXboxNameNoRegister 00000000375261f8     xbdm:xbdm.DLL
 0003:00000200       __imp_DmReboot             0000000037526200     xbdm:xbdm.DLL
 0003:00000208       __imp_DmSetTitleEx         0000000037526208     xbdm:xbdm.DLL
 0003:00000210       __imp_DmDeleteFile         0000000037526210     xbdm:xbdm.DLL
 0003:00000218       __imp_DmGetFileAttributes  0000000037526218     xbdm:xbdm.DLL
 0003:00000220       __imp_DmGetSystemTime      0000000037526220     xbdm:xbdm.DLL
 0003:00000228       __imp_DmWalkDir            0000000037526228     xbdm:xbdm.DLL
 0003:00000230       __imp_DmCloseDir           0000000037526230     xbdm:xbdm.DLL
 0003:00000238       __imp_DmSendFileA          0000000037526238     xbdm:xbdm.DLL
 0003:00000240       __imp_DmMkdir              0000000037526240     xbdm:xbdm.DLL
 0003:00000248       __imp_DmReceiveFileA       0000000037526248     xbdm:xbdm.DLL
 0003:00000250       __imp_DmReadFilePartial    0000000037526250     xbdm:xbdm.DLL
 0003:00000258       \177xbdm_NULL_THUNK_DATA_DLA 0000000037526258     xbdm:xbdm.DLL
 0003:00000260       ?numAllocations@_CryMemoryManagerPoolHelper@@2HC 0000000037526260     CryLiveCreate.obj
 0003:00000264       ?requestedMemory@_CryMemoryManagerPoolHelper@@2JC 0000000037526264     CryLiveCreate.obj
 0003:00000268       ?freedMemory@_CryMemoryManagerPoolHelper@@2JC 0000000037526268     CryLiveCreate.obj
 0003:0000026c       ?allocatedMemory@_CryMemoryManagerPoolHelper@@2JC 000000003752626c     CryLiveCreate.obj
 0003:00000270       ?gEnv@@3PEAUSSystemGlobalEnvironment@@EA 0000000037526270     CryLiveCreate.obj
 0003:00000278       ?m_pFirst@Test@CryUnitTest@@2PEAU12@EA 0000000037526278     CryLiveCreate.obj
 0003:00000280       ?m_pLast@Test@CryUnitTest@@2PEAU12@EA 0000000037526280     CryLiveCreate.obj
 0003:00000288       ?g_pHeadToRegFactories@@3PEAUSRegFactoryNode@@EA 0000000037526288     CryLiveCreate.obj
 0003:00000290       ?g_bProfilerEnabled@@3_NA  0000000037526290     CryLiveCreate.obj
 0003:00000294       ?g_iTraceAllocations@@3HA  0000000037526294     CryLiveCreate.obj
 0003:00000298       ?_CryMalloc@_CryMemoryManagerPoolHelper@@2P6APEAX_KAEA_K0@ZEA 0000000037526298     CryLiveCreate.obj
 0003:000002a0       ?_CryGetMemSize@_CryMemoryManagerPoolHelper@@2P6A_KPEAX_K@ZEA 00000000375262a0     CryLiveCreate.obj
 0003:000002a8       ?_CryRealloc@_CryMemoryManagerPoolHelper@@2P6APEAXPEAX_KAEA_K21@ZEA 00000000375262a8     CryLiveCreate.obj
 0003:000002b0       ?_CryFree@_CryMemoryManagerPoolHelper@@2P6A_KPEAX_K@ZEA 00000000375262b0     CryLiveCreate.obj
 0003:000002b8       ?_CryCrtMalloc@_CryMemoryManagerPoolHelper@@2P6APEAX_K@ZEA 00000000375262b8     CryLiveCreate.obj
 0003:000002c0       ?_CryCrtRealloc@_CryMemoryManagerPoolHelper@@2P6APEAXPEAX_K@ZEA 00000000375262c0     CryLiveCreate.obj
 0003:000002c8       ?_CryCrtFree@_CryMemoryManagerPoolHelper@@2P6A_KPEAX@ZEA 00000000375262c8     CryLiveCreate.obj
 0003:000002d0       ?_CryCrtSize@_CryMemoryManagerPoolHelper@@2P6A_KPEAX@ZEA 00000000375262d0     CryLiveCreate.obj
 0003:000002d8       ?_CryGetIMemoryManagerInterface@_CryMemoryManagerPoolHelper@@2P6AXPEAPEAX@ZEA 00000000375262d8     CryLiveCreate.obj
 0003:000002e0       ?m_bInitialized@_CryMemoryManagerPoolHelper@@2HA 00000000375262e0     CryLiveCreate.obj
 0003:000002e4       ?g_random_generator@@3VCLCGRndGen@@A 00000000375262e4     CryLiveCreate.obj
 0003:000002f0       ?s_factory@CFactory@CEngineModule_CryLiveCreate@@0V12@A 00000000375262f0     CryLiveCreate.obj
 0003:00000348       ?s_used_memory@?1??_usedMemory@?$CryStringT@_W@@SA_K_J@Z@4_KA 0000000037526348     CryLiveCreate.obj
 0003:00000350       ?s_used_memory@?1??_usedMemory@?$CryStringT@D@@SA_K_J@Z@4_KA 0000000037526350     CryLiveCreate.obj
 0003:00000358       ?s_pMemReplay@?1??CryGetIMemReplay@@YAPEAUIMemReplay@@XZ@4PEAU2@EA 0000000037526358     CryLiveCreate.obj
 0003:00000360       ?s_dummyMemReplay@?1??CryGetIMemReplay@@YAPEAUIMemReplay@@XZ@4UCDummyMemReplay@@A 0000000037526360     CryLiveCreate.obj
 0003:00000368       ??_B?1??CryGetIMemReplay@@YAPEAUIMemReplay@@XZ@51 0000000037526368     CryLiveCreate.obj
 0003:00000370       ?supportedIIDs@?1???0CFactory@CEngineModule_CryLiveCreate@@AEAA@XZ@4PAUCryGUID@@A 0000000037526370     CryLiveCreate.obj
 0003:00000390       ?p@?1??CreateClassInstance@CFactory@CEngineModule_CryLiveCreate@@UEBA?AV?$shared_ptr@UICryUnknown@@@boost@@XZ@4V?$shared_ptr@VCEngineModule_CryLiveCreate@@@5@A 0000000037526390     CryLiveCreate.obj
 0003:000003a0       ??_B?1??CreateClassInstance@CFactory@CEngineModule_CryLiveCreate@@UEBA?AV?$shared_ptr@UICryUnknown@@@boost@@XZ@51 00000000375263a0     CryLiveCreate.obj
 0003:000003a8       __pfnDliFailureHook2       00000000375263a8     delayhlp.obj
 0003:000003b0       __pfnDliNotifyHook2        00000000375263b0     delayhlp.obj
 0003:000003b8       ?__puiHead@@3PEAUUnloadInfo@@EA 00000000375263b8     delayhlp.obj
 0003:000003c0       ?s_pEditorPcFactory@LiveCreate@@3PEAVPlatformHandlerFactory_EditorPC@1@EA 00000000375263c0     LiveCreate.obj
 0003:000003c8       ?s_pGamePcFactory@LiveCreate@@3PEAVPlatformHandlerFactory_GamePC@1@EA 00000000375263c8     LiveCreate.obj
 0003:000003d0       ?s_pX360Factory@LiveCreate@@3PEAVPlatformHandlerFactory_X360@1@EA 00000000375263d0     LiveCreate.obj
 0003:000003d8       ?s_pPS3Factory@LiveCreate@@3PEAVPlatformHandlerFactory_PS3@1@EA 00000000375263d8     LiveCreate.obj
 0003:000003e0       ?s_pCameraCtrler@LiveCreate@@3PEAVCameraController@1@EA 00000000375263e0     LiveCreate.obj
 0003:000003e8       ?s_pEntitiesCtrler@LiveCreate@@3PEAVEntitiesController@1@EA 00000000375263e8     LiveCreate.obj
 0003:000003f0       ?s_pCVarCtrler@LiveCreate@@3PEAVCVarController@1@EA 00000000375263f0     LiveCreate.obj
 0003:000003f8       ?s_pExecConStrCtrler@LiveCreate@@3PEAVExecuteConsoleStringController@1@EA 00000000375263f8     LiveCreate.obj
 0003:00000400       ?s_pFileChangeNotifyCtrler@LiveCreate@@3PEAVFileChangeNotifyController@1@EA 0000000037526400     LiveCreate.obj
 0003:00000408       ?s_pScreenshotCtrler@LiveCreate@@3PEAVScreenshotController@1@EA 0000000037526408     LiveCreate.obj
 0003:000004a8       ?s_pPS3Api@PlatformHandlerFactory_PS3@LiveCreate@@2PEAVPS3TmHelper@@EA 00000000375264a8     PlatformHandler_PS3.obj
 0003:000004c0       ?g_globalSections@?$Node_Alloc_Lock@$00$00@@2PAUInternalCriticalSectionDummy@@A 00000000375264c0     StdAfx.obj
 0003:00001540       ?m_bInitialized@?$Node_Alloc_Lock@$00$00@@2_NA 0000000037527540     StdAfx.obj
 0003:00001548       __hmod__xbdm_DLL           0000000037527548     xbdm:xbdm.DLL
 0003:00001558       ?__type_info_root_node@@3U__type_info_node@@A 0000000037527558     MSVCRT:tncleanup.obj
 0003:00001ae0       __@@_PchSym_@00@UdlipUwvexDUxlwvUgllohUkhDgnsvokvioryUcGEUkilurovUhgwzucOlyq@ 0000000037527ae0     PS3TmHelperLib:StdAfx.obj
 0003:00001ae8       ?s_refCount@PS3TmDynApi@@0_KA 0000000037527ae8     PS3TmHelperLib:PS3TmDynApi.obj
 0003:00001bf4       __native_startup_state     0000000037527bf4     <common>
 0003:00001bf8       __native_startup_lock      0000000037527bf8     <common>
 0003:00001c00       __dyn_tls_init_callback    0000000037527c00     <common>
 0003:00001c08       __onexitend                0000000037527c08     <common>
 0003:00001c10       __onexitbegin              0000000037527c10     <common>
 0005:00000000       ?m_Self@CrySimpleThreadSelf@@1PEAV1@EA 000000003752a000     CryLiveCreate.obj

 entry point at        0001:0001d118

 Static symbols

 0001:0001c550       ?DelayLoadXboxDevDLL@@YA_NXZ 000000003751d550 f   PlatformHandler_X360.obj
 0001:0001cd20       pre_c_init                 000000003751dd20 f   MSVCRT:crtdll.obj
 0001:0001cfdc       __DllMainCRTStartup        000000003751dfdc f   MSVCRT:crtdll.obj
 0001:0001d5b0       _onexit$fin$0              000000003751e5b0 f   MSVCRT:atonexit.obj
 0001:0001d5cb       __DllMainCRTStartup$filt$0 000000003751e5cb f   MSVCRT:crtdll.obj
 0001:0001d5fb       __DllMainCRTStartup$fin$1  000000003751e5fb f   MSVCRT:crtdll.obj
 0001:0001d620       _IsNonwritableInCurrentImage$filt$0 000000003751e620 f   MSVCRT:pesect.obj
 0001:0001d650       ??__Eg_random_generator@@YAXXZ 000000003751e650 f   CryLiveCreate.obj
 0001:0001d660       ??__Eg_system_event_listener_livecreate@@YAXXZ 000000003751e660 f   CryLiveCreate.obj
 0001:0001d670       ??__E?s_factory@CFactory@CEngineModule_CryLiveCreate@@0V12@A@@YAXXZ 000000003751e670 f   CryLiveCreate.obj
 0001:0001d690       ??__Es_testNullImplCompile@LiveCreate@@YAXXZ 000000003751e690 f   LiveCreate.obj
 0001:0001d6a0       ??__ECryUserInvalidID@@YAXXZ 000000003751e6a0 f   LiveCreateCtrl_Camera.obj
 0001:0001d6b0       ??__ECrySessionInvalidID@@YAXXZ 000000003751e6b0 f   LiveCreateCtrl_Camera.obj
 0001:0001d6c0       ??__ECryUserInvalidID@@YAXXZ 000000003751e6c0 f   LiveCreateCtrl_CVar.obj
 0001:0001d6d0       ??__ECrySessionInvalidID@@YAXXZ 000000003751e6d0 f   LiveCreateCtrl_CVar.obj
 0001:0001d6e0       ??__ECryUserInvalidID@@YAXXZ 000000003751e6e0 f   LiveCreateCtrl_Entities.obj
 0001:0001d6f0       ??__ECrySessionInvalidID@@YAXXZ 000000003751e6f0 f   LiveCreateCtrl_Entities.obj
 0001:0001d700       ??__EautoInitializer@@YAXXZ 000000003751e700 f   StdAfx.obj
 0001:0001d760       ??__Finstance@?1??Instance@PS3TmDynApi@@SAPEAV1@XZ@YAXXZ 000000003751e760 f    CIL library: CIL module
 0001:0001d790       ??__F?s_factory@CFactory@CEngineModule_CryLiveCreate@@0V12@A@@YAXXZ 000000003751e790 f   CryLiveCreate.obj
 0001:0001d7d0       ??__Fg_system_event_listener_livecreate@@YAXXZ 000000003751e7d0 f   CryLiveCreate.obj
 0001:0001d820       ??__Fs_testNullImplCompile@LiveCreate@@YAXXZ 000000003751e820 f   LiveCreate.obj
 0001:0001d830       ??__FCrySessionInvalidID@@YAXXZ 000000003751e830 f   LiveCreateCtrl_Camera.obj
 0001:0001d880       ??__FCryUserInvalidID@@YAXXZ 000000003751e880 f   LiveCreateCtrl_Camera.obj
 0001:0001d8d0       ??__FCrySessionInvalidID@@YAXXZ 000000003751e8d0 f   LiveCreateCtrl_CVar.obj
 0001:0001d920       ??__FCryUserInvalidID@@YAXXZ 000000003751e920 f   LiveCreateCtrl_CVar.obj
 0001:0001d970       ??__FCrySessionInvalidID@@YAXXZ 000000003751e970 f   LiveCreateCtrl_Entities.obj
 0001:0001d9c0       ??__FCryUserInvalidID@@YAXXZ 000000003751e9c0 f   LiveCreateCtrl_Entities.obj
 0001:0001da10       ??__FautoInitializer@@YAXXZ 000000003751ea10 f   StdAfx.obj
